******************************************************************************
                  TI ARM Linker PC v5.2.6                      
******************************************************************************
>> Linked Sun Nov 29 18:02:33 2015

OUTPUT FILE NAME:   <SimpleBLEPeripheral.out>
ENTRY POINT SYMBOL: "ResetISR"  address: 000043c9


MEMORY CONFIGURATION

         name            origin    length      used     unused   attr    fill
----------------------  --------  ---------  --------  --------  ----  --------
  FLASH                 00000000   0000dfff  00006d9a  00007265  R  X
  FLASH_LAST_PAGE       0001f000   00001000  00000058  00000fa8  R  X
  SRAM                  20000000   000043e7  000029cd  00001a1a  RW X


SEGMENT ALLOCATION MAP

run origin  load origin   length   init length attrs members
----------  ----------- ---------- ----------- ----- -------
00000000    00000000    00006da0   00006da0    r-x
  00000000    00000000    0000003c   0000003c    r-- .resetVecs
  0000003c    0000003c    000000c4   000000c4    r-x .text.1
  00000100    00000100    0000003c   0000003c    r-- .const:ti_sysbios_knl_Task_Object__PARAMS__C
  0000013c    0000013c    00000034   00000034    r-- .const:ti_sysbios_knl_Mailbox_Object__PARAMS__C
  00000170    00000170    00000030   00000030    r-- .const:ti_sysbios_family_arm_m3_Hwi_Object__PARAMS__C
  000001a0    000001a0    0000002c   0000002c    r-- .const:ti_sysbios_hal_Hwi_Object__PARAMS__C
  000001cc    000001cc    00000028   00000028    r-- .const:ti_sysbios_heaps_HeapMem_Module__FXNS__C
  000001f4    000001f4    00000028   00000028    r-- .const:ti_sysbios_knl_Swi_Object__PARAMS__C
  0000021c    0000021c    00000024   00000024    r-- .const:ti_sysbios_gates_GateHwi_Module__FXNS__C
  00000240    00000240    00000024   00000024    r-- .const:ti_sysbios_gates_GateMutex_Module__FXNS__C
  00000264    00000264    00000024   00000024    r-- .const:ti_sysbios_heaps_HeapMem_Object__PARAMS__C
  00000288    00000288    00000024   00000024    r-- .const:ti_sysbios_knl_Clock_Object__PARAMS__C
  000002ac    000002ac    00000024   00000024    r-- .const:ti_sysbios_knl_Semaphore_Object__PARAMS__C
  000002d0    000002d0    00000020   00000020    r-- .const:ti_sysbios_family_arm_m3_Hwi_Object__DESC__C
  000002f0    000002f0    00000020   00000020    r-- .const:ti_sysbios_gates_GateHwi_Object__DESC__C
  00000310    00000310    00000020   00000020    r-- .const:ti_sysbios_gates_GateMutex_Object__DESC__C
  00000330    00000330    00000020   00000020    r-- .const:ti_sysbios_hal_Hwi_Object__DESC__C
  00000350    00000350    00000020   00000020    r-- .const:ti_sysbios_heaps_HeapMem_Object__DESC__C
  00000370    00000370    00000020   00000020    r-- .const:ti_sysbios_knl_Clock_Object__DESC__C
  00000390    00000390    00000020   00000020    r-- .const:ti_sysbios_knl_Mailbox_Object__DESC__C
  000003b0    000003b0    00000020   00000020    r-- .const:ti_sysbios_knl_Queue_Object__DESC__C
  000003d0    000003d0    00000020   00000020    r-- .const:ti_sysbios_knl_Semaphore_Object__DESC__C
  000003f0    000003f0    00000020   00000020    r-- .const:ti_sysbios_knl_Swi_Object__DESC__C
  00000410    00000410    00000020   00000020    r-- .const:ti_sysbios_knl_Task_Object__DESC__C
  00000430    00000430    00000018   00000018    r-- .const:ti_sysbios_gates_GateHwi_Object__PARAMS__C
  00000448    00000448    00000018   00000018    r-- .const:ti_sysbios_gates_GateMutex_Object__PARAMS__C
  00000460    00000460    00000018   00000018    r-- .const:ti_sysbios_knl_Queue_Object__PARAMS__C
  00000478    00000478    00000008   00000008    r-- .const:ti_sysbios_knl_Idle_funcList__C
  00000480    00000480    00000004   00000004    r-x .text.2
  00000484    00000484    00000004   00000004    r-- .const:ti_sysbios_family_arm_cc26xx_Timer_startupNeeded__C
  00000488    00000488    00000004   00000004    r-- .const:ti_sysbios_family_arm_m3_Hwi_E_alreadyDefined__C
  0000048c    0000048c    00000004   00000004    r-- .const:ti_sysbios_family_arm_m3_Hwi_E_hwiLimitExceeded__C
  00000490    00000490    00000004   00000004    r-- .const:ti_sysbios_family_arm_m3_Hwi_NUM_INTERRUPTS__C
  00000494    00000494    00000004   00000004    r-- .const:ti_sysbios_family_arm_m3_Hwi_Object__count__C
  00000498    00000498    00000004   00000004    r-- .const:ti_sysbios_family_arm_m3_Hwi_Object__table__C
  0000049c    0000049c    00000004   00000004    r-- .const:ti_sysbios_family_arm_m3_Hwi_ccr__C
  000004a0    000004a0    00000004   00000004    r-- .const:ti_sysbios_family_arm_m3_Hwi_excHandlerFunc__C
  000004a4    000004a4    00000004   00000004    r-- .const:ti_sysbios_family_arm_m3_Hwi_nullIsrFunc__C
  000004a8    000004a8    00000004   00000004    r-- .const:ti_sysbios_family_arm_m3_Hwi_numSparseInterrupts__C
  000004ac    000004ac    00000004   00000004    r-- .const:ti_sysbios_family_arm_m3_Hwi_priGroup__C
  000004b0    000004b0    00000004   00000004    r-- .const:ti_sysbios_family_arm_m3_TaskSupport_stackAlignment__C
  000004b4    000004b4    00000004   00000004    r-- .const:ti_sysbios_heaps_HeapMem_E_memory__C
  000004b8    000004b8    00000004   00000004    r-- .const:ti_sysbios_heaps_HeapMem_Module__gateObj__C
  000004bc    000004bc    00000004   00000004    r-- .const:ti_sysbios_heaps_HeapMem_Object__count__C
  000004c0    000004c0    00000004   00000004    r-- .const:ti_sysbios_heaps_HeapMem_Object__table__C
  000004c4    000004c4    00000004   00000004    r-- .const:ti_sysbios_heaps_HeapMem_reqAlign__C
  000004c8    000004c8    00000004   00000004    r-- .const:ti_sysbios_knl_Clock_serviceMargin__C
  000004cc    000004cc    00000004   00000004    r-- .const:ti_sysbios_knl_Mailbox_Object__count__C
  000004d0    000004d0    00000004   00000004    r-- .const:ti_sysbios_knl_Mailbox_Object__table__C
  000004d4    000004d4    00000004   00000004    r-- .const:ti_sysbios_knl_Queue_Object__count__C
  000004d8    000004d8    00000004   00000004    r-- .const:ti_sysbios_knl_Queue_Object__table__C
  000004dc    000004dc    00000004   00000004    r-- .const:ti_sysbios_knl_Swi_Object__count__C
  000004e0    000004e0    00000004   00000004    r-- .const:ti_sysbios_knl_Swi_Object__table__C
  000004e4    000004e4    00000004   00000004    r-- .const:ti_sysbios_knl_Swi_numPriorities__C
  000004e8    000004e8    00000004   00000004    r-- .const:ti_sysbios_knl_Task_Object__count__C
  000004ec    000004ec    00000004   00000004    r-- .const:ti_sysbios_knl_Task_Object__table__C
  000004f0    000004f0    00000004   00000004    r-- .const:ti_sysbios_knl_Task_allBlockedFunc__C
  000004f4    000004f4    00000004   00000004    r-- .const:ti_sysbios_knl_Task_defaultStackHeap__C
  000004f8    000004f8    00000004   00000004    r-- .const:ti_sysbios_knl_Task_defaultStackSize__C
  000004fc    000004fc    00000004   00000004    r-- .const:ti_sysbios_knl_Task_numConstructedTasks__C
  00000500    00000500    00000002   00000002    r-x .text.3
  00000502    00000502    00000002   00000002    r-- .const:ti_sysbios_family_arm_cc26xx_Timer_Module__id__C
  00000504    00000504    00000002   00000002    r-- .const:ti_sysbios_family_arm_cc26xx_TimestampProvider_useClockTimer__C
  00000506    00000506    00000002   00000002    r-- .const:ti_sysbios_family_arm_m3_Hwi_Module__id__C
  00000508    00000508    00000002   00000002    r-- .const:ti_sysbios_gates_GateHwi_Module__id__C
  0000050a    0000050a    00000002   00000002    r-- .const:ti_sysbios_gates_GateMutex_Module__id__C
  0000050c    0000050c    00000002   00000002    r-- .const:ti_sysbios_heaps_HeapMem_Module__id__C
  0000050e    0000050e    00000002   00000002    r-- .const:ti_sysbios_knl_Task_initStackFlag__C
  00000510    00000510    00000001   00000001    r-- .const:ti_sysbios_knl_Clock_tickMode__C
  00000514    00000514    00000008   00000008    r-- .const:xdc_runtime_Startup_firstFxns__C
  0000051c    0000051c    00000008   00000008    r-- .const:xdc_runtime_Startup_lastFxns__C
  00000524    00000524    00000004   00000004    r-- .const:xdc_runtime_Assert_E_assertFailed__C
  00000528    00000528    00000004   00000004    r-- .const:xdc_runtime_Error_E_memory__C
  0000052c    0000052c    00000004   00000004    r-- .const:xdc_runtime_Error_policyFxn__C
  00000530    00000530    00000004   00000004    r-- .const:xdc_runtime_IGateProvider_Interface__BASE__C
  00000534    00000534    00000004   00000004    r-- .const:xdc_runtime_IHeap_Interface__BASE__C
  00000538    00000538    00000004   00000004    r-- .const:xdc_runtime_IModule_Interface__BASE__C
  0000053c    0000053c    00000004   00000004    r-- .const:xdc_runtime_Main_Module__diagsEnabled__C
  00000540    00000540    00000004   00000004    r-- .const:xdc_runtime_Main_Module__diagsIncluded__C
  00000544    00000544    00000004   00000004    r-- .const:xdc_runtime_Main_Module__diagsMask__C
  00000548    00000548    00000004   00000004    r-- .const:xdc_runtime_Memory_defaultHeapInstance__C
  0000054c    0000054c    00000004   00000004    r-- .const:xdc_runtime_Startup_execImpl__C
  00000550    00000550    00000004   00000004    r-- .const:xdc_runtime_Startup_maxPasses__C
  00000554    00000554    00000004   00000004    r-- .const:xdc_runtime_Startup_sfxnRts__C
  00000558    00000558    00000004   00000004    r-- .const:xdc_runtime_Startup_sfxnTab__C
  0000055c    0000055c    00000004   00000004    r-- .const:xdc_runtime_Startup_startModsFxn__C
  00000560    00000560    00000004   00000004    r-- .const:xdc_runtime_SysCallback_abortFxn__C
  00000564    00000564    00000004   00000004    r-- .const:xdc_runtime_SysCallback_exitFxn__C
  00000568    00000568    00000004   00000004    r-- .const:xdc_runtime_System_abortFxn__C
  0000056c    0000056c    00000004   00000004    r-- .const:xdc_runtime_System_exitFxn__C
  00000570    00000570    00000004   00000004    r-- .const:xdc_runtime_System_maxAtexitHandlers__C
  00000574    00000574    00000004   00000004    r-- .const:xdc_runtime_Text_charTab__C
  00000578    00000578    00000004   00000004    r-- .const:xdc_runtime_Text_nameEmpty__C
  0000057c    0000057c    00000004   00000004    r-- .const:xdc_runtime_Text_nameStatic__C
  00000580    00000580    00000004   00000004    r-- .const:xdc_runtime_Text_nameUnknown__C
  00000584    00000584    00000002   00000002    r-- .const:xdc_runtime_Main_Module__id__C
  00000586    00000586    00000002   00000002    r-- .const:xdc_runtime_Memory_Module__id__C
  00000588    00000588    00000002   00000002    r-- .const:xdc_runtime_Text_charCnt__C
  0000058a    0000058a    00000002   00000002    r-- .const:xdc_runtime_Text_isLoaded__C
  0000058c    0000058c    00000001   00000001    r-- .const:xdc_runtime_Error_policy__C
  00000590    00000590    00000004   00000004    r-- .const:ti_sysbios_rom_ROM_AONRTCChannelEnable
  00000594    00000594    00000004   00000004    r-- .const:ti_sysbios_rom_ROM_AONRTCCompareValueSet
  00000598    00000598    00000004   00000004    r-- .const:ti_sysbios_rom_ROM_AONRTCCurrentCompareValueGet
  0000059c    0000059c    00000004   00000004    r-- .const:ti_sysbios_rom_ROM_AONRTCEventClear
  000005a0    000005a0    00000004   00000004    r-- .const:ti_sysbios_rom_ROM_ti_sysbios_family_arm_cc26xx_Timer_getCount64__E
  000005a4    000005a4    00000004   00000004    r-- .const:ti_sysbios_rom_ROM_ti_sysbios_family_arm_cc26xx_Timer_getCurrentTick__E
  000005a8    000005a8    00000004   00000004    r-- .const:ti_sysbios_rom_ROM_ti_sysbios_family_arm_cc26xx_Timer_getMaxTicks__E
  000005ac    000005ac    00000004   00000004    r-- .const:ti_sysbios_rom_ROM_ti_sysbios_family_arm_cc26xx_Timer_initDevice__I
  000005b0    000005b0    00000004   00000004    r-- .const:ti_sysbios_rom_ROM_ti_sysbios_family_arm_cc26xx_Timer_setNextTick__E
  000005b4    000005b4    00000004   00000004    r-- .const:ti_sysbios_rom_ROM_ti_sysbios_family_arm_cc26xx_Timer_setThreshold__I
  000005b8    000005b8    00000004   00000004    r-- .const:ti_sysbios_rom_ROM_ti_sysbios_family_arm_cc26xx_Timer_start__E
  000005bc    000005bc    00000004   00000004    r-- .const:ti_sysbios_rom_ROM_ti_sysbios_family_arm_cc26xx_TimestampProvider_get32__E
  000005c0    000005c0    00000004   00000004    r-- .const:ti_sysbios_rom_ROM_xdc_runtime_Startup_getState__I
  000005c4    000005c4    00000004   00000004    r-- .const:ti_sysbios_rom_ROM_xdc_runtime_System_SupportProxy_abort__E
  000005c8    000005c8    00000004   00000004    r-- .const:ti_sysbios_rom_ROM_xdc_runtime_System_SupportProxy_exit__E
  000005cc    000005cc    00000004   00000004    r-- .const:ti_sysbios_gates_GateMutex_Instance_State_sem__O
  000005d0    000005d0    00000004   00000004    r-- .const:ti_sysbios_knl_Clock_Module_State_clockQ__O
  000005d4    000005d4    00000004   00000004    r-- .const:ti_sysbios_knl_Mailbox_Instance_State_dataQue__O
  000005d8    000005d8    00000004   00000004    r-- .const:ti_sysbios_knl_Mailbox_Instance_State_dataSem__O
  000005dc    000005dc    00000004   00000004    r-- .const:ti_sysbios_knl_Mailbox_Instance_State_freeQue__O
  000005e0    000005e0    00000004   00000004    r-- .const:ti_sysbios_knl_Mailbox_Instance_State_freeSem__O
  000005e4    000005e4    00000004   00000004    r-- .const:ti_sysbios_knl_Semaphore_Instance_State_pendQ__O
  000005e8    000005e8    00000004   00000004    r-- .const:ti_sysbios_knl_Task_Module_State_inactiveQ__O
  000005ec    000005ec    00005d70   00005d70    r-x .text.4
  0000635c    0000635c    00000264   00000264    r-- .const
  000065c0    000065c0    000007e0   000007e0    r-- .cinit
0001ffa8    0001ffa8    00000058   00000058    r--
  0001ffa8    0001ffa8    00000058   00000058    r-- .ccfg
20000000    20000000    000000c8   00000000    rw-
  20000000    20000000    000000c8   00000000    rw- .vecs
20000100    20000100    00002510   00000000    rw-
  20000100    20000100    00000044   00000000    rw- .data:ti_sysbios_knl_Task_Module__state__V
  20000144    20000144    00000034   00000000    rw- .data:ti_sysbios_family_arm_m3_Hwi_Module__state__V
  20000178    20000178    0000002c   00000000    rw- .data:ti_sysbios_knl_Clock_Module__state__V
  200001a4    200001a4    00000024   00000000    rw- .data:ti_sysbios_BIOS_Module__state__V
  200001c8    200001c8    0000001c   00000000    rw- .data:ti_sysbios_knl_Swi_Module__state__V
  200001e4    200001e4    00000008   00000000    rw- .data:ti_sysbios_family_arm_cc26xx_Timer_Module__state__V
  200001ec    200001ec    00000004   00000000    rw- .data:ti_sysbios_family_arm_cc26xx_TimestampProvider_Module__state__V
  200001f0    200001f0    00000008   00000000    rw- .data:xdc_runtime_Startup_Module__state__V
  200001f8    200001f8    00000008   00000000    rw- .data:xdc_runtime_System_Module__state__V
  20000200    20000200    00000004   00000000    rw- .data:xdc_runtime_Memory_Module__state__V
  20000208    20000208    000014b1   00000000    rw- .bss
  200016c0    200016c0    00000f50   00000000    rw- .data
20003fe4    20003fe4    00000400   00000000    rw-
  20003fe4    20003fe4    00000400   00000000    rw- .stack


SECTION ALLOCATION MAP

 output                                  attributes/
section   page    origin      length       input sections
--------  ----  ----------  ----------   ----------------
.resetVecs 
*          0    00000000    0000003c     
                  00000000    0000003c     appBLE_pem3.oem3 (.resetVecs)

.text.1    0    0000003c    000000c4     
                  0000003c    000000b8     simpleBLEPeripheral.obj (.text:SimpleBLEPeripheral_performPeriodicMtr$21)
                  000000f4    00000008     (.tramp.ti_sysbios_knl_Semaphore_pend__E.1)
                  000000fc    00000004     ICallBleAPI.obj (.text:GATTServApp_AddService)

.const:ti_sysbios_knl_Task_Object__PARAMS__C 
*          0    00000100    0000003c     
                  00000100    0000003c     appBLE_pem3.oem3 (.const:ti_sysbios_knl_Task_Object__PARAMS__C)

.const:ti_sysbios_knl_Mailbox_Object__PARAMS__C 
*          0    0000013c    00000034     
                  0000013c    00000034     appBLE_pem3.oem3 (.const:ti_sysbios_knl_Mailbox_Object__PARAMS__C)

.const:ti_sysbios_family_arm_m3_Hwi_Object__PARAMS__C 
*          0    00000170    00000030     
                  00000170    00000030     appBLE_pem3.oem3 (.const:ti_sysbios_family_arm_m3_Hwi_Object__PARAMS__C)

.const:ti_sysbios_hal_Hwi_Object__PARAMS__C 
*          0    000001a0    0000002c     
                  000001a0    0000002c     appBLE_pem3.oem3 (.const:ti_sysbios_hal_Hwi_Object__PARAMS__C)

.const:ti_sysbios_heaps_HeapMem_Module__FXNS__C 
*          0    000001cc    00000028     
                  000001cc    00000028     appBLE_pem3.oem3 (.const:ti_sysbios_heaps_HeapMem_Module__FXNS__C)

.const:ti_sysbios_knl_Swi_Object__PARAMS__C 
*          0    000001f4    00000028     
                  000001f4    00000028     appBLE_pem3.oem3 (.const:ti_sysbios_knl_Swi_Object__PARAMS__C)

.const:ti_sysbios_gates_GateHwi_Module__FXNS__C 
*          0    0000021c    00000024     
                  0000021c    00000024     appBLE_pem3.oem3 (.const:ti_sysbios_gates_GateHwi_Module__FXNS__C)

.const:ti_sysbios_gates_GateMutex_Module__FXNS__C 
*          0    00000240    00000024     
                  00000240    00000024     appBLE_pem3.oem3 (.const:ti_sysbios_gates_GateMutex_Module__FXNS__C)

.const:ti_sysbios_heaps_HeapMem_Object__PARAMS__C 
*          0    00000264    00000024     
                  00000264    00000024     appBLE_pem3.oem3 (.const:ti_sysbios_heaps_HeapMem_Object__PARAMS__C)

.const:ti_sysbios_knl_Clock_Object__PARAMS__C 
*          0    00000288    00000024     
                  00000288    00000024     appBLE_pem3.oem3 (.const:ti_sysbios_knl_Clock_Object__PARAMS__C)

.const:ti_sysbios_knl_Semaphore_Object__PARAMS__C 
*          0    000002ac    00000024     
                  000002ac    00000024     appBLE_pem3.oem3 (.const:ti_sysbios_knl_Semaphore_Object__PARAMS__C)

.const:ti_sysbios_family_arm_m3_Hwi_Object__DESC__C 
*          0    000002d0    00000020     
                  000002d0    00000020     appBLE_pem3.oem3 (.const:ti_sysbios_family_arm_m3_Hwi_Object__DESC__C)

.const:ti_sysbios_gates_GateHwi_Object__DESC__C 
*          0    000002f0    00000020     
                  000002f0    00000020     appBLE_pem3.oem3 (.const:ti_sysbios_gates_GateHwi_Object__DESC__C)

.const:ti_sysbios_gates_GateMutex_Object__DESC__C 
*          0    00000310    00000020     
                  00000310    00000020     appBLE_pem3.oem3 (.const:ti_sysbios_gates_GateMutex_Object__DESC__C)

.const:ti_sysbios_hal_Hwi_Object__DESC__C 
*          0    00000330    00000020     
                  00000330    00000020     appBLE_pem3.oem3 (.const:ti_sysbios_hal_Hwi_Object__DESC__C)

.const:ti_sysbios_heaps_HeapMem_Object__DESC__C 
*          0    00000350    00000020     
                  00000350    00000020     appBLE_pem3.oem3 (.const:ti_sysbios_heaps_HeapMem_Object__DESC__C)

.const:ti_sysbios_knl_Clock_Object__DESC__C 
*          0    00000370    00000020     
                  00000370    00000020     appBLE_pem3.oem3 (.const:ti_sysbios_knl_Clock_Object__DESC__C)

.const:ti_sysbios_knl_Mailbox_Object__DESC__C 
*          0    00000390    00000020     
                  00000390    00000020     appBLE_pem3.oem3 (.const:ti_sysbios_knl_Mailbox_Object__DESC__C)

.const:ti_sysbios_knl_Queue_Object__DESC__C 
*          0    000003b0    00000020     
                  000003b0    00000020     appBLE_pem3.oem3 (.const:ti_sysbios_knl_Queue_Object__DESC__C)

.const:ti_sysbios_knl_Semaphore_Object__DESC__C 
*          0    000003d0    00000020     
                  000003d0    00000020     appBLE_pem3.oem3 (.const:ti_sysbios_knl_Semaphore_Object__DESC__C)

.const:ti_sysbios_knl_Swi_Object__DESC__C 
*          0    000003f0    00000020     
                  000003f0    00000020     appBLE_pem3.oem3 (.const:ti_sysbios_knl_Swi_Object__DESC__C)

.const:ti_sysbios_knl_Task_Object__DESC__C 
*          0    00000410    00000020     
                  00000410    00000020     appBLE_pem3.oem3 (.const:ti_sysbios_knl_Task_Object__DESC__C)

.const:ti_sysbios_gates_GateHwi_Object__PARAMS__C 
*          0    00000430    00000018     
                  00000430    00000018     appBLE_pem3.oem3 (.const:ti_sysbios_gates_GateHwi_Object__PARAMS__C)

.const:ti_sysbios_gates_GateMutex_Object__PARAMS__C 
*          0    00000448    00000018     
                  00000448    00000018     appBLE_pem3.oem3 (.const:ti_sysbios_gates_GateMutex_Object__PARAMS__C)

.const:ti_sysbios_knl_Queue_Object__PARAMS__C 
*          0    00000460    00000018     
                  00000460    00000018     appBLE_pem3.oem3 (.const:ti_sysbios_knl_Queue_Object__PARAMS__C)

.const:ti_sysbios_knl_Idle_funcList__C 
*          0    00000478    00000008     
                  00000478    00000008     appBLE_pem3.oem3 (.const:ti_sysbios_knl_Idle_funcList__C)

.text.2    0    00000480    00000004     
                  00000480    00000004     ICall.obj (.text:ICall_primAbort$10)

.const:ti_sysbios_family_arm_cc26xx_Timer_startupNeeded__C 
*          0    00000484    00000004     
                  00000484    00000004     appBLE_pem3.oem3 (.const:ti_sysbios_family_arm_cc26xx_Timer_startupNeeded__C)

.const:ti_sysbios_family_arm_m3_Hwi_E_alreadyDefined__C 
*          0    00000488    00000004     
                  00000488    00000004     appBLE_pem3.oem3 (.const:ti_sysbios_family_arm_m3_Hwi_E_alreadyDefined__C)

.const:ti_sysbios_family_arm_m3_Hwi_E_hwiLimitExceeded__C 
*          0    0000048c    00000004     
                  0000048c    00000004     appBLE_pem3.oem3 (.const:ti_sysbios_family_arm_m3_Hwi_E_hwiLimitExceeded__C)

.const:ti_sysbios_family_arm_m3_Hwi_NUM_INTERRUPTS__C 
*          0    00000490    00000004     
                  00000490    00000004     appBLE_pem3.oem3 (.const:ti_sysbios_family_arm_m3_Hwi_NUM_INTERRUPTS__C)

.const:ti_sysbios_family_arm_m3_Hwi_Object__count__C 
*          0    00000494    00000004     
                  00000494    00000004     appBLE_pem3.oem3 (.const:ti_sysbios_family_arm_m3_Hwi_Object__count__C)

.const:ti_sysbios_family_arm_m3_Hwi_Object__table__C 
*          0    00000498    00000004     
                  00000498    00000004     appBLE_pem3.oem3 (.const:ti_sysbios_family_arm_m3_Hwi_Object__table__C)

.const:ti_sysbios_family_arm_m3_Hwi_ccr__C 
*          0    0000049c    00000004     
                  0000049c    00000004     appBLE_pem3.oem3 (.const:ti_sysbios_family_arm_m3_Hwi_ccr__C)

.const:ti_sysbios_family_arm_m3_Hwi_excHandlerFunc__C 
*          0    000004a0    00000004     
                  000004a0    00000004     appBLE_pem3.oem3 (.const:ti_sysbios_family_arm_m3_Hwi_excHandlerFunc__C)

.const:ti_sysbios_family_arm_m3_Hwi_nullIsrFunc__C 
*          0    000004a4    00000004     
                  000004a4    00000004     appBLE_pem3.oem3 (.const:ti_sysbios_family_arm_m3_Hwi_nullIsrFunc__C)

.const:ti_sysbios_family_arm_m3_Hwi_numSparseInterrupts__C 
*          0    000004a8    00000004     
                  000004a8    00000004     appBLE_pem3.oem3 (.const:ti_sysbios_family_arm_m3_Hwi_numSparseInterrupts__C)

.const:ti_sysbios_family_arm_m3_Hwi_priGroup__C 
*          0    000004ac    00000004     
                  000004ac    00000004     appBLE_pem3.oem3 (.const:ti_sysbios_family_arm_m3_Hwi_priGroup__C)

.const:ti_sysbios_family_arm_m3_TaskSupport_stackAlignment__C 
*          0    000004b0    00000004     
                  000004b0    00000004     appBLE_pem3.oem3 (.const:ti_sysbios_family_arm_m3_TaskSupport_stackAlignment__C)

.const:ti_sysbios_heaps_HeapMem_E_memory__C 
*          0    000004b4    00000004     
                  000004b4    00000004     appBLE_pem3.oem3 (.const:ti_sysbios_heaps_HeapMem_E_memory__C)

.const:ti_sysbios_heaps_HeapMem_Module__gateObj__C 
*          0    000004b8    00000004     
                  000004b8    00000004     appBLE_pem3.oem3 (.const:ti_sysbios_heaps_HeapMem_Module__gateObj__C)

.const:ti_sysbios_heaps_HeapMem_Object__count__C 
*          0    000004bc    00000004     
                  000004bc    00000004     appBLE_pem3.oem3 (.const:ti_sysbios_heaps_HeapMem_Object__count__C)

.const:ti_sysbios_heaps_HeapMem_Object__table__C 
*          0    000004c0    00000004     
                  000004c0    00000004     appBLE_pem3.oem3 (.const:ti_sysbios_heaps_HeapMem_Object__table__C)

.const:ti_sysbios_heaps_HeapMem_reqAlign__C 
*          0    000004c4    00000004     
                  000004c4    00000004     appBLE_pem3.oem3 (.const:ti_sysbios_heaps_HeapMem_reqAlign__C)

.const:ti_sysbios_knl_Clock_serviceMargin__C 
*          0    000004c8    00000004     
                  000004c8    00000004     appBLE_pem3.oem3 (.const:ti_sysbios_knl_Clock_serviceMargin__C)

.const:ti_sysbios_knl_Mailbox_Object__count__C 
*          0    000004cc    00000004     
                  000004cc    00000004     appBLE_pem3.oem3 (.const:ti_sysbios_knl_Mailbox_Object__count__C)

.const:ti_sysbios_knl_Mailbox_Object__table__C 
*          0    000004d0    00000004     
                  000004d0    00000004     appBLE_pem3.oem3 (.const:ti_sysbios_knl_Mailbox_Object__table__C)

.const:ti_sysbios_knl_Queue_Object__count__C 
*          0    000004d4    00000004     
                  000004d4    00000004     appBLE_pem3.oem3 (.const:ti_sysbios_knl_Queue_Object__count__C)

.const:ti_sysbios_knl_Queue_Object__table__C 
*          0    000004d8    00000004     
                  000004d8    00000004     appBLE_pem3.oem3 (.const:ti_sysbios_knl_Queue_Object__table__C)

.const:ti_sysbios_knl_Swi_Object__count__C 
*          0    000004dc    00000004     
                  000004dc    00000004     appBLE_pem3.oem3 (.const:ti_sysbios_knl_Swi_Object__count__C)

.const:ti_sysbios_knl_Swi_Object__table__C 
*          0    000004e0    00000004     
                  000004e0    00000004     appBLE_pem3.oem3 (.const:ti_sysbios_knl_Swi_Object__table__C)

.const:ti_sysbios_knl_Swi_numPriorities__C 
*          0    000004e4    00000004     
                  000004e4    00000004     appBLE_pem3.oem3 (.const:ti_sysbios_knl_Swi_numPriorities__C)

.const:ti_sysbios_knl_Task_Object__count__C 
*          0    000004e8    00000004     
                  000004e8    00000004     appBLE_pem3.oem3 (.const:ti_sysbios_knl_Task_Object__count__C)

.const:ti_sysbios_knl_Task_Object__table__C 
*          0    000004ec    00000004     
                  000004ec    00000004     appBLE_pem3.oem3 (.const:ti_sysbios_knl_Task_Object__table__C)

.const:ti_sysbios_knl_Task_allBlockedFunc__C 
*          0    000004f0    00000004     
                  000004f0    00000004     appBLE_pem3.oem3 (.const:ti_sysbios_knl_Task_allBlockedFunc__C)

.const:ti_sysbios_knl_Task_defaultStackHeap__C 
*          0    000004f4    00000004     
                  000004f4    00000004     appBLE_pem3.oem3 (.const:ti_sysbios_knl_Task_defaultStackHeap__C)

.const:ti_sysbios_knl_Task_defaultStackSize__C 
*          0    000004f8    00000004     
                  000004f8    00000004     appBLE_pem3.oem3 (.const:ti_sysbios_knl_Task_defaultStackSize__C)

.const:ti_sysbios_knl_Task_numConstructedTasks__C 
*          0    000004fc    00000004     
                  000004fc    00000004     appBLE_pem3.oem3 (.const:ti_sysbios_knl_Task_numConstructedTasks__C)

.text.3    0    00000500    00000002     
                  00000500    00000002     appBLE_pem3.oem3 (.text:ti_sysbios_BIOS_nullFunc__I)

.const:ti_sysbios_family_arm_cc26xx_Timer_Module__id__C 
*          0    00000502    00000002     
                  00000502    00000002     appBLE_pem3.oem3 (.const:ti_sysbios_family_arm_cc26xx_Timer_Module__id__C)

.const:ti_sysbios_family_arm_cc26xx_TimestampProvider_useClockTimer__C 
*          0    00000504    00000002     
                  00000504    00000002     appBLE_pem3.oem3 (.const:ti_sysbios_family_arm_cc26xx_TimestampProvider_useClockTimer__C)

.const:ti_sysbios_family_arm_m3_Hwi_Module__id__C 
*          0    00000506    00000002     
                  00000506    00000002     appBLE_pem3.oem3 (.const:ti_sysbios_family_arm_m3_Hwi_Module__id__C)

.const:ti_sysbios_gates_GateHwi_Module__id__C 
*          0    00000508    00000002     
                  00000508    00000002     appBLE_pem3.oem3 (.const:ti_sysbios_gates_GateHwi_Module__id__C)

.const:ti_sysbios_gates_GateMutex_Module__id__C 
*          0    0000050a    00000002     
                  0000050a    00000002     appBLE_pem3.oem3 (.const:ti_sysbios_gates_GateMutex_Module__id__C)

.const:ti_sysbios_heaps_HeapMem_Module__id__C 
*          0    0000050c    00000002     
                  0000050c    00000002     appBLE_pem3.oem3 (.const:ti_sysbios_heaps_HeapMem_Module__id__C)

.const:ti_sysbios_knl_Task_initStackFlag__C 
*          0    0000050e    00000002     
                  0000050e    00000002     appBLE_pem3.oem3 (.const:ti_sysbios_knl_Task_initStackFlag__C)

.const:ti_sysbios_knl_Clock_tickMode__C 
*          0    00000510    00000001     
                  00000510    00000001     appBLE_pem3.oem3 (.const:ti_sysbios_knl_Clock_tickMode__C)

.const:xdc_runtime_Startup_firstFxns__C 
*          0    00000514    00000008     
                  00000514    00000008     appBLE_pem3.oem3 (.const:xdc_runtime_Startup_firstFxns__C)

.const:xdc_runtime_Startup_lastFxns__C 
*          0    0000051c    00000008     
                  0000051c    00000008     appBLE_pem3.oem3 (.const:xdc_runtime_Startup_lastFxns__C)

.const:xdc_runtime_Assert_E_assertFailed__C 
*          0    00000524    00000004     
                  00000524    00000004     appBLE_pem3.oem3 (.const:xdc_runtime_Assert_E_assertFailed__C)

.const:xdc_runtime_Error_E_memory__C 
*          0    00000528    00000004     
                  00000528    00000004     appBLE_pem3.oem3 (.const:xdc_runtime_Error_E_memory__C)

.const:xdc_runtime_Error_policyFxn__C 
*          0    0000052c    00000004     
                  0000052c    00000004     appBLE_pem3.oem3 (.const:xdc_runtime_Error_policyFxn__C)

.const:xdc_runtime_IGateProvider_Interface__BASE__C 
*          0    00000530    00000004     
                  00000530    00000004     appBLE_pem3.oem3 (.const:xdc_runtime_IGateProvider_Interface__BASE__C)

.const:xdc_runtime_IHeap_Interface__BASE__C 
*          0    00000534    00000004     
                  00000534    00000004     appBLE_pem3.oem3 (.const:xdc_runtime_IHeap_Interface__BASE__C)

.const:xdc_runtime_IModule_Interface__BASE__C 
*          0    00000538    00000004     
                  00000538    00000004     appBLE_pem3.oem3 (.const:xdc_runtime_IModule_Interface__BASE__C)

.const:xdc_runtime_Main_Module__diagsEnabled__C 
*          0    0000053c    00000004     
                  0000053c    00000004     appBLE_pem3.oem3 (.const:xdc_runtime_Main_Module__diagsEnabled__C)

.const:xdc_runtime_Main_Module__diagsIncluded__C 
*          0    00000540    00000004     
                  00000540    00000004     appBLE_pem3.oem3 (.const:xdc_runtime_Main_Module__diagsIncluded__C)

.const:xdc_runtime_Main_Module__diagsMask__C 
*          0    00000544    00000004     
                  00000544    00000004     appBLE_pem3.oem3 (.const:xdc_runtime_Main_Module__diagsMask__C)

.const:xdc_runtime_Memory_defaultHeapInstance__C 
*          0    00000548    00000004     
                  00000548    00000004     appBLE_pem3.oem3 (.const:xdc_runtime_Memory_defaultHeapInstance__C)

.const:xdc_runtime_Startup_execImpl__C 
*          0    0000054c    00000004     
                  0000054c    00000004     appBLE_pem3.oem3 (.const:xdc_runtime_Startup_execImpl__C)

.const:xdc_runtime_Startup_maxPasses__C 
*          0    00000550    00000004     
                  00000550    00000004     appBLE_pem3.oem3 (.const:xdc_runtime_Startup_maxPasses__C)

.const:xdc_runtime_Startup_sfxnRts__C 
*          0    00000554    00000004     
                  00000554    00000004     appBLE_pem3.oem3 (.const:xdc_runtime_Startup_sfxnRts__C)

.const:xdc_runtime_Startup_sfxnTab__C 
*          0    00000558    00000004     
                  00000558    00000004     appBLE_pem3.oem3 (.const:xdc_runtime_Startup_sfxnTab__C)

.const:xdc_runtime_Startup_startModsFxn__C 
*          0    0000055c    00000004     
                  0000055c    00000004     appBLE_pem3.oem3 (.const:xdc_runtime_Startup_startModsFxn__C)

.const:xdc_runtime_SysCallback_abortFxn__C 
*          0    00000560    00000004     
                  00000560    00000004     appBLE_pem3.oem3 (.const:xdc_runtime_SysCallback_abortFxn__C)

.const:xdc_runtime_SysCallback_exitFxn__C 
*          0    00000564    00000004     
                  00000564    00000004     appBLE_pem3.oem3 (.const:xdc_runtime_SysCallback_exitFxn__C)

.const:xdc_runtime_System_abortFxn__C 
*          0    00000568    00000004     
                  00000568    00000004     appBLE_pem3.oem3 (.const:xdc_runtime_System_abortFxn__C)

.const:xdc_runtime_System_exitFxn__C 
*          0    0000056c    00000004     
                  0000056c    00000004     appBLE_pem3.oem3 (.const:xdc_runtime_System_exitFxn__C)

.const:xdc_runtime_System_maxAtexitHandlers__C 
*          0    00000570    00000004     
                  00000570    00000004     appBLE_pem3.oem3 (.const:xdc_runtime_System_maxAtexitHandlers__C)

.const:xdc_runtime_Text_charTab__C 
*          0    00000574    00000004     
                  00000574    00000004     appBLE_pem3.oem3 (.const:xdc_runtime_Text_charTab__C)

.const:xdc_runtime_Text_nameEmpty__C 
*          0    00000578    00000004     
                  00000578    00000004     appBLE_pem3.oem3 (.const:xdc_runtime_Text_nameEmpty__C)

.const:xdc_runtime_Text_nameStatic__C 
*          0    0000057c    00000004     
                  0000057c    00000004     appBLE_pem3.oem3 (.const:xdc_runtime_Text_nameStatic__C)

.const:xdc_runtime_Text_nameUnknown__C 
*          0    00000580    00000004     
                  00000580    00000004     appBLE_pem3.oem3 (.const:xdc_runtime_Text_nameUnknown__C)

.const:xdc_runtime_Main_Module__id__C 
*          0    00000584    00000002     
                  00000584    00000002     appBLE_pem3.oem3 (.const:xdc_runtime_Main_Module__id__C)

.const:xdc_runtime_Memory_Module__id__C 
*          0    00000586    00000002     
                  00000586    00000002     appBLE_pem3.oem3 (.const:xdc_runtime_Memory_Module__id__C)

.const:xdc_runtime_Text_charCnt__C 
*          0    00000588    00000002     
                  00000588    00000002     appBLE_pem3.oem3 (.const:xdc_runtime_Text_charCnt__C)

.const:xdc_runtime_Text_isLoaded__C 
*          0    0000058a    00000002     
                  0000058a    00000002     appBLE_pem3.oem3 (.const:xdc_runtime_Text_isLoaded__C)

.const:xdc_runtime_Error_policy__C 
*          0    0000058c    00000001     
                  0000058c    00000001     appBLE_pem3.oem3 (.const:xdc_runtime_Error_policy__C)

.const:ti_sysbios_rom_ROM_AONRTCChannelEnable 
*          0    00000590    00000004     
                  00000590    00000004     appBLE_pem3.oem3 (.const:ti_sysbios_rom_ROM_AONRTCChannelEnable)

.const:ti_sysbios_rom_ROM_AONRTCCompareValueSet 
*          0    00000594    00000004     
                  00000594    00000004     appBLE_pem3.oem3 (.const:ti_sysbios_rom_ROM_AONRTCCompareValueSet)

.const:ti_sysbios_rom_ROM_AONRTCCurrentCompareValueGet 
*          0    00000598    00000004     
                  00000598    00000004     appBLE_pem3.oem3 (.const:ti_sysbios_rom_ROM_AONRTCCurrentCompareValueGet)

.const:ti_sysbios_rom_ROM_AONRTCEventClear 
*          0    0000059c    00000004     
                  0000059c    00000004     appBLE_pem3.oem3 (.const:ti_sysbios_rom_ROM_AONRTCEventClear)

.const:ti_sysbios_rom_ROM_ti_sysbios_family_arm_cc26xx_Timer_getCount64__E 
*          0    000005a0    00000004     
                  000005a0    00000004     appBLE_pem3.oem3 (.const:ti_sysbios_rom_ROM_ti_sysbios_family_arm_cc26xx_Timer_getCount64__E)

.const:ti_sysbios_rom_ROM_ti_sysbios_family_arm_cc26xx_Timer_getCurrentTick__E 
*          0    000005a4    00000004     
                  000005a4    00000004     appBLE_pem3.oem3 (.const:ti_sysbios_rom_ROM_ti_sysbios_family_arm_cc26xx_Timer_getCurrentTick__E)

.const:ti_sysbios_rom_ROM_ti_sysbios_family_arm_cc26xx_Timer_getMaxTicks__E 
*          0    000005a8    00000004     
                  000005a8    00000004     appBLE_pem3.oem3 (.const:ti_sysbios_rom_ROM_ti_sysbios_family_arm_cc26xx_Timer_getMaxTicks__E)

.const:ti_sysbios_rom_ROM_ti_sysbios_family_arm_cc26xx_Timer_initDevice__I 
*          0    000005ac    00000004     
                  000005ac    00000004     appBLE_pem3.oem3 (.const:ti_sysbios_rom_ROM_ti_sysbios_family_arm_cc26xx_Timer_initDevice__I)

.const:ti_sysbios_rom_ROM_ti_sysbios_family_arm_cc26xx_Timer_setNextTick__E 
*          0    000005b0    00000004     
                  000005b0    00000004     appBLE_pem3.oem3 (.const:ti_sysbios_rom_ROM_ti_sysbios_family_arm_cc26xx_Timer_setNextTick__E)

.const:ti_sysbios_rom_ROM_ti_sysbios_family_arm_cc26xx_Timer_setThreshold__I 
*          0    000005b4    00000004     
                  000005b4    00000004     appBLE_pem3.oem3 (.const:ti_sysbios_rom_ROM_ti_sysbios_family_arm_cc26xx_Timer_setThreshold__I)

.const:ti_sysbios_rom_ROM_ti_sysbios_family_arm_cc26xx_Timer_start__E 
*          0    000005b8    00000004     
                  000005b8    00000004     appBLE_pem3.oem3 (.const:ti_sysbios_rom_ROM_ti_sysbios_family_arm_cc26xx_Timer_start__E)

.const:ti_sysbios_rom_ROM_ti_sysbios_family_arm_cc26xx_TimestampProvider_get32__E 
*          0    000005bc    00000004     
                  000005bc    00000004     appBLE_pem3.oem3 (.const:ti_sysbios_rom_ROM_ti_sysbios_family_arm_cc26xx_TimestampProvider_get32__E)

.const:ti_sysbios_rom_ROM_xdc_runtime_Startup_getState__I 
*          0    000005c0    00000004     
                  000005c0    00000004     appBLE_pem3.oem3 (.const:ti_sysbios_rom_ROM_xdc_runtime_Startup_getState__I)

.const:ti_sysbios_rom_ROM_xdc_runtime_System_SupportProxy_abort__E 
*          0    000005c4    00000004     
                  000005c4    00000004     appBLE_pem3.oem3 (.const:ti_sysbios_rom_ROM_xdc_runtime_System_SupportProxy_abort__E)

.const:ti_sysbios_rom_ROM_xdc_runtime_System_SupportProxy_exit__E 
*          0    000005c8    00000004     
                  000005c8    00000004     appBLE_pem3.oem3 (.const:ti_sysbios_rom_ROM_xdc_runtime_System_SupportProxy_exit__E)

.const:ti_sysbios_gates_GateMutex_Instance_State_sem__O 
*          0    000005cc    00000004     
                  000005cc    00000004     appBLE_pem3.oem3 (.const:ti_sysbios_gates_GateMutex_Instance_State_sem__O)

.const:ti_sysbios_knl_Clock_Module_State_clockQ__O 
*          0    000005d0    00000004     
                  000005d0    00000004     appBLE_pem3.oem3 (.const:ti_sysbios_knl_Clock_Module_State_clockQ__O)

.const:ti_sysbios_knl_Mailbox_Instance_State_dataQue__O 
*          0    000005d4    00000004     
                  000005d4    00000004     appBLE_pem3.oem3 (.const:ti_sysbios_knl_Mailbox_Instance_State_dataQue__O)

.const:ti_sysbios_knl_Mailbox_Instance_State_dataSem__O 
*          0    000005d8    00000004     
                  000005d8    00000004     appBLE_pem3.oem3 (.const:ti_sysbios_knl_Mailbox_Instance_State_dataSem__O)

.const:ti_sysbios_knl_Mailbox_Instance_State_freeQue__O 
*          0    000005dc    00000004     
                  000005dc    00000004     appBLE_pem3.oem3 (.const:ti_sysbios_knl_Mailbox_Instance_State_freeQue__O)

.const:ti_sysbios_knl_Mailbox_Instance_State_freeSem__O 
*          0    000005e0    00000004     
                  000005e0    00000004     appBLE_pem3.oem3 (.const:ti_sysbios_knl_Mailbox_Instance_State_freeSem__O)

.const:ti_sysbios_knl_Semaphore_Instance_State_pendQ__O 
*          0    000005e4    00000004     
                  000005e4    00000004     appBLE_pem3.oem3 (.const:ti_sysbios_knl_Semaphore_Instance_State_pendQ__O)

.const:ti_sysbios_knl_Task_Module_State_inactiveQ__O 
*          0    000005e8    00000004     
                  000005e8    00000004     appBLE_pem3.oem3 (.const:ti_sysbios_knl_Task_Module_State_inactiveQ__O)

.text.4    0    000005ec    00005d70     
                  000005ec    00000376     driverlib.lib : setup.obj (.text:HapiTrimDeviceShutDown$42)
                  00000962    00000002     sysbios.aem3 : mangled__BIOS_lib.obj (.text:ti_sysbios_family_arm_cc26xx_Power_defaultClockFunc__E)
                  00000964    0000034c                  : mangled__BIOS_lib.obj (.text:ti_sysbios_family_arm_cc26xx_Power_auxISR__E)
                  00000cb0    000002f4                  : mangled__BIOS_lib.obj (.text:ti_sysbios_family_arm_cc26xx_Power_sleep__E)
                  00000fa4    00000290     simpleBLEPeripheral.obj (.text:SimpleBLEPeripheral_init$21)
                  00001234    00000228     peripheral.obj (.text:gapRole_processGAPMsg$6)
                  0000145c    00000224     peripheral.obj (.text:GAPRole_SetParameter)
                  00001680    000001f4     rtsv7M3_T_le_eabi.lib : ull_div_t2.obj (.text)
                  00001874    000001c6     driverlib.lib : sys_ctrl.obj (.text:SysCtrlSetRechargeBeforePowerDown)
                  00001a3a    000001b6     rtsv7M3_T_le_eabi.lib : fd_add_t2.obj (.text)
                  00001bf0    00000188     PINCC26XX.obj (.text:PIN_init)
                  00001d78    00000124     peripheral.obj (.text:GAPRole_GetParameter)
                  00001e9c    00000104     sysbios.aem3 : mangled__BIOS_lib.obj (.text:calibrateRcoscHf1$28)
                  00001fa0    00000100     simpleBLEPeripheral.obj (.text:SimpleBLEPeripheral_performPeriodicTemp$21)
                  000020a0    000000fc     rtsv7M3_T_le_eabi.lib : fd_mul_t2.obj (.text)
                  0000219c    000000f8     sysbios.aem3 : mangled__BIOS_lib.obj (.text:ti_sysbios_family_arm_cc26xx_Power_startFirstMeasurement__E)
                  00002294    000000f6     driverlib.lib : setup.obj (.text:GetTrimForAnabypassValue1$42)
                  0000238a    00000002     sysbios.aem3 : mangled__BIOS_lib.obj (.text:ti_sysbios_family_arm_cc26xx_Power_defaultNotifyTrapFunc__E)
                  0000238c    000000f4     peripheral.obj (.text:gapRole_taskFxn$6)
                  00002480    000000f0     sysbios.aem3 : mangled__BIOS_lib.obj (.text:ti_sysbios_family_arm_cc26xx_Power_standbyPolicy__E)
                  00002570    000000ec     ICall.obj (.text:ICall_primWaitMatch$10)
                  0000265c    000000e0     simpleBLEPeripheral.obj (.text:SimpleBLEPeripheral_taskFxn$21)
                  0000273c    000000d8     sysbios.aem3 : mangled__BIOS_lib.obj (.text:ti_sysbios_family_arm_cc26xx_Power_setDependency__E)
                  00002814    000000d0                  : mangled__BIOS_lib.obj (.text:ti_sysbios_family_arm_cc26xx_Power_releaseDependency__E)
                  000028e4    000000b4     PINCC26XX.obj (.text:PINCC26XX_setIoCfg$17)
                  00002998    000000b4     driverlib.lib : setup.obj (.text:trimDevice)
                  00002a4c    000000b0     devinfoservice.obj (.text:devInfo_ReadAttrCB$3)
                  00002afc    000000b0     sysbios.aem3 : mangled__BIOS_lib.obj (.text:ti_sysbios_knl_Clock_workFuncDynamic__E)
                  00002bac    000000a4                  : mangled__BIOS_lib.obj (.text:ti_sysbios_family_arm_cc26xx_Power_initiateCalibration__E)
                  00002c50    000000a0     driverlib.lib : aux_adc.obj (.text:NOROM_AUXADCDisable)
                  00002cf0    000000a0     auto_init.aem3 : auto_init.oem3 (.text)
                  00002d90    000000a0     peripheral.obj (.text:gapRole_init$6)
                  00002e30    0000009c     rtsv7M3_T_le_eabi.lib : memcpy_t2.obj (.text)
                  00002ecc    00000094     driverlib.lib : osc.obj (.text:OSCHF_GetStartupTime)
                  00002f60    00000094     simpleGATTprofile.obj (.text:simpleProfile_WriteAttrCB$7)
                  00002ff4    00000090     PINCC26XX.obj (.text:PIN_open)
                  00003084    0000008c     sysbios.aem3 : mangled__BIOS_lib.obj (.text:ti_sysbios_family_arm_cc26xx_Power_LF_clockFunc__E)
                  00003110    0000008c                  : mangled__BIOS_lib.obj (.text:ti_sysbios_family_arm_cc26xx_Power_Module_startup__E)
                  0000319c    0000008a     driverlib.lib : aux_adc.obj (.text:NOROM_AUXADCEnableSync)
                  00003226    00000002     appBLE_pem3.oem3 (.text:ti_sysbios_rom_cortexm_cc26xx_CC26xx_badRomRevision__E)
                  00003228    00000088     simpleBLEPeripheral.obj (.text:SimpleBLEPeripheral_processStateChangeEvt$21)
                  000032b0    00000088     sysbios.aem3 : mangled__BIOS_lib.obj (.text:ti_sysbios_family_arm_cc26xx_Timer_start__E)
                  00003338    00000086     rtsv7M3_T_le_eabi.lib : fd_cmp_t2.obj (.text:__aeabi_cdcmple)
                  000033be    00000084     driverlib.lib : setup.obj (.text:GetTrimForAmpcompCtrl$42)
                  00003442    00000002     sysbios.aem3 : mangled__BIOS_lib.obj (.text:xdc_runtime_SysCallback_defaultAbort)
                  00003444    00000084     ICall.obj (.text:ICall_heapMalloc)
                  000034c8    00000084     ICall.obj (.text:ICall_primSetTimer$10)
                  0000354c    0000007c     ICall.obj (.text:ICall_createRemoteTasks)
                  000035c8    0000007a     rtsv7M3_T_le_eabi.lib : memset_t2.obj (.text)
                  00003642    00000002     sysbios.aem3 : mangled__BIOS_lib.obj (.text:xdc_runtime_SysCallback_defaultExit)
                  00003644    00000074     ICall.obj (.text:ICall_primSend$10)
                  000036b8    00000074     simpleBLEPeripheral.obj (.text:adcIsr)
                  0000372c    00000072     driverlib.lib : chipinfo.obj (.text:ChipInfo_GetHwRevision)
                  0000379e    00000002     --HOLE-- [fill = 0]
                  000037a0    00000070     peripheral.obj (.text:gapRole_startConnUpdate$6)
                  00003810    0000006c     ICallCC2650.obj (.text:ICallPlatform_pwrUpdActivityCounter)
                  0000387c    0000006c     driverlib.lib : sys_ctrl.obj (.text:SysCtrl_DCDC_VoltageConditionalControl)
                  000038e8    0000006a     rtsv7M3_T_le_eabi.lib : copy_decompress_rle.obj (.text)
                  00003952    00000066     gattservapp_util.obj (.text:gattServApp_SendNotiInd$5)
                  000039b8    00000066     simpleGATTprofile.obj (.text:simpleProfile_ReadAttrCB$7)
                  00003a1e    00000002     --HOLE-- [fill = 0]
                  00003a20    00000064     gattservapp_util.obj (.text:GATTServApp_ProcessCharCfg)
                  00003a84    00000064     driverlib.lib : osc.obj (.text:OSCHF_AttemptToSwitchToXosc)
                  00003ae8    00000062                   : sys_ctrl.obj (.text:SysCtrlAdjustRechargeAfterPowerDown)
                  00003b4a    00000002     --HOLE-- [fill = 0]
                  00003b4c    00000060     appBLE_pem3.oem3 (.text:ti_sysbios_family_arm_cc26xx_Power_XOSC_HF_clockFunc__E)
                  00003bac    00000060     sysbios.aem3 : mangled__BIOS_lib.obj (.text:ti_sysbios_family_arm_cc26xx_Timer_setNextTick__E)
                  00003c0c    0000005c     simpleGATTprofile.obj (.text:SimpleProfile_SetParameter)
                  00003c68    0000005c     appBLE_pem3.oem3 (.text:xdc_runtime_Startup_getState__I)
                  00003cc4    0000005a     driverlib.lib : ddi.obj (.text:NOROM_DDI16BitfieldWrite)
                  00003d1e    00000002     --HOLE-- [fill = 0]
                  00003d20    00000058     ICall.obj (.text:ICall_primEnroll$10)
                  00003d78    00000058     sysbios.aem3 : mangled__BIOS_lib.obj (.text:ti_sysbios_family_arm_cc26xx_Power_notify__I)
                  00003dd0    00000054     ICallCC2650.obj (.text:ICallPlatform_pwrRegisterNotify)
                  00003e24    00000054     ICall.obj (.text:ICall_primThreadServes$10)
                  00003e78    00000052     ICall.obj (.text:ICall_primWait$10)
                  00003eca    00000052     driverlib.lib : osc.obj (.text:NOROM_OSCClockSourceSet)
                  00003f1c    00000050     ICallBleAPI.obj (.text:GAP_DeviceInit)
                  00003f6c    00000050     ICallBleAPI.obj (.text:GAP_UpdateAdvertisingData)
                  00003fbc    00000050     ICall.obj (.text:ICall_primGetEntityId$10)
                  0000400c    00000050     ICall.obj (.text:ICall_primRegisterApp$10)
                  0000405c    0000004c     peripheral.obj (.text:GAPRole_SendUpdateParam)
                  000040a8    0000004c     ICall.obj (.text:ICall_newTask$10)
                  000040f4    0000004c     peripheral.obj (.text:gapRole_processStackMsg$6)
                  00004140    0000004c     rtsv7M3_T_le_eabi.lib : cpy_tbl.obj (.text)
                  0000418c    0000004a     gattservapp_util.obj (.text:GATTServApp_ProcessCCCWriteReq)
                  000041d6    00000002     --HOLE-- [fill = 0]
                  000041d8    00000048     PINCC26XX.obj (.text:PIN_Isr$17)
                  00004220    00000048     util.obj (.text:Util_constructClock)
                  00004268    00000048     ICallBleAPI.obj (.text:gapSendParamAndPtrCmd$8)
                  000042b0    00000048     ICallBleAPI.obj (.text:gattIndNoti$8)
                  000042f8    00000046     driverlib.lib : ddi.obj (.text:NOROM_DDI16BitfieldRead)
                  0000433e    00000002     --HOLE-- [fill = 0]
                  00004340    00000044     ICallBleAPI.obj (.text:GAP_TerminateLinkReq)
                  00004384    00000044     simpleGATTprofile.obj (.text:SimpleProfile_GetParameter)
                  000043c8    00000044     boot.aem3 : boot.oem3 (.text)
                  0000440c    00000044     rtsv7M3_T_le_eabi.lib : exit.obj (.text)
                  00004450    00000044     sysbios.aem3 : mangled__BIOS_lib.obj (.text:ti_sysbios_family_arm_cc26xx_Timer_initDevice__I)
                  00004494    00000042     ICall.obj (.text:ICall_primCreateSemaphore$10)
                  000044d6    00000042     ICall.obj (.text:ICall_primCreateTask$10)
                  00004518    00000040     peripheral.obj (.text:GAPRole_createTask)
                  00004558    00000040     ICallBleAPI.obj (.text:GATT_SendRsp)
                  00004598    00000040     driverlib.lib : osc.obj (.text:NOROM_OSCInterfaceEnable)
                  000045d8    00000040     simpleBLEPeripheral.obj (.text:SimpleBLEPeripheral_createTask)
                  00004618    00000040     appBLE_pem3.oem3 (.text:ti_sysbios_family_arm_cc26xx_Power_XOSC_HF)
                  00004658    00000040     sysbios.aem3 : mangled__BIOS_lib.obj (.text:ti_sysbios_family_arm_cc26xx_Power_isStableXOSC_HF__E)
                  00004698    00000040                  : mangled__BIOS_lib.obj (.text:ti_sysbios_family_arm_cc26xx_Timer_getCurrentTick__E)
                  000046d8    0000003e     ICallBleAPI.obj (.text:hciSendParamsCmd$8)
                  00004716    00000002     --HOLE-- [fill = 0]
                  00004718    0000003c     ICallBleAPI.obj (.text:GAP_GetParamValue)
                  00004754    0000003c     ICallBleAPI.obj (.text:GATTServApp_RegisterService)
                  00004790    0000003c     ICallCC2650.obj (.text:ICallPlatform_pwrConfigACAction)
                  000047cc    0000003c     ICallBleAPI.obj (.text:profileSetParameter$8)
                  00004808    0000003c     ICallBleAPI.obj (.text:sendWaitMatchCS$8)
                  00004844    0000003c     ICallBleAPI.obj (.text:sendWaitMatchValueCS$8)
                  00004880    0000003c     sysbios.aem3 : mangled__BIOS_lib.obj (.text:ti_sysbios_family_arm_cc26xx_Power_releaseConstraint__E)
                  000048bc    00000038     ICallBleAPI.obj (.text:GAPBondMgr_LinkEst)
                  000048f4    00000038     ICall.obj (.text:ICall_primGetMaxMSecs$10)
                  0000492c    00000038     simpleBLEPeripheral.obj (.text:SimpleBLEPeripheral_sendAttRsp$21)
                  00004964    00000038     util.obj (.text:Util_restartClock)
                  0000499c    00000038     ICallBleAPI.obj (.text:linkDB_NumConns)
                  000049d4    00000038     sysbios.aem3 : mangled__BIOS_lib.obj (.text:ti_sysbios_family_arm_cc26xx_Power_setConstraint__E)
                  00004a0c    00000038                  : mangled__BIOS_lib.obj (.text:ti_sysbios_family_arm_cc26xx_Timer_setThreshold__I)
                  00004a44    00000036     ICallCC2650.obj (.text:ICallPlatform_pwrDispenseImpl$11)
                  00004a7a    00000036     ICallCC2650.obj (.text:ICallPlatform_pwrRequireImpl$11)
                  00004ab0    00000036     ICall.obj (.text:ICall_primWaitSemaphore$10)
                  00004ae6    00000036     driverlib.lib : adi.obj (.text:SafeHapiAuxAdiSelect)
                  00004b1c    00000034                   : chipinfo.obj (.text:ChipInfo_GetChipFamily)
                  00004b50    00000034     ICallBleAPI.obj (.text:GAPBondMgr_SetParameter)
                  00004b84    00000034     ICallBleAPI.obj (.text:GAP_SetParamValue)
                  00004bb8    00000034     ICall.obj (.text:ICall_primEntityId2ServiceId$10)
                  00004bec    00000034     ICall.obj (.text:ICall_primFetchMsg$10)
                  00004c20    00000034     ICall.obj (.text:ICall_primRegisterISR$10)
                  00004c54    00000034     ICall.obj (.text:ICall_primRegisterISR_Ext$10)
                  00004c88    00000034     ICall.obj (.text:ICall_searchServiceEntity$10)
                  00004cbc    00000034     driverlib.lib : setup.obj (.text:SetAonRtcSubSecInc$42)
                  00004cf0    00000034     simpleBLEPeripheral.obj (.text:SimpleBLEPeripheral_processGATTMsg$21)
                  00004d24    00000034     ICallBleAPI.obj (.text:osal_snv_read)
                  00004d58    00000034     ICallBleAPI.obj (.text:osal_snv_write)
                  00004d8c    00000034     ICallBleAPI.obj (.text:profileAddService$8)
                  00004dc0    00000034     ICallBleAPI.obj (.text:registerTask$8)
                  00004df4    00000032     driverlib.lib : osc.obj (.text:OSCHF_SwitchToRcOscTurnOffXosc)
                  00004e26    00000032     ICallBleAPI.obj (.text:gapSendParamsCmd$8)
                  00004e58    00000032     ICallBleAPI.obj (.text:gapSendPtrParamsCmd$8)
                  00004e8a    00000032     ICallBleAPI.obj (.text:matchGapSetGetParamCS$8)
                  00004ebc    00000032     ICallBleAPI.obj (.text:matchGattCmdStatus$8)
                  00004eee    00000032     ICallBleAPI.obj (.text:matchUtilNvCS$8)
                  00004f20    00000030     ICallCC2650.obj (.text:ICallPlatform_pwrNotify$11)
                  00004f50    00000030     ICall.obj (.text:ICall_heapInit)
                  00004f80    00000030     ICall.obj (.text:ICall_msecs2Ticks$10)
                  00004fb0    00000030     PINCC26XX.obj (.text:PIN_setOutputValue)
                  00004fe0    00000030     appBLE_pem3.oem3 (.text:ti_sysbios_BIOS_atExitFunc__I)
                  00005010    00000030     sysbios.aem3 : mangled__BIOS_lib.obj (.text:ti_sysbios_family_arm_cc26xx_Power_registerNotify__E)
                  00005040    00000030                  : mangled__BIOS_lib.obj (.text:ti_sysbios_family_arm_cc26xx_Power_switchXOSC_HF__E)
                  00005070    0000002e     driverlib.lib : setup.obj (.text:GetTrimForRadcExtCfg$42)
                  0000509e    0000002e     simpleBLEPeripheral.obj (.text:ICall_fetchServiceMsg$21)
                  000050cc    0000002e     peripheral.obj (.text:ICall_fetchServiceMsg$6)
                  000050fa    0000002e     ICall.obj (.text:ICall_msgDequeue$10)
                  00005128    0000002e     ICallBleAPI.obj (.text:matchProfileAddServiceCS$8)
                  00005156    0000002c     driverlib.lib : aon_batmon.obj (.text:AONBatMonTemperatureGetDegC)
                  00005182    00000002     --HOLE-- [fill = 0]
                  00005184    0000002c     ICallBleAPI.obj (.text:GAPBondMgr_Register)
                  000051b0    0000002c     ICallBleAPI.obj (.text:HCI_EXT_ConnEventNoticeCmd)
                  000051dc    0000002c     ICall.obj (.text:ICall_heapFree)
                  00005208    0000002c     simpleGATTprofile.obj (.text:ICall_malloc$7)
                  00005234    0000002c     ICall.obj (.text:ICall_msgEnqueue$10)
                  00005260    0000002c     ICall.obj (.text:ICall_primAllocMsg$10)
                  0000528c    0000002c     ICall.obj (.text:ICall_primFetchServiceMsg$10)
                  000052b8    0000002c     ICall.obj (.text:ICall_searchTask$10)
                  000052e4    0000002c     ICallBleAPI.obj (.text:ICall_sendServiceMsg$8)
                  00005310    0000002c     driverlib.lib : aon_rtc.obj (.text:NOROM_AONRTCCurrentCompareValueGet)
                  0000533c    0000002c     PINCC26XX.obj (.text:PIN_setConfig)
                  00005368    0000002a     ICallBleAPI.obj (.text:ICall_waitMatch$8)
                  00005392    0000002a     util.obj (.text:Util_enqueueMsg)
                  000053bc    0000002a     ICallBleAPI.obj (.text:matchProfileCS$8)
                  000053e6    00000028     gattservapp_util.obj (.text:GATTServApp_WriteCharCfg)
                  0000540e    00000028     driverlib.lib : setup.obj (.text:GetTrimForAmpcompTh2$42)
                  00005436    00000002     --HOLE-- [fill = 0]
                  00005438    00000028     ICall.obj (.text:ICall_init)
                  00005460    00000028     ICall.obj (.text:ICall_msgPrepend$10)
                  00005488    00000028     simpleBLEPeripheral.obj (.text:ICall_registerApp$21)
                  000054b0    00000028     peripheral.obj (.text:ICall_registerApp$6)
                  000054d8    00000028     simpleBLEPeripheral.obj (.text:SimpleBLEPeripheral_freeAttRsp$21)
                  00005500    00000028     simpleGATTprofile.obj (.text:SimpleProfile_AddService)
                  00005528    00000028     gattservapp_util.obj (.text:gattServApp_FindCharCfgItem$5)
                  00005550    00000028     appBLE_pem3.oem3 (.text:ti_sysbios_family_arm_cc26xx_Power_isDependencyActive)
                  00005578    00000028     sysbios.aem3 : mangled__BIOS_lib.obj (.text:ti_sysbios_family_arm_cc26xx_Timer_getMaxTicks__E)
                  000055a0    00000026     driverlib.lib : osc.obj (.text:NOROM_OSCClockSourceGet)
                  000055c6    00000024     ICallBleAPI.obj (.text:GAPBondMgr_LinkTerm)
                  000055ea    00000002     --HOLE-- [fill = 0]
                  000055ec    00000024     gattservapp_util.obj (.text:GATTServApp_FindAttr)
                  00005610    00000024     ICallBleAPI.obj (.text:ICall_getLocalMsgEntityId$8)
                  00005634    00000024     ICallBleAPI.obj (.text:ICall_threadServes$8)
                  00005658    00000024     simpleBLEPeripheral.obj (.text:SimpleBLEPeripheral_enqueueMsg$21)
                  0000567c    00000024     appBLE_pem3.oem3 (.text:ti_sysbios_BIOS_registerRTSLock__I)
                  000056a0    00000024     appBLE_pem3.oem3 (.text:ti_sysbios_BIOS_removeRTSLock__I)
                  000056c4    00000024     appBLE_pem3.oem3 (.text:ti_sysbios_BIOS_startFunc__I)
                  000056e8    00000024     sysbios.aem3 : mangled__BIOS_lib.obj (.text:ti_sysbios_family_arm_cc26xx_Timer_dynamicStub__E)
                  0000570c    00000022     driverlib.lib : setup.obj (.text:GetTrimForAmpcompTh1$42)
                  0000572e    00000022     ICall.obj (.text:ICall_dispatch$10)
                  00005750    00000022     util.obj (.text:ICall_malloc$23)
                  00005772    00000002     --HOLE-- [fill = 0]
                  00005774    00000020     gattservapp_util.obj (.text:GATTServApp_InitCharCfg)
                  00005794    00000020     ICallBleAPI.obj (.text:GATT_bm_alloc)
                  000057b4    00000020     driverlib.lib : setup.obj (.text:GetTrimForRcOscLfRtuneCtuneTrim$42)
                  000057d4    00000020                   : setup.obj (.text:GetTrimForXoscHfCtl$42)
                  000057f4    00000020     ICallBleAPI.obj (.text:ICall_allocMsg$8)
                  00005814    00000020     ICallBleAPI.obj (.text:ICall_getEntityId$8)
                  00005834    00000020     simpleBLEPeripheral.obj (.text:ICall_malloc$21)
                  00005854    00000020     ICall.obj (.text:ICall_primService$10)
                  00005874    00000020     ICall.obj (.text:ICall_searchService$10)
                  00005894    00000020     util.obj (.text:Util_dequeueMsg)
                  000058b4    00000020     rtsv7M3_T_le_eabi.lib : u_tofd_t2.obj (.text)
                  000058d4    00000020     appBLE_pem3.oem3 (.text:ti_sysbios_BIOS_rtsLock__I)
                  000058f4    00000020     sysbios.aem3 : mangled__BIOS_lib.obj (.text:ti_sysbios_family_arm_cc26xx_TimestampProvider_get32__E)
                  00005914    0000001e     ICall.obj (.text:ICall_primSendServiceMsg$10)
                  00005932    0000001e     main.obj (.text:main)
                  00005950    0000001e     ICallBleAPI.obj (.text:matchHciCS$8)
                  0000596e    0000001e     ICallBleAPI.obj (.text:waitMatchCS$8)
                  0000598c    0000001c     peripheral.obj (.text:GAPRole_StartDevice)
                  000059a8    0000001c     ICallBleAPI.obj (.text:GATT_bm_free)
                  000059c4    0000001c     simpleBLEPeripheral.obj (.text:ICall_wait$21)
                  000059e0    0000001c     peripheral.obj (.text:ICall_wait$6)
                  000059fc    0000001c     PINCC26XX.obj (.text:PINCC26XX_setIoCfgMux$17)
                  00005a18    0000001c     peripheral.obj (.text:gapRole_HandleParamUpdateNoSuccess$6)
                  00005a34    0000001c     ICallBleAPI.obj (.text:getStatusValueFromErrNo$8)
                  00005a50    0000001a     ICall.obj (.text:ICall_enterCSImpl)
                  00005a6a    0000001a     ICall.obj (.text:ICall_primSetTimerMSecs$10)
                  00005a84    0000001a     driverlib.lib : osc.obj (.text:OSCHF_TurnOnXosc)
                  00005a9e    0000001a     simpleBLEPeripheral.obj (.text:SimpleBLEPeripheral_processAppMsg$21)
                  00005ab8    0000001a     ICallBleAPI.obj (.text:matchGattIndNotiCS$8)
                  00005ad2    00000018     driverlib.lib : chipinfo.obj (.text:ChipInfo_GetPackageType)
                  00005aea    00000002     --HOLE-- [fill = 0]
                  00005aec    00000018     peripheral.obj (.text:GAPRole_TerminateConnection)
                  00005b04    00000018     ICallBleAPI.obj (.text:GATT_Notification)
                  00005b1c    00000018     driverlib.lib : setup.obj (.text:GetTrimForAdcShModeEn$42)
                  00005b34    00000018                   : setup.obj (.text:GetTrimForAdcShVbufEn$42)
                  00005b4c    00000018                   : setup.obj (.text:GetTrimForDblrLoopFilterResetVoltage$42)
                  00005b64    00000018                   : setup.obj (.text:GetTrimForRcOscLfIBiasTrim$42)
                  00005b7c    00000018                   : setup.obj (.text:GetTrimForXoscHfIbiastherm$42)
                  00005b94    00000018                   : setup.obj (.text:GetTrimForXoscLfRegulatorAndCmirrwrRatio$42)
                  00005bac    00000018     ICallCC2650.obj (.text:ICallPlatform_pwrDispense)
                  00005bc4    00000018     ICallCC2650.obj (.text:ICallPlatform_pwrRequire)
                  00005bdc    00000018     simpleBLEPeripheral.obj (.text:ICall_free$21)
                  00005bf4    00000018     util.obj (.text:ICall_free$23)
                  00005c0c    00000018     ICall.obj (.text:ICall_freeMsg$10)
                  00005c24    00000018     simpleBLEPeripheral.obj (.text:ICall_freeMsg$21)
                  00005c3c    00000018     peripheral.obj (.text:ICall_freeMsg$6)
                  00005c54    00000018     ICallBleAPI.obj (.text:ICall_freeMsg$8)
                  00005c6c    00000018     ICall.obj (.text:ICall_initPrim$10)
                  00005c84    00000018     ICall.obj (.text:ICall_primMalloc$10)
                  00005c9c    00000018     simpleBLEPeripheral.obj (.text:SimpleBLEPeripheral_mtrClockHandler$21)
                  00005cb4    00000018     simpleBLEPeripheral.obj (.text:SimpleBLEPeripheral_tempClockHandler$21)
                  00005ccc    00000018     util.obj (.text:Util_constructQueue)
                  00005ce4    00000018     simpleBLEPeripheral.obj (.text:buttonHwiFxn$21)
                  00005cfc    00000018     peripheral.obj (.text:gapRole_setEvent$6)
                  00005d14    00000018     rtsv7M3_T_le_eabi.lib : args_main.obj (.text)
                  00005d2c    00000018                           : ll_mul_t2.obj (.text)
                  00005d44    00000018     appBLE_pem3.oem3 (.text:ti_sysbios_BIOS_rtsUnlock__I)
                  00005d5c    00000018     appBLE_pem3.oem3 (.text:ti_sysbios_family_arm_cc26xx_Power_RFCORECLKS)
                  00005d74    00000018     sysbios.aem3 : mangled__BIOS_lib.obj (.text:ti_sysbios_family_arm_cc26xx_Timer_getCount64__E)
                  00005d8c    00000018     appBLE_pem3.oem3 (.text:ti_sysbios_rom_cortexm_cc26xx_CC26xx_checkRevision__E)
                  00005da4    00000016     driverlib.lib : setup.obj (.text:GetTrimForXoscHfFastStart$42)
                  00005dba    00000016     ICall.obj (.text:ICall_abort$10)
                  00005dd0    00000016     ICall.obj (.text:ICall_leaveCSImpl)
                  00005de6    00000016     ICall.obj (.text:ICall_primStopTimer$10)
                  00005dfc    00000016     simpleBLEPeripheral.obj (.text:SimpleBLEPeripheral_processCharValueChangeEvt$21)
                  00005e12    00000016     appBLE_pem3.oem3 (.text:ti_sysbios_BIOS_exitFunc__I)
                  00005e28    00000014     devinfoservice.obj (.text:DevInfo_AddService)
                  00005e3c    00000014     ICallCC2650.obj (.text:ICallPlatform_pwrIsStableXOSCHF)
                  00005e50    00000014     simpleGATTprofile.obj (.text:SimpleProfile_RegisterAppCBs)
                  00005e64    00000014     driverlib.lib : chipinfo.obj (.text:ThisCodeIsBuiltForCC26xxHwRev22AndLater_HaltIfViolated)
                  00005e78    00000014     rtsv7M3_T_le_eabi.lib : _lock.obj (.text)
                  00005e8c    00000014                           : strlen.obj (.text)
                  00005ea0    00000014     ICallBleAPI.obj (.text:setICallCmdEvtHdr$8)
                  00005eb4    00000014     appBLE_pem3.oem3 (.text:ti_sysbios_knl_Clock_doTick__I)
                  00005ec8    00000012     driverlib.lib : aux_adc.obj (.text:NOROM_AUXADCReadFifo)
                  00005eda    00000012     appBLE_pem3.oem3 (.text:xdc_runtime_Startup_exec__I)
                  00005eec    00000010     devinfoservice.obj (.text:DevInfo_SetParameter)
                  00005efc    00000010     ICallBleAPI.obj (.text:GAP_EndDiscoverable)
                  00005f0c    00000010     gattservapp_util.obj (.text:GATTServApp_ReadCharCfg)
                  00005f1c    00000010     ICallCC2650.obj (.text:ICallPlatform_pwrGetXOSCStartupTime)
                  00005f2c    00000010     ICall.obj (.text:ICall_primGetTickPeriod$10)
                  00005f3c    00000010     ICall.obj (.text:ICall_taskEntry$10)
                  00005f4c    00000010     util.obj (.text:Util_isActive)
                  00005f5c    0000000e     ICallCC2650.obj (.text:ICallPlatform_pwrGetTransitionState)
                  00005f6a    0000000e     ICall.obj (.text:ICall_primDisableMInt$10)
                  00005f78    0000000e     ICall.obj (.text:ICall_primEnableMInt$10)
                  00005f86    0000000e     ICall.obj (.text:ICall_primFreeMsg$10)
                  00005f94    0000000e     ICall.obj (.text:ICall_primGetTicks$10)
                  00005fa2    0000000e     driverlib.lib : vims.obj (.text:NOROM_VIMSModeGet)
                  00005fb0    0000000e                   : setup.obj (.text:SignExtendVddrTrimValue$42)
                  00005fbe    0000000e     simpleBLEPeripheral.obj (.text:SimpleBLEPeripheral_processStackMsg$21)
                  00005fcc    0000000e     rtsv7M3_T_le_eabi.lib : copy_decompress_none.obj (.text:decompress:none)
                  00005fda    0000000e     ICallBleAPI.obj (.text:matchGSARegisterServiceCS$8)
                  00005fe8    0000000e     ICallBleAPI.obj (.text:matchGapLinkEstCS$8)
                  00005ff6    0000000e     ICallBleAPI.obj (.text:matchGattSendRspCS$8)
                  00006004    0000000e     ICallBleAPI.obj (.text:matchLinkDBNumConnsCS$8)
                  00006012    0000000e     ICallBleAPI.obj (.text:setDispatchCmdEvtHdr$8)
                  00006020    0000000c     ICallBleAPI.obj (.text:GAP_MakeDiscoverable)
                  0000602c    0000000c     ICallBleAPI.obj (.text:GAP_TerminateAuth)
                  00006038    0000000c     ICallBleAPI.obj (.text:GAP_UpdateLinkParamReq)
                  00006044    0000000c     ICallBleAPI.obj (.text:GGS_SetParameter)
                  00006050    0000000c     ICall.obj (.text:ICall_clockFunc$10)
                  0000605c    0000000c     ICall.obj (.text:ICall_primDisableInt$10)
                  00006068    0000000c     ICall.obj (.text:ICall_primEnableInt$10)
                  00006074    0000000c     ICall.obj (.text:ICall_primFree$10)
                  00006080    0000000c     ICall.obj (.text:ICall_primSignal$10)
                  0000608c    0000000c     driverlib.lib : cpu.obj (.text:NOROM_CPUcpsid)
                  00006098    0000000c                   : cpu.obj (.text:NOROM_CPUcpsie)
                  000060a4    0000000c     rtsv7M3_T_le_eabi.lib : copy_zero_init.obj (.text:decompress:ZI)
                  000060b0    0000000c     ICallBleAPI.obj (.text:matchProfileSetParamCS$8)
                  000060bc    0000000c     sysbios.aem3 : mangled__BIOS_lib.obj (.text:ti_sysbios_BIOS_getThreadType__E)
                  000060c8    0000000c                  : mangled__BIOS_lib.obj (.text:ti_sysbios_family_arm_cc26xx_Power_getTransitionState__E)
                  000060d4    0000000c                  : mangled__BIOS_lib.obj (.text:ti_sysbios_hal_Hwi_Params__init__S)
                  000060e0    0000000c     appBLE_pem3.oem3 (.text:xdc_runtime_Startup_reset__I)
                  000060ec    0000000a     ICallCC2650.obj (.text:ICallPlatform_pwrSwitchXOSCHF)
                  000060f6    0000000a     ICall.obj (.text:ICall_primE2S$10)
                  00006100    00000008     ICallBleAPI.obj (.text:GATT_Indication)
                  00006108    00000008     simpleBLEPeripheral.obj (.text:SimpleBLEPeripheral_charValueChangeCB$21)
                  00006110    00000008     simpleBLEPeripheral.obj (.text:SimpleBLEPeripheral_stateChangeCB$21)
                  00006118    00000008     ICallBleAPI.obj (.text:matchHciExtConnEventNoticeCS$8)
                  00006120    00000006     ICallBleAPI.obj (.text:GAP_RegisterForMsgs)
                  00006126    00000006     ICallBleAPI.obj (.text:GATT_RegisterForMsgs)
                  0000612c    00000006     ICallBleAPI.obj (.text:GGS_AddService)
                  00006132    00000006     ICall.obj (.text:ICall_mallocImpl)
                  00006138    00000006     PINCC26XX.obj (.text:PIN_registerIntCb)
                  0000613e    00000006     sysbios.aem3 : mangled__BIOS_lib.obj (.text:__xdc__init)
                  00006144    00000006     rtsv7M3_T_le_eabi.lib : copy_decompress_rle.obj (.text:decompress:rle24)
                  0000614a    00000006     ICallBleAPI.obj (.text:gattAddService$8)
                  00006150    00000006     ICallBleAPI.obj (.text:matchBondMgrSetParamCS$8)
                  00006156    00000006     ICallBleAPI.obj (.text:matchGGSSetParamCS$8)
                  0000615c    00000006     ICallBleAPI.obj (.text:matchGapDeviceInitCS$8)
                  00006162    00000006     ICallBleAPI.obj (.text:matchGapEndDiscoverableCS$8)
                  00006168    00000006     ICallBleAPI.obj (.text:matchGapGetParamCS$8)
                  0000616e    00000006     ICallBleAPI.obj (.text:matchGapMakeDiscoverableCS$8)
                  00006174    00000006     ICallBleAPI.obj (.text:matchGapSetParamCS$8)
                  0000617a    00000006     ICallBleAPI.obj (.text:matchGapTerminateAuthCS$8)
                  00006180    00000006     ICallBleAPI.obj (.text:matchGapTerminateLinkReqCS$8)
                  00006186    00000006     ICallBleAPI.obj (.text:matchGapUpdateAdvDataCS$8)
                  0000618c    00000006     ICallBleAPI.obj (.text:matchGapUpdateLinkParamReqCS$8)
                  00006192    00000006     ICallBleAPI.obj (.text:matchUtilNvReadCS$8)
                  00006198    00000006     ICallBleAPI.obj (.text:matchUtilNvWriteCS$8)
                  0000619e    00000004     util.obj (.text:Util_startClock)
                  000061a2    00000004     util.obj (.text:Util_stopClock)
                  000061a6    00000004     peripheral.obj (.text:gapRole_SetupGAP$6)
                  000061aa    00000004     appBLE_pem3.oem3 (.text:ti_sysbios_family_arm_cc26xx_Power_NOP)
                  000061ae    00000004     sysbios.aem3 : mangled__BIOS_lib.obj (.text:ti_sysbios_knl_Clock_isActive__E)
                  000061b2    00000002     --HOLE-- [fill = 0]
                  000061b4    00000008     (.tramp.xdc_runtime_Core_assignParams__I.1)
                  000061bc    00000008     (.tramp.ti_sysbios_hal_Hwi_enableInterrupt__E.1)
                  000061c4    00000008     (.tramp.ti_sysbios_hal_Hwi_disableInterrupt__E.1)
                  000061cc    00000008     (.tramp.ti_sysbios_knl_Task_enable__E.1)
                  000061d4    00000008     (.tramp.ti_sysbios_family_arm_m3_Hwi_enableFxn__E.1)
                  000061dc    00000008     (.tramp.xdc_runtime_Startup_startMods__I.1)
                  000061e4    00000008     (.tramp.ti_sysbios_knl_Swi_post__E.1)
                  000061ec    00000008     (.tramp.ti_sysbios_knl_Clock_logTick__E.1)
                  000061f4    00000008     (.tramp.ti_sysbios_BIOS_RtsGateProxy_leave__E.1)
                  000061fc    00000008     (.tramp.ti_sysbios_knl_Queue_construct.1)
                  00006204    00000008     (.tramp.ti_sysbios_BIOS_start__E.1)
                  0000620c    00000008     (.tramp.ti_sysbios_BIOS_RtsGateProxy_enter__E.1)
                  00006214    00000008     (.tramp.ti_sysbios_knl_Queue_dequeue__E.1)
                  0000621c    00000008     (.tramp.ti_sysbios_knl_Task_startup__E.1)
                  00006224    00000008     (.tramp.ti_sysbios_knl_Swi_startup__E.1)
                  0000622c    00000008     (.tramp.ti_sysbios_hal_Hwi_startup__E.1)
                  00006234    00000008     (.tramp.ti_sysbios_family_arm_cc26xx_Timer_startup__E.1)
                  0000623c    00000008     (.tramp.xdc_runtime_System_atexit__E.1)
                  00006244    00000008     (.tramp.ti_sysbios_knl_Queue_enqueue__E.1)
                  0000624c    00000008     (.tramp.ti_sysbios_knl_Queue_put__E.1)
                  00006254    00000008     (.tramp.ti_sysbios_BIOS_setThreadType__E.1)
                  0000625c    00000008     (.tramp.ti_sysbios_hal_Hwi_create.1)
                  00006264    00000008     (.tramp.ti_sysbios_knl_Task_construct.1)
                  0000626c    00000008     (.tramp.xdc_runtime_System_exit__E.1)
                  00006274    00000008     (.tramp.ti_sysbios_knl_Clock_construct.1)
                  0000627c    00000008     (.tramp.ti_sysbios_knl_Semaphore_create.1)
                  00006284    00000008     (.tramp.ti_sysbios_knl_Task_create.1)
                  0000628c    00000008     (.tramp.ti_sysbios_knl_Task_Params__init__S.1)
                  00006294    00000008     (.tramp.ti_sysbios_knl_Clock_create.1)
                  0000629c    00000008     (.tramp.ti_sysbios_knl_Clock_Params__init__S.1)
                  000062a4    00000008     (.tramp.ti_sysbios_knl_Clock_scheduleNextTick__E.1)
                  000062ac    00000008     (.tramp.ti_sysbios_knl_Clock_walkQueueDynamic__E.1)
                  000062b4    00000008     (.tramp.ti_sysbios_family_arm_m3_Hwi_restoreFxn__E.1)
                  000062bc    00000008     (.tramp.ti_sysbios_family_arm_m3_Hwi_disableFxn__E.1)
                  000062c4    00000008     (.tramp.ti_sysbios_knl_Semaphore_post__E.1)
                  000062cc    00000008     (.tramp.ti_sysbios_knl_Clock_getTicks__E.1)
                  000062d4    00000008     (.tramp.ti_sysbios_knl_Task_self__E.1)
                  000062dc    00000008     (.tramp.ti_sysbios_knl_Clock_stop__E.1)
                  000062e4    00000008     (.tramp.ti_sysbios_knl_Clock_start__E.1)
                  000062ec    00000008     (.tramp.ti_sysbios_knl_Clock_setTimeout__E.1)
                  000062f4    00000008     (.tramp.ti_sysbios_knl_Clock_TimerProxy_getCurrentTick__E.1)
                  000062fc    00000008     (.tramp.ti_sysbios_knl_Task_sleep__E.1)
                  00006304    00000008     (.tramp.ti_sysbios_family_arm_m3_Hwi_construct.1)
                  0000630c    00000008     (.tramp.ti_sysbios_family_arm_m3_Hwi_Params__init__S.1)
                  00006314    00000008     (.tramp.ti_sysbios_knl_Semaphore_construct.1)
                  0000631c    00000008     (.tramp.ti_sysbios_knl_Semaphore_Params__init__S.1)
                  00006324    00000008     (.tramp.ti_sysbios_knl_Task_restore__E.1)
                  0000632c    00000008     (.tramp.ti_sysbios_knl_Swi_restore__E.1)
                  00006334    00000008     (.tramp.ti_sysbios_knl_Swi_disable__E.1)
                  0000633c    00000008     (.tramp.ti_sysbios_knl_Queue_next__E.1)
                  00006344    00000008     (.tramp.ti_sysbios_knl_Queue_head__E.1)
                  0000634c    00000008     (.tramp.ti_sysbios_knl_Queue_empty__E.1)
                  00006354    00000008     (.tramp.ti_sysbios_knl_Task_disable__E.1)

.const     0    0000635c    00000264     
                  0000635c    000000bc     ICall.obj (.const)
                  00006418    0000004c     appBLE_pem3.oem3 (.const:ti_sysbios_family_arm_cc26xx_Power_db)
                  00006464    00000048     appBLE_pem3.oem3 (.const:.string)
                  000064ac    0000002c     gatt_uuid.obj (.const)
                  000064d8    00000028     appBLE_pem3.oem3 (.const:xdc_runtime_Startup_sfxnTab__A)
                  00006500    00000027     bleUserConfig.obj (.const:txPowerTable)
                  00006527    00000014     devinfoservice.obj (.const:.string)
                  0000653b    00000001     ICallCC2650.obj (.const)
                  0000653c    00000014     devinfoservice.obj (.const)
                  00006550    00000014     simpleGATTprofile.obj (.const)
                  00006564    00000014     appBLE_pem3.oem3 (.const:xdc_runtime_Startup_sfxnRts__A)
                  00006578    0000000c     simpleGATTprofile.obj (.const:.string)
                  00006584    0000000c     appBLE_pem3.oem3 (.const:xdc_runtime_Startup_firstFxns__A)
                  00006590    00000006     bleUserConfig.obj (.const)
                  00006596    00000005     simpleBLEPeripheral.obj (.const:.string)
                  0000659b    00000001     appBLE_pem3.oem3 (.const:xdc_runtime_Text_charTab__A)
                  0000659c    00000004     appBLE_pem3.oem3 (.const:ti_sysbios_family_arm_cc26xx_Power_Module_State_clockObj__O)
                  000065a0    00000004     appBLE_pem3.oem3 (.const:ti_sysbios_family_arm_cc26xx_Power_Module_State_lfClockObj__O)
                  000065a4    00000004     appBLE_pem3.oem3 (.const:ti_sysbios_family_arm_cc26xx_Power_Module_State_notifyQ__O)
                  000065a8    00000004     appBLE_pem3.oem3 (.const:ti_sysbios_family_arm_cc26xx_Power_notifyTrapFunc__C)
                  000065ac    00000004     appBLE_pem3.oem3 (.const:ti_sysbios_family_arm_cc26xx_Power_totalTicksSTANDBY__C)
                  000065b0    00000004     appBLE_pem3.oem3 (.const:ti_sysbios_family_arm_cc26xx_Power_wakeDelaySTANDBY__C)
                  000065b4    00000004     appBLE_pem3.oem3 (.const:ti_sysbios_family_arm_m3_Hwi_disablePriority__C)
                  000065b8    00000004     appBLE_pem3.oem3 (.const:ti_sysbios_knl_Clock_tickPeriod__C)
                  000065bc    00000004     appBLE_pem3.oem3 (.const:ti_sysbios_knl_Idle_funcList__A)

.cinit     0    000065c0    000007e0     
                  000065c0    00000647     (.cinit..data.load) [load image, compression = rle]
                  00006c07    00000001     --HOLE-- [fill = 0]
                  00006c08    0000002d     (.cinit..data:ti_sysbios_family_arm_m3_Hwi_Module__state__V.load) [load image, compression = rle]
                  00006c35    00000003     --HOLE-- [fill = 0]
                  00006c38    0000002c     (.cinit..data:ti_sysbios_knl_Task_Module__state__V.load) [load image, compression = rle]
                  00006c64    00000004     --HOLE-- [fill = 0]
                  00006c68    00000021     (.cinit..data:ti_sysbios_knl_Clock_Module__state__V.load) [load image, compression = rle]
                  00006c89    00000007     --HOLE-- [fill = 0]
                  00006c90    0000001f     (.cinit..data:ti_sysbios_BIOS_Module__state__V.load) [load image, compression = rle]
                  00006caf    00000001     --HOLE-- [fill = 0]
                  00006cb0    00000011     (.cinit..data:ti_sysbios_knl_Swi_Module__state__V.load) [load image, compression = rle]
                  00006cc1    00000007     --HOLE-- [fill = 0]
                  00006cc8    0000000d     (.cinit..data:ti_sysbios_family_arm_cc26xx_Timer_Module__state__V.load) [load image, compression = rle]
                  00006cd5    00000003     --HOLE-- [fill = 0]
                  00006cd8    0000000c     (__TI_handler_table)
                  00006ce4    00000004     --HOLE-- [fill = 0]
                  00006ce8    0000000a     (.cinit..data:xdc_runtime_Memory_Module__state__V.load) [load image, compression = rle]
                  00006cf2    00000006     --HOLE-- [fill = 0]
                  00006cf8    00000009     (.cinit..data:ti_sysbios_family_arm_cc26xx_TimestampProvider_Module__state__V.load) [load image, compression = rle]
                  00006d01    00000007     --HOLE-- [fill = 0]
                  00006d08    00000009     (.cinit..data:xdc_runtime_Startup_Module__state__V.load) [load image, compression = rle]
                  00006d11    00000007     --HOLE-- [fill = 0]
                  00006d18    00000009     (.cinit..data:xdc_runtime_System_Module__state__V.load) [load image, compression = rle]
                  00006d21    00000007     --HOLE-- [fill = 0]
                  00006d28    00000008     (.cinit..bss.load) [load image, compression = zero_init]
                  00006d30    00000008     (.cinit..vecs.load) [load image, compression = zero_init]
                  00006d38    00000068     (__TI_cinit_table)

.init_array 
*          0    00000000    00000000     UNINITIALIZED

.ccfg      0    0001ffa8    00000058     
                  0001ffa8    00000058     ccfg_appBLE.obj (.ccfg:retain)

.vecs      0    20000000    000000c8     UNINITIALIZED
                  20000000    000000c8     appBLE_pem3.oem3 (.vecs)

.data:ti_sysbios_knl_Task_Module__state__V 
*          0    20000100    00000044     UNINITIALIZED
                  20000100    00000044     appBLE_pem3.oem3 (.data:ti_sysbios_knl_Task_Module__state__V)

.data:ti_sysbios_family_arm_m3_Hwi_Module__state__V 
*          0    20000144    00000034     UNINITIALIZED
                  20000144    00000034     appBLE_pem3.oem3 (.data:ti_sysbios_family_arm_m3_Hwi_Module__state__V)

.data:ti_sysbios_knl_Clock_Module__state__V 
*          0    20000178    0000002c     UNINITIALIZED
                  20000178    0000002c     appBLE_pem3.oem3 (.data:ti_sysbios_knl_Clock_Module__state__V)

.data:ti_sysbios_BIOS_Module__state__V 
*          0    200001a4    00000024     UNINITIALIZED
                  200001a4    00000024     appBLE_pem3.oem3 (.data:ti_sysbios_BIOS_Module__state__V)

.data:ti_sysbios_knl_Swi_Module__state__V 
*          0    200001c8    0000001c     UNINITIALIZED
                  200001c8    0000001c     appBLE_pem3.oem3 (.data:ti_sysbios_knl_Swi_Module__state__V)

.data:ti_sysbios_family_arm_cc26xx_Timer_Module__state__V 
*          0    200001e4    00000008     UNINITIALIZED
                  200001e4    00000008     appBLE_pem3.oem3 (.data:ti_sysbios_family_arm_cc26xx_Timer_Module__state__V)

.data:ti_sysbios_family_arm_cc26xx_TimestampProvider_Module__state__V 
*          0    200001ec    00000004     UNINITIALIZED
                  200001ec    00000004     appBLE_pem3.oem3 (.data:ti_sysbios_family_arm_cc26xx_TimestampProvider_Module__state__V)

.data:xdc_runtime_Startup_Module__state__V 
*          0    200001f0    00000008     UNINITIALIZED
                  200001f0    00000008     appBLE_pem3.oem3 (.data:xdc_runtime_Startup_Module__state__V)

.data:xdc_runtime_System_Module__state__V 
*          0    200001f8    00000008     UNINITIALIZED
                  200001f8    00000008     appBLE_pem3.oem3 (.data:xdc_runtime_System_Module__state__V)

.data:xdc_runtime_Memory_Module__state__V 
*          0    20000200    00000004     UNINITIALIZED
                  20000200    00000004     appBLE_pem3.oem3 (.data:xdc_runtime_Memory_Module__state__V)

.bss       0    20000208    000014b1     UNINITIALIZED
                  20000208    00000a70     ICall.obj (.bss:heapmgrHeapStore$10)
                  20000c78    00000680     appBLE_pem3.oem3 (.bss:ti_sysbios_heaps_HeapMem_Instance_State_0_buf__A)
                  200012f8    00000200     appBLE_pem3.oem3 (.bss:taskStackSection)
                  200014f8    000000dc     PINCC26XX.obj (.bss)
                  200015d4    000000c8     appBLE_pem3.oem3 (.bss:ti_sysbios_family_arm_m3_Hwi_dispatchTable)
                  2000169c    00000014     (.common:oscHfGlobals$41)
                  200016b0    00000008     (.common:powerQualGlobals$43)
                  200016b8    00000001     (.common:driverlib_release_0_43243)

.data      0    200016c0    00000f50     UNINITIALIZED
                  200016c0    00000480     simpleBLEPeripheral.obj (.data)
                  20001b40    0000036c     peripheral.obj (.data)
                  20001eac    000001e0     devinfoservice.obj (.data)
                  2000208c    00000180     simpleGATTprofile.obj (.data)
                  2000220c    000000bc     appBLE_pem3.oem3 (.data)
                  200022c8    0000008c     ICall.obj (.data)
                  20002354    00000070     appBLE_pem3.oem3 (.data:ti_sysbios_family_arm_cc26xx_Power_Module__state__V)
                  200023c4    0000004c     appBLE_pem3.oem3 (.data:ti_sysbios_knl_Task_Object__table__V)
                  20002410    00000048     appBLE_pem3.oem3 (.data:ti_sysbios_family_arm_cc26xx_Timer_Object__table__V)
                  20002458    00000038     appBLE_pem3.oem3 (.data:ti_sysbios_gates_GateMutex_Object__table__V)
                  20002490    00000034     bleUserConfig.obj (.data:rfRegTbl)
                  200024c4    00000030     appBLE_pem3.oem3 (.data:ti_sysbios_family_arm_m3_Hwi_Object__table__V)
                  200024f4    00000030     appBLE_pem3.oem3 (.data:ti_sysbios_knl_Swi_Module_State_0_readyQ__A)
                  20002524    00000030     appBLE_pem3.oem3 (.data:ti_sysbios_knl_Swi_Object__table__V)
                  20002554    00000030     appBLE_pem3.oem3 (.data:ti_sysbios_knl_Task_Module_State_0_readyQ__A)
                  20002584    0000002c     Board.obj (.data:BoardGpioInitTable)
                  200025b0    0000001c     main.obj (.data)
                  200025cc    0000001c     sysbios.aem3 : mangled__BIOS_lib.obj (.data)
                  200025e8    0000000c     ICallBleAPI.obj (.data)
                  200025f4    00000008     ICallCC2650.obj (.data)
                  200025fc    00000008     rtsv7M3_T_le_eabi.lib : _lock.obj (.data)
                  20002604    00000008                           : exit.obj (.data)
                  2000260c    00000004                           : stkdepth_vars.obj (.data)

.stack     0    20003fe4    00000400     UNINITIALIZED
                  20003fe4    00000400     --HOLE--

.bootVecs 
*          0    00000000    00000008     DSECT
                  00000000    00000008     boot.aem3 : boot.oem3 (.bootVecs)

xdc.meta   0    00000000    000000ee     COPY SECTION
                  00000000    000000ee     appBLE_pem3.oem3 (xdc.meta)

xdc.noload 
*          0    00000000    00000000     COPY SECTION

.TI.noinit 
*          0    20000208    00000000     UNINITIALIZED

.TI.persistent 
*          0    200016c0    00000000     UNINITIALIZED


LINKER GENERATED COPY TABLES

__TI_cinit_table @ 00006d38 records: 13, size/record: 8, table size: 104
	.data: load addr=000065c0, load size=00000647 bytes, run addr=200016c0, run size=00000f50 bytes, compression=rle
	.data:ti_sysbios_family_arm_m3_Hwi_Module__state__V: load addr=00006c08, load size=0000002d bytes, run addr=20000144, run size=00000034 bytes, compression=rle
	.data:ti_sysbios_knl_Task_Module__state__V: load addr=00006c38, load size=0000002c bytes, run addr=20000100, run size=00000044 bytes, compression=rle
	.data:ti_sysbios_knl_Clock_Module__state__V: load addr=00006c68, load size=00000021 bytes, run addr=20000178, run size=0000002c bytes, compression=rle
	.data:ti_sysbios_BIOS_Module__state__V: load addr=00006c90, load size=0000001f bytes, run addr=200001a4, run size=00000024 bytes, compression=rle
	.data:ti_sysbios_knl_Swi_Module__state__V: load addr=00006cb0, load size=00000011 bytes, run addr=200001c8, run size=0000001c bytes, compression=rle
	.data:ti_sysbios_family_arm_cc26xx_Timer_Module__state__V: load addr=00006cc8, load size=0000000d bytes, run addr=200001e4, run size=00000008 bytes, compression=rle
	.data:xdc_runtime_Memory_Module__state__V: load addr=00006ce8, load size=0000000a bytes, run addr=20000200, run size=00000004 bytes, compression=rle
	.data:ti_sysbios_family_arm_cc26xx_TimestampProvider_Module__state__V: load addr=00006cf8, load size=00000009 bytes, run addr=200001ec, run size=00000004 bytes, compression=rle
	.data:xdc_runtime_Startup_Module__state__V: load addr=00006d08, load size=00000009 bytes, run addr=200001f0, run size=00000008 bytes, compression=rle
	.data:xdc_runtime_System_Module__state__V: load addr=00006d18, load size=00000009 bytes, run addr=200001f8, run size=00000008 bytes, compression=rle
	.bss: load addr=00006d28, load size=00000008 bytes, run addr=20000208, run size=000014b1 bytes, compression=zero_init
	.vecs: load addr=00006d30, load size=00000008 bytes, run addr=20000000, run size=000000c8 bytes, compression=zero_init


LINKER GENERATED HANDLER TABLE

__TI_handler_table @ 00006cd8 records: 3, size/record: 4, table size: 12
	index: 0, handler: __TI_decompress_rle24
	index: 1, handler: __TI_decompress_none
	index: 2, handler: __TI_zero_init


FAR CALL TRAMPOLINES

callee name               trampoline name
   callee addr  tramp addr   call addr  call info
--------------  -----------  ---------  ----------------
ti_sysbios_knl_Semaphore_pend__E  $Tramp$TT$L$PI$$ti_sysbios_knl_Semaphore_pend__E
   1001a0cd     000000f4     00000076   simpleBLEPeripheral.obj (.text:SimpleBLEPeripheral_performPeriodicMtr$21)
                             00001ff8   simpleBLEPeripheral.obj (.text:SimpleBLEPeripheral_performPeriodicTemp$21)
                             000025d8   ICall.obj (.text:ICall_primWaitMatch$10)
                             00003008   PINCC26XX.obj (.text:PIN_open)
                             00003ebc   ICall.obj (.text:ICall_primWait$10)
                             00004ad8   ICall.obj (.text:ICall_primWaitSemaphore$10)
xdc_runtime_Core_assignParams__I  $Tramp$TT$L$PI$$xdc_runtime_Core_assignParams__I
   1001c5f1     000061b4     000060d8   sysbios.aem3 : mangled__BIOS_lib.obj (.text:ti_sysbios_hal_Hwi_Params__init__S)
ti_sysbios_hal_Hwi_enableInterrupt__E  $Tramp$TT$L$PI$$ti_sysbios_hal_Hwi_enableInterrupt__E
   1001c285     000061bc     0000606c   ICall.obj (.text:ICall_primEnableInt$10)
ti_sysbios_hal_Hwi_disableInterrupt__E  $Tramp$TT$L$PI$$ti_sysbios_hal_Hwi_disableInterrupt__E
   1001c281     000061c4     00006060   ICall.obj (.text:ICall_primDisableInt$10)
ti_sysbios_knl_Task_enable__E  $Tramp$TT$L$PI$$ti_sysbios_knl_Task_enable__E
   1001c243     000061cc     00005f7e   ICall.obj (.text:ICall_primEnableMInt$10)
ti_sysbios_family_arm_m3_Hwi_enableFxn__E  $Tramp$TT$L$PI$$ti_sysbios_family_arm_m3_Hwi_enableFxn__E
   1001c155     000061d4     00005f7a   ICall.obj (.text:ICall_primEnableMInt$10)
xdc_runtime_Startup_startMods__I  $Tramp$TT$L$PI$$xdc_runtime_Startup_startMods__I
   1001c30d     000061dc     00005ee4   appBLE_pem3.oem3 (.text:xdc_runtime_Startup_exec__I)
ti_sysbios_knl_Swi_post__E  $Tramp$TT$L$PI$$ti_sysbios_knl_Swi_post__E
   1001b321     000061e4     00005ebe   appBLE_pem3.oem3 (.text:ti_sysbios_knl_Clock_doTick__I)
ti_sysbios_knl_Clock_logTick__E  $Tramp$TT$L$PI$$ti_sysbios_knl_Clock_logTick__E
   1001be67     000061ec     00005eb6   appBLE_pem3.oem3 (.text:ti_sysbios_knl_Clock_doTick__I)
ti_sysbios_BIOS_RtsGateProxy_leave__E  $Tramp$TT$L$PI$$ti_sysbios_BIOS_RtsGateProxy_leave__E
   1001c24d     000061f4     00005d52   appBLE_pem3.oem3 (.text:ti_sysbios_BIOS_rtsUnlock__I)
ti_sysbios_knl_Queue_construct  $Tramp$TT$L$PI$$ti_sysbios_knl_Queue_construct
   1001b8f5     000061fc     00005cd6   util.obj (.text:Util_constructQueue)
ti_sysbios_BIOS_start__E  $Tramp$TT$L$PI$$ti_sysbios_BIOS_start__E
   1001c055     00006204     00005948   main.obj (.text:main)
ti_sysbios_BIOS_RtsGateProxy_enter__E  $Tramp$TT$L$PI$$ti_sysbios_BIOS_RtsGateProxy_enter__E
   1001c249     0000620c     000058da   appBLE_pem3.oem3 (.text:ti_sysbios_BIOS_rtsLock__I)
ti_sysbios_knl_Queue_dequeue__E  $Tramp$TT$L$PI$$ti_sysbios_knl_Queue_dequeue__E
   1001c1a9     00006214     000058a6   util.obj (.text:Util_dequeueMsg)
ti_sysbios_knl_Task_startup__E  $Tramp$TT$L$PI$$ti_sysbios_knl_Task_startup__E
   1001c309     0000621c     000056dc   appBLE_pem3.oem3 (.text:ti_sysbios_BIOS_startFunc__I)
ti_sysbios_knl_Swi_startup__E  $Tramp$TT$L$PI$$ti_sysbios_knl_Swi_startup__E
   1001c23d     00006224     000056d8   appBLE_pem3.oem3 (.text:ti_sysbios_BIOS_startFunc__I)
ti_sysbios_hal_Hwi_startup__E  $Tramp$TT$L$PI$$ti_sysbios_hal_Hwi_startup__E
   1001c28d     0000622c     000056d4   appBLE_pem3.oem3 (.text:ti_sysbios_BIOS_startFunc__I)
ti_sysbios_family_arm_cc26xx_Timer_startup__E  $Tramp$TT$L$PI$$ti_sysbios_family_arm_cc26xx_Timer_startup__E
   1001b795     00006234     000056d0   appBLE_pem3.oem3 (.text:ti_sysbios_BIOS_startFunc__I)
xdc_runtime_System_atexit__E  $Tramp$TT$L$PI$$xdc_runtime_System_atexit__E
   1001c681     0000623c     000056c8   appBLE_pem3.oem3 (.text:ti_sysbios_BIOS_startFunc__I)
ti_sysbios_knl_Queue_enqueue__E  $Tramp$TT$L$PI$$ti_sysbios_knl_Queue_enqueue__E
   1001c1b5     00006244     000053ae   util.obj (.text:Util_enqueueMsg)
ti_sysbios_knl_Queue_put__E  $Tramp$TT$L$PI$$ti_sysbios_knl_Queue_put__E
   1001bf2d     0000624c     0000502e   sysbios.aem3 : mangled__BIOS_lib.obj (.text:ti_sysbios_family_arm_cc26xx_Power_registerNotify__E)
ti_sysbios_BIOS_setThreadType__E  $Tramp$TT$L$PI$$ti_sysbios_BIOS_setThreadType__E
   1001c045     00006254     00004fec   appBLE_pem3.oem3 (.text:ti_sysbios_BIOS_atExitFunc__I)
                             00005e1c   appBLE_pem3.oem3 (.text:ti_sysbios_BIOS_exitFunc__I)
ti_sysbios_hal_Hwi_create  $Tramp$TT$L$PI$$ti_sysbios_hal_Hwi_create
   1001ab79     0000625c     00004c40   ICall.obj (.text:ICall_primRegisterISR$10)
                             00004c74   ICall.obj (.text:ICall_primRegisterISR_Ext$10)
ti_sysbios_knl_Task_construct  $Tramp$TT$L$PI$$ti_sysbios_knl_Task_construct
   1001b125     00006264     00004546   peripheral.obj (.text:GAPRole_createTask)
                             00004606   simpleBLEPeripheral.obj (.text:SimpleBLEPeripheral_createTask)
xdc_runtime_System_exit__E  $Tramp$TT$L$PI$$xdc_runtime_System_exit__E
   1001c7d1     0000626c     000043f4   boot.aem3 : boot.oem3 (.text)
                             00005e22   appBLE_pem3.oem3 (.text:ti_sysbios_BIOS_exitFunc__I)
ti_sysbios_knl_Clock_construct  $Tramp$TT$L$PI$$ti_sysbios_knl_Clock_construct
   1001b579     00006274     0000425c   util.obj (.text:Util_constructClock)
ti_sysbios_knl_Semaphore_create  $Tramp$TT$L$PI$$ti_sysbios_knl_Semaphore_create
   1001b5ad     0000627c     000040cc   ICall.obj (.text:ICall_newTask$10)
                             000044bc   ICall.obj (.text:ICall_primCreateSemaphore$10)
ti_sysbios_knl_Task_create  $Tramp$TT$L$PI$$ti_sysbios_knl_Task_create
   1001ae19     00006284     00003586   ICall.obj (.text:ICall_createRemoteTasks)
                             00004500   ICall.obj (.text:ICall_primCreateTask$10)
ti_sysbios_knl_Task_Params__init__S  $Tramp$TT$L$PI$$ti_sysbios_knl_Task_Params__init__S
   1001c1d9     0000628c     0000356a   ICall.obj (.text:ICall_createRemoteTasks)
                             000044ea   ICall.obj (.text:ICall_primCreateTask$10)
                             00004526   peripheral.obj (.text:GAPRole_createTask)
                             000045e6   simpleBLEPeripheral.obj (.text:SimpleBLEPeripheral_createTask)
ti_sysbios_knl_Clock_create  $Tramp$TT$L$PI$$ti_sysbios_knl_Clock_create
   1001b3ed     00006294     000034fa   ICall.obj (.text:ICall_primSetTimer$10)
ti_sysbios_knl_Clock_Params__init__S  $Tramp$TT$L$PI$$ti_sysbios_knl_Clock_Params__init__S
   1001c185     0000629c     000034e6   ICall.obj (.text:ICall_primSetTimer$10)
                             00004236   util.obj (.text:Util_constructClock)
ti_sysbios_knl_Clock_scheduleNextTick__E  $Tramp$TT$L$PI$$ti_sysbios_knl_Clock_scheduleNextTick__E
   1001bebd     000062a4     00002b86   sysbios.aem3 : mangled__BIOS_lib.obj (.text:ti_sysbios_knl_Clock_workFuncDynamic__E)
ti_sysbios_knl_Clock_walkQueueDynamic__E  $Tramp$TT$L$PI$$ti_sysbios_knl_Clock_walkQueueDynamic__E
   1001a80d     000062ac     00002b48   sysbios.aem3 : mangled__BIOS_lib.obj (.text:ti_sysbios_knl_Clock_workFuncDynamic__E)
                             00002b66                : mangled__BIOS_lib.obj (.text:ti_sysbios_knl_Clock_workFuncDynamic__E)
ti_sysbios_family_arm_m3_Hwi_restoreFxn__E  $Tramp$TT$L$PI$$ti_sysbios_family_arm_m3_Hwi_restoreFxn__E
   1001c219     000062b4     00002980   PINCC26XX.obj (.text:PINCC26XX_setIoCfg$17)
                             00003ba0   appBLE_pem3.oem3 (.text:ti_sysbios_family_arm_cc26xx_Power_XOSC_HF_clockFunc__E)
                             00005dd8   ICall.obj (.text:ICall_leaveCSImpl)
ti_sysbios_family_arm_m3_Hwi_disableFxn__E  $Tramp$TT$L$PI$$ti_sysbios_family_arm_m3_Hwi_disableFxn__E
   1001c149     000062bc     00002960   PINCC26XX.obj (.text:PINCC26XX_setIoCfg$17)
                             00003b4e   appBLE_pem3.oem3 (.text:ti_sysbios_family_arm_cc26xx_Power_XOSC_HF_clockFunc__E)
                             00005a5c   ICall.obj (.text:ICall_enterCSImpl)
                             00005f70   ICall.obj (.text:ICall_primDisableMInt$10)
ti_sysbios_knl_Semaphore_post__E  $Tramp$TT$L$PI$$ti_sysbios_knl_Semaphore_post__E
   1001ac41     000062c4     0000264c   ICall.obj (.text:ICall_primWaitMatch$10)
                             00003070   PINCC26XX.obj (.text:PIN_open)
                             000036a2   ICall.obj (.text:ICall_primSend$10)
                             000036e4   simpleBLEPeripheral.obj (.text:adcIsr)
                             0000370c   simpleBLEPeripheral.obj (.text:adcIsr)
                             000053b6   util.obj (.text:Util_enqueueMsg)
                             00005caa   simpleBLEPeripheral.obj (.text:SimpleBLEPeripheral_mtrClockHandler$21)
                             00005cc2   simpleBLEPeripheral.obj (.text:SimpleBLEPeripheral_tempClockHandler$21)
                             00005cf4   simpleBLEPeripheral.obj (.text:buttonHwiFxn$21)
                             00005d0a   peripheral.obj (.text:gapRole_setEvent$6)
                             00006084   ICall.obj (.text:ICall_primSignal$10)
ti_sysbios_knl_Clock_getTicks__E  $Tramp$TT$L$PI$$ti_sysbios_knl_Clock_getTicks__E
   1001b6d9     000062cc     000025c4   ICall.obj (.text:ICall_primWaitMatch$10)
                             0000262e   ICall.obj (.text:ICall_primWaitMatch$10)
                             00005f98   ICall.obj (.text:ICall_primGetTicks$10)
ti_sysbios_knl_Task_self__E  $Tramp$TT$L$PI$$ti_sysbios_knl_Task_self__E
   1001c1e5     000062d4     0000257a   ICall.obj (.text:ICall_primWaitMatch$10)
                             00003d24   ICall.obj (.text:ICall_primEnroll$10)
                             00003e38   ICall.obj (.text:ICall_primThreadServes$10)
                             00003e7c   ICall.obj (.text:ICall_primWait$10)
                             00003fc0   ICall.obj (.text:ICall_primGetEntityId$10)
                             00004010   ICall.obj (.text:ICall_primRegisterApp$10)
                             00004bf0   ICall.obj (.text:ICall_primFetchMsg$10)
ti_sysbios_knl_Clock_stop__E  $Tramp$TT$L$PI$$ti_sysbios_knl_Clock_stop__E
   1001c225     000062dc     000024ee   sysbios.aem3 : mangled__BIOS_lib.obj (.text:ti_sysbios_family_arm_cc26xx_Power_standbyPolicy__E)
                             00003526   ICall.obj (.text:ICall_primSetTimer$10)
                             00004636   appBLE_pem3.oem3 (.text:ti_sysbios_family_arm_cc26xx_Power_XOSC_HF)
                             00004972   util.obj (.text:Util_restartClock)
                             00005dee   ICall.obj (.text:ICall_primStopTimer$10)
                             000061a2   util.obj (.text:Util_stopClock)
ti_sysbios_knl_Clock_start__E  $Tramp$TT$L$PI$$ti_sysbios_knl_Clock_start__E
   1001bfe3     000062e4     000024e0   sysbios.aem3 : mangled__BIOS_lib.obj (.text:ti_sysbios_family_arm_cc26xx_Power_standbyPolicy__E)
                             000030ee                : mangled__BIOS_lib.obj (.text:ti_sysbios_family_arm_cc26xx_Power_LF_clockFunc__E)
                             0000353e   ICall.obj (.text:ICall_primSetTimer$10)
                             00003b9a   appBLE_pem3.oem3 (.text:ti_sysbios_family_arm_cc26xx_Power_XOSC_HF_clockFunc__E)
                             00004644   appBLE_pem3.oem3 (.text:ti_sysbios_family_arm_cc26xx_Power_XOSC_HF)
                             00004990   util.obj (.text:Util_restartClock)
                             0000619e   util.obj (.text:Util_startClock)
ti_sysbios_knl_Clock_setTimeout__E  $Tramp$TT$L$PI$$ti_sysbios_knl_Clock_setTimeout__E
   1001c2c1     000062ec     000024d8   sysbios.aem3 : mangled__BIOS_lib.obj (.text:ti_sysbios_family_arm_cc26xx_Power_standbyPolicy__E)
                             000030e6                : mangled__BIOS_lib.obj (.text:ti_sysbios_family_arm_cc26xx_Power_LF_clockFunc__E)
                             00003538   ICall.obj (.text:ICall_primSetTimer$10)
                             00003b94   appBLE_pem3.oem3 (.text:ti_sysbios_family_arm_cc26xx_Power_XOSC_HF_clockFunc__E)
                             0000463e   appBLE_pem3.oem3 (.text:ti_sysbios_family_arm_cc26xx_Power_XOSC_HF)
                             0000498a   util.obj (.text:Util_restartClock)
ti_sysbios_knl_Clock_TimerProxy_getCurrentTick__E  $Tramp$TT$L$PI$$ti_sysbios_knl_Clock_TimerProxy_getCurrentTick__E
   1001c095     000062f4     000024a8   sysbios.aem3 : mangled__BIOS_lib.obj (.text:ti_sysbios_family_arm_cc26xx_Power_standbyPolicy__E)
                             00002b14                : mangled__BIOS_lib.obj (.text:ti_sysbios_knl_Clock_workFuncDynamic__E)
ti_sysbios_knl_Task_sleep__E  $Tramp$TT$L$PI$$ti_sysbios_knl_Task_sleep__E
   1001a96d     000062fc     00001fe2   simpleBLEPeripheral.obj (.text:SimpleBLEPeripheral_performPeriodicTemp$21)
ti_sysbios_family_arm_m3_Hwi_construct  $Tramp$TT$L$PI$$ti_sysbios_family_arm_m3_Hwi_construct
   1001af29     00006304     000011f4   simpleBLEPeripheral.obj (.text:SimpleBLEPeripheral_init$21)
                             00001d2e   PINCC26XX.obj (.text:PIN_init)
ti_sysbios_family_arm_m3_Hwi_Params__init__S  $Tramp$TT$L$PI$$ti_sysbios_family_arm_m3_Hwi_Params__init__S
   1001c13d     0000630c     000011de   simpleBLEPeripheral.obj (.text:SimpleBLEPeripheral_init$21)
                             00001d1c   PINCC26XX.obj (.text:PIN_init)
ti_sysbios_knl_Semaphore_construct  $Tramp$TT$L$PI$$ti_sysbios_knl_Semaphore_construct
   1001b709     00006314     000011d0   simpleBLEPeripheral.obj (.text:SimpleBLEPeripheral_init$21)
                             00001202   simpleBLEPeripheral.obj (.text:SimpleBLEPeripheral_init$21)
                             00001cbe   PINCC26XX.obj (.text:PIN_init)
ti_sysbios_knl_Semaphore_Params__init__S  $Tramp$TT$L$PI$$ti_sysbios_knl_Semaphore_Params__init__S
   1001c1c1     0000631c     000011be   simpleBLEPeripheral.obj (.text:SimpleBLEPeripheral_init$21)
                             00001caa   PINCC26XX.obj (.text:PIN_init)
                             000044a8   ICall.obj (.text:ICall_primCreateSemaphore$10)
ti_sysbios_knl_Task_restore__E  $Tramp$TT$L$PI$$ti_sysbios_knl_Task_restore__E
   1001ba49     00006324     00000f4e   sysbios.aem3 : mangled__BIOS_lib.obj (.text:ti_sysbios_family_arm_cc26xx_Power_sleep__E)
                             000035aa   ICall.obj (.text:ICall_createRemoteTasks)
                             00005de0   ICall.obj (.text:ICall_leaveCSImpl)
ti_sysbios_knl_Swi_restore__E  $Tramp$TT$L$PI$$ti_sysbios_knl_Swi_restore__E
   1001b5e1     0000632c     00000f44   sysbios.aem3 : mangled__BIOS_lib.obj (.text:ti_sysbios_family_arm_cc26xx_Power_sleep__E)
ti_sysbios_knl_Swi_disable__E  $Tramp$TT$L$PI$$ti_sysbios_knl_Swi_disable__E
   1001c0d5     00006334     00000d48   sysbios.aem3 : mangled__BIOS_lib.obj (.text:ti_sysbios_family_arm_cc26xx_Power_sleep__E)
                             00004fe2   appBLE_pem3.oem3 (.text:ti_sysbios_BIOS_atExitFunc__I)
ti_sysbios_knl_Queue_next__E  $Tramp$TT$L$PI$$ti_sysbios_knl_Queue_next__E
   1001c2d9     0000633c     00000d38   sysbios.aem3 : mangled__BIOS_lib.obj (.text:ti_sysbios_family_arm_cc26xx_Power_sleep__E)
                             00000ee0                : mangled__BIOS_lib.obj (.text:ti_sysbios_family_arm_cc26xx_Power_sleep__E)
                             00000f2a                : mangled__BIOS_lib.obj (.text:ti_sysbios_family_arm_cc26xx_Power_sleep__E)
                             00003daa                : mangled__BIOS_lib.obj (.text:ti_sysbios_family_arm_cc26xx_Power_notify__I)
ti_sysbios_knl_Queue_head__E  $Tramp$TT$L$PI$$ti_sysbios_knl_Queue_head__E
   1001c2d5     00006344     00000d18   sysbios.aem3 : mangled__BIOS_lib.obj (.text:ti_sysbios_family_arm_cc26xx_Power_sleep__E)
                             00000ec4                : mangled__BIOS_lib.obj (.text:ti_sysbios_family_arm_cc26xx_Power_sleep__E)
                             00000f0e                : mangled__BIOS_lib.obj (.text:ti_sysbios_family_arm_cc26xx_Power_sleep__E)
                             00003d90                : mangled__BIOS_lib.obj (.text:ti_sysbios_family_arm_cc26xx_Power_notify__I)
ti_sysbios_knl_Queue_empty__E  $Tramp$TT$L$PI$$ti_sysbios_knl_Queue_empty__E
   1001c113     0000634c     00000cfc   sysbios.aem3 : mangled__BIOS_lib.obj (.text:ti_sysbios_family_arm_cc26xx_Power_sleep__E)
                             00000eb0                : mangled__BIOS_lib.obj (.text:ti_sysbios_family_arm_cc26xx_Power_sleep__E)
                             00000f02                : mangled__BIOS_lib.obj (.text:ti_sysbios_family_arm_cc26xx_Power_sleep__E)
                             000026ea   simpleBLEPeripheral.obj (.text:SimpleBLEPeripheral_taskFxn$21)
                             00003d84   sysbios.aem3 : mangled__BIOS_lib.obj (.text:ti_sysbios_family_arm_cc26xx_Power_notify__I)
                             00005898   util.obj (.text:Util_dequeueMsg)
ti_sysbios_knl_Task_disable__E  $Tramp$TT$L$PI$$ti_sysbios_knl_Task_disable__E
   1001c0f5     00006354     00000cee   sysbios.aem3 : mangled__BIOS_lib.obj (.text:ti_sysbios_family_arm_cc26xx_Power_sleep__E)
                             00003554   ICall.obj (.text:ICall_createRemoteTasks)
                             00004fe6   appBLE_pem3.oem3 (.text:ti_sysbios_BIOS_atExitFunc__I)
                             00005a52   ICall.obj (.text:ICall_enterCSImpl)
                             00005f6c   ICall.obj (.text:ICall_primDisableMInt$10)

[54 trampolines]
[134 trampoline calls]


GLOBAL SYMBOLS: SORTED ALPHABETICALLY BY Name 

address   name                                                                      
-------   ----                                                                      
00005157  AONBatMonTemperatureGetDegC                                               
20002584  BoardGpioInitTable                                                        
0000440d  C$$EXIT                                                                   
00004b1d  ChipInfo_GetChipFamily                                                    
0000372d  ChipInfo_GetHwRevision                                                    
00005ad3  ChipInfo_GetPackageType                                                   
00005e29  DevInfo_AddService                                                        
00005eed  DevInfo_SetParameter                                                      
000048bd  GAPBondMgr_LinkEst                                                        
000055c7  GAPBondMgr_LinkTerm                                                       
00005185  GAPBondMgr_Register                                                       
00004b51  GAPBondMgr_SetParameter                                                   
00001d79  GAPRole_GetParameter                                                      
0000405d  GAPRole_SendUpdateParam                                                   
0000145d  GAPRole_SetParameter                                                      
0000598d  GAPRole_StartDevice                                                       
00005aed  GAPRole_TerminateConnection                                               
00004519  GAPRole_createTask                                                        
00003f1d  GAP_DeviceInit                                                            
00005efd  GAP_EndDiscoverable                                                       
00004719  GAP_GetParamValue                                                         
00006021  GAP_MakeDiscoverable                                                      
00006121  GAP_RegisterForMsgs                                                       
00004b85  GAP_SetParamValue                                                         
0000602d  GAP_TerminateAuth                                                         
00004341  GAP_TerminateLinkReq                                                      
00003f6d  GAP_UpdateAdvertisingData                                                 
00006039  GAP_UpdateLinkParamReq                                                    
000000fd  GATTServApp_AddService                                                    
000055ed  GATTServApp_FindAttr                                                      
00005775  GATTServApp_InitCharCfg                                                   
0000418d  GATTServApp_ProcessCCCWriteReq                                            
00003a21  GATTServApp_ProcessCharCfg                                                
00005f0d  GATTServApp_ReadCharCfg                                                   
00004755  GATTServApp_RegisterService                                               
000053e7  GATTServApp_WriteCharCfg                                                  
00006101  GATT_Indication                                                           
00005b05  GATT_Notification                                                         
00006127  GATT_RegisterForMsgs                                                      
00004559  GATT_SendRsp                                                              
00005795  GATT_bm_alloc                                                             
000059a9  GATT_bm_free                                                              
0000612d  GGS_AddService                                                            
00006045  GGS_SetParameter                                                          
000051b1  HCI_EXT_ConnEventNoticeCmd                                                
00004791  ICallPlatform_pwrConfigACAction                                           
00005bad  ICallPlatform_pwrDispense                                                 
00005f5d  ICallPlatform_pwrGetTransitionState                                       
00005f1d  ICallPlatform_pwrGetXOSCStartupTime                                       
00005e3d  ICallPlatform_pwrIsStableXOSCHF                                           
00003dd1  ICallPlatform_pwrRegisterNotify                                           
00005bc5  ICallPlatform_pwrRequire                                                  
000060ed  ICallPlatform_pwrSwitchXOSCHF                                             
00003811  ICallPlatform_pwrUpdActivityCounter                                       
0000354d  ICall_createRemoteTasks                                                   
200022c8  ICall_dispatcher                                                          
00005a51  ICall_enterCSImpl                                                         
200022d0  ICall_enterCriticalSection                                                
000051dd  ICall_freeImpl                                                            
000051dd  ICall_heapFree                                                            
00004f51  ICall_heapInit                                                            
00003445  ICall_heapMalloc                                                          
00005439  ICall_init                                                                
00005dd1  ICall_leaveCSImpl                                                         
200022d4  ICall_leaveCriticalSection                                                
00006133  ICall_mallocImpl                                                          
200016e8  LED_value                                                                 
00005311  NOROM_AONRTCCurrentCompareValueGet                                        
00002c51  NOROM_AUXADCDisable                                                       
0000319d  NOROM_AUXADCEnableSync                                                    
00005ec9  NOROM_AUXADCReadFifo                                                      
0000608d  NOROM_CPUcpsid                                                            
00006099  NOROM_CPUcpsie                                                            
000042f9  NOROM_DDI16BitfieldRead                                                   
00003cc5  NOROM_DDI16BitfieldWrite                                                  
000055a1  NOROM_OSCClockSourceGet                                                   
00003ecb  NOROM_OSCClockSourceSet                                                   
00004599  NOROM_OSCInterfaceEnable                                                  
00005fa3  NOROM_VIMSModeGet                                                         
00003a85  OSCHF_AttemptToSwitchToXosc                                               
00002ecd  OSCHF_GetStartupTime                                                      
00004df5  OSCHF_SwitchToRcOscTurnOffXosc                                            
00005a85  OSCHF_TurnOnXosc                                                          
20001558  PIN_HandleTable                                                           
200014f8  PIN_NumPins                                                               
00001bf1  PIN_init                                                                  
00002ff5  PIN_open                                                                  
00006139  PIN_registerIntCb                                                         
0000533d  PIN_setConfig                                                             
00004fb1  PIN_setOutputValue                                                        
000043c9  ResetISR                                                                  
UNDEFED   SHT$$INIT_ARRAY$$Base                                                     
UNDEFED   SHT$$INIT_ARRAY$$Limit                                                    
00004ae7  SafeHapiAuxAdiSelect                                                      
000045d9  SimpleBLEPeripheral_createTask                                            
00005501  SimpleProfile_AddService                                                  
00004385  SimpleProfile_GetParameter                                                
00005e51  SimpleProfile_RegisterAppCBs                                              
00003c0d  SimpleProfile_SetParameter                                                
00003ae9  SysCtrlAdjustRechargeAfterPowerDown                                       
00001875  SysCtrlSetRechargeBeforePowerDown                                         
0000387d  SysCtrl_DCDC_VoltageConditionalControl                                    
200023c4  TSK_idle                                                                  
00005e65  ThisCodeIsBuiltForCC26xxHwRev22AndLater_HaltIfViolated                    
00004221  Util_constructClock                                                       
00005ccd  Util_constructQueue                                                       
00005895  Util_dequeueMsg                                                           
00005393  Util_enqueueMsg                                                           
00005f4d  Util_isActive                                                             
00004965  Util_restartClock                                                         
0000619f  Util_startClock                                                           
000061a3  Util_stopClock                                                            
00000000  __ASM__                                                                   
00000068  __ISA__                                                                   
0000007a  __PLAT__                                                                  
200043e4  __STACK_END                                                               
00000400  __STACK_SIZE                                                              
200043e4  __STACK_TOP                                                               
000000a1  __TARG__                                                                  
00006d38  __TI_CINIT_Base                                                           
00006da0  __TI_CINIT_Limit                                                          
00006cd8  __TI_Handler_Table_Base                                                   
00006ce4  __TI_Handler_Table_Limit                                                  
00002cf1  __TI_auto_init                                                            
20002604  __TI_cleanup_ptr                                                          
00005fcd  __TI_decompress_none                                                      
00006145  __TI_decompress_rle24                                                     
20002608  __TI_dtors_ptr                                                            
000065c0  __TI_static_base__                                                        
000060a5  __TI_zero_init                                                            
000000c6  __TRDR__                                                                  
00003339  __aeabi_cdcmpeq                                                           
00003339  __aeabi_cdcmple                                                           
00001a45  __aeabi_dadd                                                              
000020a1  __aeabi_dmul                                                              
00001a3b  __aeabi_dsub                                                              
00005d2d  __aeabi_lmul                                                              
000035c9  __aeabi_memclr                                                            
000035c9  __aeabi_memclr4                                                           
000035c9  __aeabi_memclr8                                                           
00002e31  __aeabi_memcpy                                                            
00002e31  __aeabi_memcpy4                                                           
00002e31  __aeabi_memcpy8                                                           
000035cb  __aeabi_memset                                                            
000035cb  __aeabi_memset4                                                           
000035cb  __aeabi_memset8                                                           
000058b5  __aeabi_ui2d                                                              
00001681  __aeabi_uldivmod                                                          
ffffffff  __binit__                                                                 
ffffffff  __c_args__                                                                
0001ffa8  __ccfg                                                                    
20003fe4  __stack                                                                   
0000613f  __xdc__init                                                               
200022c4  __xdc__init__addr                                                         
00005d15  _args_main                                                                
000043c9  _c_int00                                                                  
200025fc  _lock                                                                     
00005e79  _nop                                                                      
00005e81  _register_lock                                                            
00005e7b  _register_unlock                                                          
20002600  _unlock                                                                   
00004411  abort                                                                     
20001728  adcFlag                                                                   
000036b9  adcIsr                                                                    
20001750  adcSamples                                                                
200017b0  adc_hwi                                                                   
000064c6  appearanceUUID                                                            
ffffffff  binit                                                                     
000064c2  charAggFormatUUID                                                         
000064b8  charExtPropsUUID                                                          
000064c0  charFormatUUID                                                            
000064ba  charUserDescUUID                                                          
000064ae  characterUUID                                                             
000064bc  clientCharCfgUUID                                                         
00004141  copy_in                                                                   
00006537  devInfo11073CertUUID                                                      
00006544  devInfoCBs                                                                
0000652f  devInfoFirmwareRevUUID                                                    
00006531  devInfoHardwareRevUUID                                                    
00006535  devInfoMfrNameUUID                                                        
0000652b  devInfoModelNumberUUID                                                    
00006539  devInfoPnpIdUUID                                                          
0000652d  devInfoSerialNumberUUID                                                   
00006527  devInfoServUUID                                                           
00006533  devInfoSoftwareRevUUID                                                    
00006529  devInfoSystemIdUUID                                                       
000064c4  deviceNameUUID                                                            
200016b8  driverlib_release_0_43243                                                 
00004419  exit                                                                      
000064d2  extReportRefUUID                                                          
20001c54  gapRoleTask                                                               
20001ca4  gapRoleTaskStack                                                          
00005cfd  gapRole_clockHandler                                                      
000064b0  gapServiceUUID                                                            
000064b2  gattServiceUUID                                                           
200016f0  hmtrsem                                                                   
200016ec  htempsem                                                                  
200016c8  i                                                                         
000064b6  includeUUID                                                               
200016f4  j                                                                         
200025e8  lastAppOpcodeSent                                                         
200016d0  led_blink_time                                                            
20001b40  linkDBNumConns                                                            
0000499d  linkDB_NumConns                                                           
00005933  main                                                                      
2000260c  main_func_sp                                                              
00002e31  memcpy                                                                    
000035d1  memset                                                                    
20001794  mtrsem                                                                    
00004d25  osal_snv_read                                                             
00004d59  osal_snv_write                                                            
000064cc  periConnParamUUID                                                         
000064c8  periPrivacyFlagUUID                                                       
200025ec  pfnBMAlloc                                                                
200025f0  pfnBMFree                                                                 
000064ac  primaryServiceUUID                                                        
000064ca  reconnectAddrUUID                                                         
000064d4  reportRefUUID                                                             
20002490  rfRegTbl                                                                  
20001718  sample_avg                                                                
20001720  sample_sum                                                                
20001834  sbpTask                                                                   
20001884  sbpTaskStack                                                              
000064b4  secondaryServiceUUID                                                      
000064be  servCharCfgUUID                                                           
000064ce  serviceChangedUUID                                                        
00006558  simpleProfileCBs                                                          
00006578  simpleProfileServUUID                                                     
0000657a  simpleProfilechar1UUID                                                    
0000657c  simpleProfilechar2UUID                                                    
0000657e  simpleProfilechar3UUID                                                    
00006580  simpleProfilechar4UUID                                                    
00006582  simpleProfilechar5UUID                                                    
200016dc  singleMtrSample                                                           
200016da  singleTempSample                                                          
00005e8d  strlen                                                                    
200016c0  temp_volt                                                                 
20001778  tempsem                                                                   
200001a4  ti_sysbios_BIOS_Module__state__V                                          
1001bc29  ti_sysbios_BIOS_RtsGateProxy_Handle__label__S                             
UNDEFED   ti_sysbios_BIOS_RtsGateProxy_Handle__label__S__mangled__                  
1001bab9  ti_sysbios_BIOS_RtsGateProxy_Object__delete__S                            
UNDEFED   ti_sysbios_BIOS_RtsGateProxy_Object__delete__S__mangled__                 
1001c179  ti_sysbios_BIOS_RtsGateProxy_Params__init__S                              
UNDEFED   ti_sysbios_BIOS_RtsGateProxy_Params__init__S__mangled__                   
1001c249  ti_sysbios_BIOS_RtsGateProxy_enter__E                                     
1001c24d  ti_sysbios_BIOS_RtsGateProxy_leave__E                                     
1001c275  ti_sysbios_BIOS_RtsGateProxy_query__E                                     
UNDEFED   ti_sysbios_BIOS_RtsGateProxy_query__E__mangled__                          
00004fe1  ti_sysbios_BIOS_atExitFunc__I                                             
00005e13  ti_sysbios_BIOS_exitFunc__I                                               
1001c035  ti_sysbios_BIOS_exit__E                                                   
1001bff9  ti_sysbios_BIOS_getCpuFreq__E                                             
000060bd  ti_sysbios_BIOS_getThreadType__E                                          
00000501  ti_sysbios_BIOS_nullFunc__I                                               
0000567d  ti_sysbios_BIOS_registerRTSLock__I                                        
000056a1  ti_sysbios_BIOS_removeRTSLock__I                                          
000058d5  ti_sysbios_BIOS_rtsLock__I                                                
00005d45  ti_sysbios_BIOS_rtsUnlock__I                                              
1001c045  ti_sysbios_BIOS_setThreadType__E                                          
000056c5  ti_sysbios_BIOS_startFunc__I                                              
1001c055  ti_sysbios_BIOS_start__E                                                  
00002999  ti_sysbios_family_arm_cc26xx_Boot_trimDevice                              
00003085  ti_sysbios_family_arm_cc26xx_Power_LF_clockFunc__E                        
0000659c  ti_sysbios_family_arm_cc26xx_Power_Module_State_clockObj__O               
000065a0  ti_sysbios_family_arm_cc26xx_Power_Module_State_lfClockObj__O             
000065a4  ti_sysbios_family_arm_cc26xx_Power_Module_State_notifyQ__O                
20002354  ti_sysbios_family_arm_cc26xx_Power_Module__state__V                       
00003111  ti_sysbios_family_arm_cc26xx_Power_Module_startup__E                      
000061ab  ti_sysbios_family_arm_cc26xx_Power_NOP                                    
00005d5d  ti_sysbios_family_arm_cc26xx_Power_RFCORECLKS                             
00004619  ti_sysbios_family_arm_cc26xx_Power_XOSC_HF                                
00003b4d  ti_sysbios_family_arm_cc26xx_Power_XOSC_HF_clockFunc__E                   
00000965  ti_sysbios_family_arm_cc26xx_Power_auxISR__E                              
2000221f  ti_sysbios_family_arm_cc26xx_Power_constraintCounts                       
00006418  ti_sysbios_family_arm_cc26xx_Power_db                                     
00000963  ti_sysbios_family_arm_cc26xx_Power_defaultClockFunc__E                    
0000238b  ti_sysbios_family_arm_cc26xx_Power_defaultNotifyTrapFunc__E               
000060c9  ti_sysbios_family_arm_cc26xx_Power_getTransitionState__E                  
00002ecd  ti_sysbios_family_arm_cc26xx_Power_getXoscStartupTime__E                  
00002bad  ti_sysbios_family_arm_cc26xx_Power_initiateCalibration__E                 
00005551  ti_sysbios_family_arm_cc26xx_Power_isDependencyActive                     
00004659  ti_sysbios_family_arm_cc26xx_Power_isStableXOSC_HF__E                     
000065a8  ti_sysbios_family_arm_cc26xx_Power_notifyTrapFunc__C                      
00003d79  ti_sysbios_family_arm_cc26xx_Power_notify__I                              
2000220c  ti_sysbios_family_arm_cc26xx_Power_refCount                               
00005011  ti_sysbios_family_arm_cc26xx_Power_registerNotify__E                      
00004881  ti_sysbios_family_arm_cc26xx_Power_releaseConstraint__E                   
00002815  ti_sysbios_family_arm_cc26xx_Power_releaseDependency__E                   
20002224  ti_sysbios_family_arm_cc26xx_Power_resourceHandlers                       
000049d5  ti_sysbios_family_arm_cc26xx_Power_setConstraint__E                       
0000273d  ti_sysbios_family_arm_cc26xx_Power_setDependency__E                       
00000cb1  ti_sysbios_family_arm_cc26xx_Power_sleep__E                               
00002481  ti_sysbios_family_arm_cc26xx_Power_standbyPolicy__E                       
0000219d  ti_sysbios_family_arm_cc26xx_Power_startFirstMeasurement__E               
00005041  ti_sysbios_family_arm_cc26xx_Power_switchXOSC_HF__E                       
000065ac  ti_sysbios_family_arm_cc26xx_Power_totalTicksSTANDBY__C                   
000065b0  ti_sysbios_family_arm_cc26xx_Power_wakeDelaySTANDBY__C                    
00000502  ti_sysbios_family_arm_cc26xx_Timer_Module__id__C                          
20002230  ti_sysbios_family_arm_cc26xx_Timer_Module__root__V                        
1001bb49  ti_sysbios_family_arm_cc26xx_Timer_Module__startupDone__S                 
200001e4  ti_sysbios_family_arm_cc26xx_Timer_Module__state__V                       
1001ba71  ti_sysbios_family_arm_cc26xx_Timer_Module_startup__E                      
20002410  ti_sysbios_family_arm_cc26xx_Timer_Object__table__V                       
000056e9  ti_sysbios_family_arm_cc26xx_Timer_dynamicStub__E                         
00005d75  ti_sysbios_family_arm_cc26xx_Timer_getCount64__E                          
00004699  ti_sysbios_family_arm_cc26xx_Timer_getCurrentTick__E                      
1001c251  ti_sysbios_family_arm_cc26xx_Timer_getExpiredTicks__E                     
00005579  ti_sysbios_family_arm_cc26xx_Timer_getMaxTicks__E                         
1001c255  ti_sysbios_family_arm_cc26xx_Timer_getPeriod__E                           
00004451  ti_sysbios_family_arm_cc26xx_Timer_initDevice__I                          
1001a469  ti_sysbios_family_arm_cc26xx_Timer_periodicStub__E                        
1001b769  ti_sysbios_family_arm_cc26xx_Timer_postInit__I                            
00003bad  ti_sysbios_family_arm_cc26xx_Timer_setNextTick__E                         
1001c259  ti_sysbios_family_arm_cc26xx_Timer_setPeriod__E                           
00004a0d  ti_sysbios_family_arm_cc26xx_Timer_setThreshold__I                        
000032b1  ti_sysbios_family_arm_cc26xx_Timer_start__E                               
00000484  ti_sysbios_family_arm_cc26xx_Timer_startupNeeded__C                       
1001b795  ti_sysbios_family_arm_cc26xx_Timer_startup__E                             
200001ec  ti_sysbios_family_arm_cc26xx_TimestampProvider_Module__state__V           
1001bb69  ti_sysbios_family_arm_cc26xx_TimestampProvider_Module_startup__E          
000058f5  ti_sysbios_family_arm_cc26xx_TimestampProvider_get32__E                   
1001b9d1  ti_sysbios_family_arm_cc26xx_TimestampProvider_get64__E                   
1001c12f  ti_sysbios_family_arm_cc26xx_TimestampProvider_getFreq__E                 
00000504  ti_sysbios_family_arm_cc26xx_TimestampProvider_useClockTimer__C           
00000488  ti_sysbios_family_arm_m3_Hwi_E_alreadyDefined__C                          
0000048c  ti_sysbios_family_arm_m3_Hwi_E_hwiLimitExceeded__C                        
1001aed1  ti_sysbios_family_arm_m3_Hwi_Instance_finalize__E                         
1001a3c9  ti_sysbios_family_arm_m3_Hwi_Instance_init__E                             
20002240  ti_sysbios_family_arm_m3_Hwi_Module_State_0_excActive__A                  
20002244  ti_sysbios_family_arm_m3_Hwi_Module_State_0_excContext__A                 
20002248  ti_sysbios_family_arm_m3_Hwi_Module_State_0_excStack__A                   
00000506  ti_sysbios_family_arm_m3_Hwi_Module__id__C                                
20002238  ti_sysbios_family_arm_m3_Hwi_Module__root__V                              
1001bb89  ti_sysbios_family_arm_m3_Hwi_Module__startupDone__S                       
20000144  ti_sysbios_family_arm_m3_Hwi_Module__state__V                             
1001b1c1  ti_sysbios_family_arm_m3_Hwi_Module_startup__E                            
00000490  ti_sysbios_family_arm_m3_Hwi_NUM_INTERRUPTS__C                            
000002d0  ti_sysbios_family_arm_m3_Hwi_Object__DESC__C                              
00000170  ti_sysbios_family_arm_m3_Hwi_Object__PARAMS__C                            
00000494  ti_sysbios_family_arm_m3_Hwi_Object__count__C                             
1001aab1  ti_sysbios_family_arm_m3_Hwi_Object__create__S                            
1001bba9  ti_sysbios_family_arm_m3_Hwi_Object__delete__S                            
1001be69  ti_sysbios_family_arm_m3_Hwi_Object__destruct__S                          
1001b7c1  ti_sysbios_family_arm_m3_Hwi_Object__get__S                               
00000498  ti_sysbios_family_arm_m3_Hwi_Object__table__C                             
200024c4  ti_sysbios_family_arm_m3_Hwi_Object__table__V                             
1001c13d  ti_sysbios_family_arm_m3_Hwi_Params__init__S                              
0000049c  ti_sysbios_family_arm_m3_Hwi_ccr__C                                       
1001af29  ti_sysbios_family_arm_m3_Hwi_construct                                    
1001ab15  ti_sysbios_family_arm_m3_Hwi_create                                       
1001c25d  ti_sysbios_family_arm_m3_Hwi_delete                                       
1001c261  ti_sysbios_family_arm_m3_Hwi_destruct                                     
1001c149  ti_sysbios_family_arm_m3_Hwi_disableFxn__E                                
1001b299  ti_sysbios_family_arm_m3_Hwi_disableInterrupt__E                          
000065b4  ti_sysbios_family_arm_m3_Hwi_disablePriority__C                           
1001aa49  ti_sysbios_family_arm_m3_Hwi_dispatchC__I                                 
200015d4  ti_sysbios_family_arm_m3_Hwi_dispatchTable                                
1001c89d  ti_sysbios_family_arm_m3_Hwi_dispatch__I                                  
1001c1fb  ti_sysbios_family_arm_m3_Hwi_doSwiRestore__I                              
1001c213  ti_sysbios_family_arm_m3_Hwi_doTaskRestore__I                             
1001c155  ti_sysbios_family_arm_m3_Hwi_enableFxn__E                                 
1001b2dd  ti_sysbios_family_arm_m3_Hwi_enableInterrupt__E                           
1001ca01  ti_sysbios_family_arm_m3_Hwi_excHandlerAsm__I                             
000004a0  ti_sysbios_family_arm_m3_Hwi_excHandlerFunc__C                            
1001bbc9  ti_sysbios_family_arm_m3_Hwi_excHandler__I                                
1001b465  ti_sysbios_family_arm_m3_Hwi_getStackInfo__E                              
1001a699  ti_sysbios_family_arm_m3_Hwi_initNVIC__E                                  
1001c9b9  ti_sysbios_family_arm_m3_Hwi_initStacks__E                                
000004a4  ti_sysbios_family_arm_m3_Hwi_nullIsrFunc__C                               
000004a8  ti_sysbios_family_arm_m3_Hwi_numSparseInterrupts__C                       
e000e000  ti_sysbios_family_arm_m3_Hwi_nvic                                         
1001ca3f  ti_sysbios_family_arm_m3_Hwi_pendSV__I                                    
1001c065  ti_sysbios_family_arm_m3_Hwi_plug__E                                      
1001a319  ti_sysbios_family_arm_m3_Hwi_postInit__I                                  
000004ac  ti_sysbios_family_arm_m3_Hwi_priGroup__C                                  
20000000  ti_sysbios_family_arm_m3_Hwi_ramVectors                                   
00000000  ti_sysbios_family_arm_m3_Hwi_resetVectors                                 
1001c219  ti_sysbios_family_arm_m3_Hwi_restoreFxn__E                                
1001ca57  ti_sysbios_family_arm_m3_Hwi_return                                       
1001be85  ti_sysbios_family_arm_m3_Hwi_setPriority__E                               
1001c203  ti_sysbios_family_arm_m3_Hwi_startup__E                                   
1001c00d  ti_sysbios_family_arm_m3_Hwi_switchFromBootStack__E                       
1001c265  ti_sysbios_family_arm_m3_TaskSupport_Module__startupDone__S               
1001c96d  ti_sysbios_family_arm_m3_TaskSupport_buildTaskStack                       
1001c161  ti_sysbios_family_arm_m3_TaskSupport_getStackAlignment__E                 
1001ca59  ti_sysbios_family_arm_m3_TaskSupport_glue                                 
000004b0  ti_sysbios_family_arm_m3_TaskSupport_stackAlignment__C                    
1001b49d  ti_sysbios_family_arm_m3_TaskSupport_start__E                             
1001ca69  ti_sysbios_family_arm_m3_TaskSupport_swap__E                              
1001ca21  ti_sysbios_family_xxx_Hwi_switchAndRunFunc                                
1001bbe9  ti_sysbios_gates_GateHwi_Handle__label__S                                 
1001b463  ti_sysbios_gates_GateHwi_Instance_init__E                                 
0000021c  ti_sysbios_gates_GateHwi_Module__FXNS__C                                  
00000508  ti_sysbios_gates_GateHwi_Module__id__C                                    
2000224c  ti_sysbios_gates_GateHwi_Module__root__V                                  
000002f0  ti_sysbios_gates_GateHwi_Object__DESC__C                                  
00000430  ti_sysbios_gates_GateHwi_Object__PARAMS__C                                
1001ba95  ti_sysbios_gates_GateHwi_Object__create__S                                
1001bc09  ti_sysbios_gates_GateHwi_Object__delete__S                                
20002254  ti_sysbios_gates_GateHwi_Object__table__V                                 
1001c16d  ti_sysbios_gates_GateHwi_enter__E                                         
1001c21f  ti_sysbios_gates_GateHwi_leave__E                                         
1001c269  ti_sysbios_gates_GateHwi_query__E                                         
1001bc29  ti_sysbios_gates_GateMutex_Handle__label__S                               
000005cc  ti_sysbios_gates_GateMutex_Instance_State_sem__O                          
1001c075  ti_sysbios_gates_GateMutex_Instance_finalize__E                           
1001bea1  ti_sysbios_gates_GateMutex_Instance_init__E                               
00000240  ti_sysbios_gates_GateMutex_Module__FXNS__C                                
0000050a  ti_sysbios_gates_GateMutex_Module__id__C                                  
20002258  ti_sysbios_gates_GateMutex_Module__root__V                                
00000310  ti_sysbios_gates_GateMutex_Object__DESC__C                                
00000448  ti_sysbios_gates_GateMutex_Object__PARAMS__C                              
1001b649  ti_sysbios_gates_GateMutex_Object__create__S                              
1001bab9  ti_sysbios_gates_GateMutex_Object__delete__S                              
1001bc49  ti_sysbios_gates_GateMutex_Object__destruct__S                            
20002458  ti_sysbios_gates_GateMutex_Object__table__V                               
1001c179  ti_sysbios_gates_GateMutex_Params__init__S                                
1001b7ed  ti_sysbios_gates_GateMutex_construct                                      
1001b679  ti_sysbios_gates_GateMutex_create                                         
1001c26d  ti_sysbios_gates_GateMutex_delete                                         
1001c271  ti_sysbios_gates_GateMutex_destruct                                       
1001b6a9  ti_sysbios_gates_GateMutex_enter__E                                       
1001bf9d  ti_sysbios_gates_GateMutex_leave__E                                       
1001c275  ti_sysbios_gates_GateMutex_query__E                                       
1001c279  ti_sysbios_hal_Hwi_HwiProxy_Module__startupDone__S                        
UNDEFED   ti_sysbios_hal_Hwi_HwiProxy_Module__startupDone__S__mangled__             
1001c085  ti_sysbios_hal_Hwi_HwiProxy_Object__create__S                             
1001bba9  ti_sysbios_hal_Hwi_HwiProxy_Object__delete__S                             
UNDEFED   ti_sysbios_hal_Hwi_HwiProxy_Object__delete__S__mangled__                  
1001c13d  ti_sysbios_hal_Hwi_HwiProxy_Params__init__S                               
UNDEFED   ti_sysbios_hal_Hwi_HwiProxy_Params__init__S__mangled__                    
1001be49  ti_sysbios_hal_Hwi_HwiProxy_create                                        
1001c27d  ti_sysbios_hal_Hwi_HwiProxy_delete                                        
1001c281  ti_sysbios_hal_Hwi_HwiProxy_disableInterrupt__E                           
UNDEFED   ti_sysbios_hal_Hwi_HwiProxy_disableInterrupt__E__mangled__                
1001c285  ti_sysbios_hal_Hwi_HwiProxy_enableInterrupt__E                            
UNDEFED   ti_sysbios_hal_Hwi_HwiProxy_enableInterrupt__E__mangled__                 
1001c289  ti_sysbios_hal_Hwi_HwiProxy_getStackInfo__E                               
UNDEFED   ti_sysbios_hal_Hwi_HwiProxy_getStackInfo__E__mangled__                    
1001c28d  ti_sysbios_hal_Hwi_HwiProxy_startup__E                                    
UNDEFED   ti_sysbios_hal_Hwi_HwiProxy_startup__E__mangled__                         
1001c291  ti_sysbios_hal_Hwi_HwiProxy_switchFromBootStack__E                        
UNDEFED   ti_sysbios_hal_Hwi_HwiProxy_switchFromBootStack__E__mangled__             
1001c1f1  ti_sysbios_hal_Hwi_Instance_finalize__E                                   
1001b9f9  ti_sysbios_hal_Hwi_Instance_init__E                                       
20002260  ti_sysbios_hal_Hwi_Module__root__V                                        
1001c021  ti_sysbios_hal_Hwi_Module_startup__E                                      
00000330  ti_sysbios_hal_Hwi_Object__DESC__C                                        
000001a0  ti_sysbios_hal_Hwi_Object__PARAMS__C                                      
1001bc69  ti_sysbios_hal_Hwi_Object__delete__S                                      
000060d5  ti_sysbios_hal_Hwi_Params__init__S                                        
1001ab79  ti_sysbios_hal_Hwi_create                                                 
1001c295  ti_sysbios_hal_Hwi_delete                                                 
1001c281  ti_sysbios_hal_Hwi_disableInterrupt__E                                    
UNDEFED   ti_sysbios_hal_Hwi_disableInterrupt__E__mangled__                         
1001c285  ti_sysbios_hal_Hwi_enableInterrupt__E                                     
UNDEFED   ti_sysbios_hal_Hwi_enableInterrupt__E__mangled__                          
1001c289  ti_sysbios_hal_Hwi_getStackInfo__E                                        
UNDEFED   ti_sysbios_hal_Hwi_getStackInfo__E__mangled__                             
1001b819  ti_sysbios_hal_Hwi_initStack                                              
1001c28d  ti_sysbios_hal_Hwi_startup__E                                             
UNDEFED   ti_sysbios_hal_Hwi_startup__E__mangled__                                  
1001c299  ti_sysbios_hal_Hwi_switchFromBootStack__E                                 
UNDEFED   ti_sysbios_hal_Hwi_switchFromBootStack__E__mangled__                      
000004b4  ti_sysbios_heaps_HeapMem_E_memory__C                                      
1001bc89  ti_sysbios_heaps_HeapMem_Handle__label__S                                 
20000c78  ti_sysbios_heaps_HeapMem_Instance_State_0_buf__A                          
1001b4d5  ti_sysbios_heaps_HeapMem_Instance_init__E                                 
1001bc29  ti_sysbios_heaps_HeapMem_Module_GateProxy_Handle__label__S                
UNDEFED   ti_sysbios_heaps_HeapMem_Module_GateProxy_Handle__label__S__mangled__     
1001bab9  ti_sysbios_heaps_HeapMem_Module_GateProxy_Object__delete__S               
UNDEFED   ti_sysbios_heaps_HeapMem_Module_GateProxy_Object__delete__S__mangled__    
1001c179  ti_sysbios_heaps_HeapMem_Module_GateProxy_Params__init__S                 
UNDEFED   ti_sysbios_heaps_HeapMem_Module_GateProxy_Params__init__S__mangled__      
1001c29d  ti_sysbios_heaps_HeapMem_Module_GateProxy_enter__E                        
1001c2a1  ti_sysbios_heaps_HeapMem_Module_GateProxy_leave__E                        
1001c275  ti_sysbios_heaps_HeapMem_Module_GateProxy_query__E                        
UNDEFED   ti_sysbios_heaps_HeapMem_Module_GateProxy_query__E__mangled__             
000001cc  ti_sysbios_heaps_HeapMem_Module__FXNS__C                                  
000004b8  ti_sysbios_heaps_HeapMem_Module__gateObj__C                               
0000050c  ti_sysbios_heaps_HeapMem_Module__id__C                                    
20002268  ti_sysbios_heaps_HeapMem_Module__root__V                                  
00000350  ti_sysbios_heaps_HeapMem_Object__DESC__C                                  
00000264  ti_sysbios_heaps_HeapMem_Object__PARAMS__C                                
000004bc  ti_sysbios_heaps_HeapMem_Object__count__C                                 
1001b845  ti_sysbios_heaps_HeapMem_Object__create__S                                
1001bca9  ti_sysbios_heaps_HeapMem_Object__delete__S                                
1001b871  ti_sysbios_heaps_HeapMem_Object__get__S                                   
000004c0  ti_sysbios_heaps_HeapMem_Object__table__C                                 
20002270  ti_sysbios_heaps_HeapMem_Object__table__V                                 
1001a199  ti_sysbios_heaps_HeapMem_alloc__E                                         
1001a795  ti_sysbios_heaps_HeapMem_free__E                                          
1001b209  ti_sysbios_heaps_HeapMem_getStats__E                                      
1001b545  ti_sysbios_heaps_HeapMem_init__I                                          
1001c2a5  ti_sysbios_heaps_HeapMem_isBlocking__E                                    
000004c4  ti_sysbios_heaps_HeapMem_reqAlign__C                                      
1001c105  ti_sysbios_heaps_HeapMem_restore__E                                       
1001bfcd  ti_sysbios_knl_Clock_Instance_finalize__E                                 
1001b50d  ti_sysbios_knl_Clock_Instance_init__E                                     
000005d0  ti_sysbios_knl_Clock_Module_State_clockQ__O                               
20002288  ti_sysbios_knl_Clock_Module__root__V                                      
20000178  ti_sysbios_knl_Clock_Module__state__V                                     
1001bcc9  ti_sysbios_knl_Clock_Module_startup__E                                    
00000370  ti_sysbios_knl_Clock_Object__DESC__C                                      
00000288  ti_sysbios_knl_Clock_Object__PARAMS__C                                    
1001badd  ti_sysbios_knl_Clock_Object__delete__S                                    
1001bce9  ti_sysbios_knl_Clock_Object__destruct__S                                  
1001c185  ti_sysbios_knl_Clock_Params__init__S                                      
1001c2a9  ti_sysbios_knl_Clock_TimerProxy_Module__startupDone__S                    
UNDEFED   ti_sysbios_knl_Clock_TimerProxy_Module__startupDone__S__mangled__         
1001c095  ti_sysbios_knl_Clock_TimerProxy_getCurrentTick__E                         
1001c2ad  ti_sysbios_knl_Clock_TimerProxy_getExpiredTicks__E                        
1001c0a5  ti_sysbios_knl_Clock_TimerProxy_getMaxTicks__E                            
1001c2b1  ti_sysbios_knl_Clock_TimerProxy_getPeriod__E                              
1001c0b5  ti_sysbios_knl_Clock_TimerProxy_setNextTick__E                            
1001b795  ti_sysbios_knl_Clock_TimerProxy_startup__E                                
UNDEFED   ti_sysbios_knl_Clock_TimerProxy_startup__E__mangled__                     
1001ba21  ti_sysbios_knl_Clock_addI__E                                              
1001b579  ti_sysbios_knl_Clock_construct                                            
1001b3ed  ti_sysbios_knl_Clock_create                                               
1001c2b5  ti_sysbios_knl_Clock_delete                                               
1001c2b9  ti_sysbios_knl_Clock_destruct                                             
00005eb5  ti_sysbios_knl_Clock_doTick__I                                            
1001b6d9  ti_sysbios_knl_Clock_getTicks__E                                          
1001c191  ti_sysbios_knl_Clock_getTimerHandle__E                                    
000061af  ti_sysbios_knl_Clock_isActive__E                                          
1001be67  ti_sysbios_knl_Clock_logTick__E                                           
1001c2bd  ti_sysbios_knl_Clock_removeI__E                                           
1001bebd  ti_sysbios_knl_Clock_scheduleNextTick__E                                  
000004c8  ti_sysbios_knl_Clock_serviceMargin__C                                     
1001c2c1  ti_sysbios_knl_Clock_setTimeout__E                                        
1001a719  ti_sysbios_knl_Clock_startI__E                                            
1001bfe3  ti_sysbios_knl_Clock_start__E                                             
1001c225  ti_sysbios_knl_Clock_stop__E                                              
00000510  ti_sysbios_knl_Clock_tickMode__C                                          
000065b8  ti_sysbios_knl_Clock_tickPeriod__C                                        
1001a80d  ti_sysbios_knl_Clock_walkQueueDynamic__E                                  
00002afd  ti_sysbios_knl_Clock_workFuncDynamic__E                                   
1001a885  ti_sysbios_knl_Clock_workFunc__E                                          
20002290  ti_sysbios_knl_Event_Module__root__V                                      
000065bc  ti_sysbios_knl_Idle_funcList__A                                           
00000478  ti_sysbios_knl_Idle_funcList__C                                           
1001c20b  ti_sysbios_knl_Idle_loop__E                                               
1001bd09  ti_sysbios_knl_Idle_run__E                                                
000005d4  ti_sysbios_knl_Mailbox_Instance_State_dataQue__O                          
000005d8  ti_sysbios_knl_Mailbox_Instance_State_dataSem__O                          
000005dc  ti_sysbios_knl_Mailbox_Instance_State_freeQue__O                          
000005e0  ti_sysbios_knl_Mailbox_Instance_State_freeSem__O                          
1001a9dd  ti_sysbios_knl_Mailbox_Instance_finalize__E                               
1001a001  ti_sysbios_knl_Mailbox_Instance_init__E                                   
20002298  ti_sysbios_knl_Mailbox_Module__root__V                                    
1001b251  ti_sysbios_knl_Mailbox_Module_startup__E                                  
00000390  ti_sysbios_knl_Mailbox_Object__DESC__C                                    
0000013c  ti_sysbios_knl_Mailbox_Object__PARAMS__C                                  
000004cc  ti_sysbios_knl_Mailbox_Object__count__C                                   
1001bd29  ti_sysbios_knl_Mailbox_Object__delete__S                                  
1001bed9  ti_sysbios_knl_Mailbox_Object__destruct__S                                
1001b89d  ti_sysbios_knl_Mailbox_Object__get__S                                     
000004d0  ti_sysbios_knl_Mailbox_Object__table__C                                   
1001c19d  ti_sysbios_knl_Mailbox_Params__init__S                                    
1001af81  ti_sysbios_knl_Mailbox_construct                                          
1001abdd  ti_sysbios_knl_Mailbox_create                                             
1001c2c5  ti_sysbios_knl_Mailbox_delete                                             
1001c2c9  ti_sysbios_knl_Mailbox_destruct                                           
1001a8fd  ti_sysbios_knl_Mailbox_pend__E                                            
1001b8c9  ti_sysbios_knl_Mailbox_postInit__I                                        
1001a591  ti_sysbios_knl_Mailbox_post__E                                            
1001c22b  ti_sysbios_knl_Queue_Instance_init__E                                     
200022a0  ti_sysbios_knl_Queue_Module__root__V                                      
000003b0  ti_sysbios_knl_Queue_Object__DESC__C                                      
00000460  ti_sysbios_knl_Queue_Object__PARAMS__C                                    
000004d4  ti_sysbios_knl_Queue_Object__count__C                                     
1001bd49  ti_sysbios_knl_Queue_Object__delete__S                                    
1001bef5  ti_sysbios_knl_Queue_Object__destruct__S                                  
1001bd69  ti_sysbios_knl_Queue_Object__get__S                                       
000004d8  ti_sysbios_knl_Queue_Object__table__C                                     
1001b8f5  ti_sysbios_knl_Queue_construct                                            
1001b921  ti_sysbios_knl_Queue_create                                               
1001c2cd  ti_sysbios_knl_Queue_delete                                               
1001c1a9  ti_sysbios_knl_Queue_dequeue__E                                           
1001c2d1  ti_sysbios_knl_Queue_destruct                                             
1001c231  ti_sysbios_knl_Queue_elemClear__E                                         
1001c113  ti_sysbios_knl_Queue_empty__E                                             
1001c1b5  ti_sysbios_knl_Queue_enqueue__E                                           
1001bf11  ti_sysbios_knl_Queue_get__E                                               
1001c2d5  ti_sysbios_knl_Queue_head__E                                              
1001c2d9  ti_sysbios_knl_Queue_next__E                                              
1001bf2d  ti_sysbios_knl_Queue_put__E                                               
1001c121  ti_sysbios_knl_Queue_remove__E                                            
000005e4  ti_sysbios_knl_Semaphore_Instance_State_pendQ__O                          
1001c0c5  ti_sysbios_knl_Semaphore_Instance_finalize__E                             
1001bb01  ti_sysbios_knl_Semaphore_Instance_init__E                                 
200022a8  ti_sysbios_knl_Semaphore_Module__root__V                                  
000003d0  ti_sysbios_knl_Semaphore_Object__DESC__C                                  
000002ac  ti_sysbios_knl_Semaphore_Object__PARAMS__C                                
1001bb25  ti_sysbios_knl_Semaphore_Object__delete__S                                
1001bd89  ti_sysbios_knl_Semaphore_Object__destruct__S                              
1001c1c1  ti_sysbios_knl_Semaphore_Params__init__S                                  
1001b709  ti_sysbios_knl_Semaphore_construct                                        
1001b5ad  ti_sysbios_knl_Semaphore_create                                           
1001c2dd  ti_sysbios_knl_Semaphore_delete                                           
1001c2e1  ti_sysbios_knl_Semaphore_destruct                                         
1001b94d  ti_sysbios_knl_Semaphore_pendTimeout__I                                   
1001a0cd  ti_sysbios_knl_Semaphore_pend__E                                          
1001ac41  ti_sysbios_knl_Semaphore_post__E                                          
1001bf9b  ti_sysbios_knl_Swi_Instance_finalize__E                                   
1001aca5  ti_sysbios_knl_Swi_Instance_init__E                                       
200024f4  ti_sysbios_knl_Swi_Module_State_0_readyQ__A                               
200022b0  ti_sysbios_knl_Swi_Module__root__V                                        
200001c8  ti_sysbios_knl_Swi_Module__state__V                                       
1001c237  ti_sysbios_knl_Swi_Module_startup__E                                      
000003f0  ti_sysbios_knl_Swi_Object__DESC__C                                        
000001f4  ti_sysbios_knl_Swi_Object__PARAMS__C                                      
000004dc  ti_sysbios_knl_Swi_Object__count__C                                       
1001bda9  ti_sysbios_knl_Swi_Object__delete__S                                      
1001bf49  ti_sysbios_knl_Swi_Object__destruct__S                                    
1001b979  ti_sysbios_knl_Swi_Object__get__S                                         
000004e0  ti_sysbios_knl_Swi_Object__table__C                                       
20002524  ti_sysbios_knl_Swi_Object__table__V                                       
1001c1cd  ti_sysbios_knl_Swi_Params__init__S                                        
1001b085  ti_sysbios_knl_Swi_construct                                              
1001ad05  ti_sysbios_knl_Swi_create                                                 
1001c2e5  ti_sysbios_knl_Swi_delete                                                 
1001c2e9  ti_sysbios_knl_Swi_destruct                                               
1001c0d5  ti_sysbios_knl_Swi_disable__E                                             
1001c0e5  ti_sysbios_knl_Swi_enabled__E                                             
000004e4  ti_sysbios_knl_Swi_numPriorities__C                                       
1001c2ed  ti_sysbios_knl_Swi_postInit__I                                            
1001b321  ti_sysbios_knl_Swi_post__E                                                
1001ad61  ti_sysbios_knl_Swi_restoreHwi__E                                          
1001b5e1  ti_sysbios_knl_Swi_restore__E                                             
1001b0d5  ti_sysbios_knl_Swi_runLoop__I                                             
1001afd9  ti_sysbios_knl_Swi_run__I                                                 
1001b031  ti_sysbios_knl_Swi_schedule__I                                            
1001c23d  ti_sysbios_knl_Swi_startup__E                                             
200012f8  ti_sysbios_knl_Task_Instance_State_0_stack__A                             
1001a4fd  ti_sysbios_knl_Task_Instance_finalize__E                                  
1001a25d  ti_sysbios_knl_Task_Instance_init__E                                      
200022c0  ti_sysbios_knl_Task_Module_State_0_idleTask__A                            
20002554  ti_sysbios_knl_Task_Module_State_0_readyQ__A                              
000005e8  ti_sysbios_knl_Task_Module_State_inactiveQ__O                             
200022b8  ti_sysbios_knl_Task_Module__root__V                                       
20000100  ti_sysbios_knl_Task_Module__state__V                                      
1001adbd  ti_sysbios_knl_Task_Module_startup__E                                     
00000410  ti_sysbios_knl_Task_Object__DESC__C                                       
00000100  ti_sysbios_knl_Task_Object__PARAMS__C                                     
000004e8  ti_sysbios_knl_Task_Object__count__C                                      
1001bdc9  ti_sysbios_knl_Task_Object__delete__S                                     
1001bf65  ti_sysbios_knl_Task_Object__destruct__S                                   
1001bde9  ti_sysbios_knl_Task_Object__get__S                                        
000004ec  ti_sysbios_knl_Task_Object__table__C                                      
200023c4  ti_sysbios_knl_Task_Object__table__V                                      
1001c1d9  ti_sysbios_knl_Task_Params__init__S                                       
1001c2f1  ti_sysbios_knl_Task_SupportProxy_Module__startupDone__S                   
UNDEFED   ti_sysbios_knl_Task_SupportProxy_Module__startupDone__S__mangled__        
1001c2f5  ti_sysbios_knl_Task_SupportProxy_getStackAlignment__E                     
UNDEFED   ti_sysbios_knl_Task_SupportProxy_getStackAlignment__E__mangled__          
1001c2f9  ti_sysbios_knl_Task_SupportProxy_start__E                                 
UNDEFED   ti_sysbios_knl_Task_SupportProxy_start__E__mangled__                      
1001c2fd  ti_sysbios_knl_Task_SupportProxy_swap__E                                  
UNDEFED   ti_sysbios_knl_Task_SupportProxy_swap__E__mangled__                       
000004f0  ti_sysbios_knl_Task_allBlockedFunc__C                                     
1001b365  ti_sysbios_knl_Task_allBlockedFunction__I                                 
1001b615  ti_sysbios_knl_Task_blockI__E                                             
1001b125  ti_sysbios_knl_Task_construct                                             
1001ae19  ti_sysbios_knl_Task_create                                                
000004f4  ti_sysbios_knl_Task_defaultStackHeap__C                                   
000004f8  ti_sysbios_knl_Task_defaultStackSize__C                                   
1001c301  ti_sysbios_knl_Task_delete                                                
1001c305  ti_sysbios_knl_Task_destruct                                              
1001c0f5  ti_sysbios_knl_Task_disable__E                                            
1001c243  ti_sysbios_knl_Task_enable__E                                             
1001be09  ti_sysbios_knl_Task_enter__I                                              
1001b429  ti_sysbios_knl_Task_exit__E                                               
0000050e  ti_sysbios_knl_Task_initStackFlag__C                                      
000004fc  ti_sysbios_knl_Task_numConstructedTasks__C                                
1001a615  ti_sysbios_knl_Task_postInit__I                                           
1001b739  ti_sysbios_knl_Task_processVitalTaskFlag__I                               
1001be29  ti_sysbios_knl_Task_restoreHwi__E                                         
1001ba49  ti_sysbios_knl_Task_restore__E                                            
1001b175  ti_sysbios_knl_Task_schedule__I                                           
1001c1e5  ti_sysbios_knl_Task_self__E                                               
1001bf81  ti_sysbios_knl_Task_sleepTimeout__I                                       
1001a96d  ti_sysbios_knl_Task_sleep__E                                              
1001ae75  ti_sysbios_knl_Task_startCore__E                                          
1001c309  ti_sysbios_knl_Task_startup__E                                            
1001ca71  ti_sysbios_knl_Task_swapReturn                                            
1001b9a5  ti_sysbios_knl_Task_unblockI__E                                           
1001bfb5  ti_sysbios_knl_Task_unblock__E                                            
1001b3a9  ti_sysbios_knl_Task_yield__E                                              
00000590  ti_sysbios_rom_ROM_AONRTCChannelEnable                                    
00000594  ti_sysbios_rom_ROM_AONRTCCompareValueSet                                  
00000598  ti_sysbios_rom_ROM_AONRTCCurrentCompareValueGet                           
0000059c  ti_sysbios_rom_ROM_AONRTCEventClear                                       
000005a0  ti_sysbios_rom_ROM_ti_sysbios_family_arm_cc26xx_Timer_getCount64__E       
000005a4  ti_sysbios_rom_ROM_ti_sysbios_family_arm_cc26xx_Timer_getCurrentTick__E   
000005a8  ti_sysbios_rom_ROM_ti_sysbios_family_arm_cc26xx_Timer_getMaxTicks__E      
000005ac  ti_sysbios_rom_ROM_ti_sysbios_family_arm_cc26xx_Timer_initDevice__I       
000005b0  ti_sysbios_rom_ROM_ti_sysbios_family_arm_cc26xx_Timer_setNextTick__E      
000005b4  ti_sysbios_rom_ROM_ti_sysbios_family_arm_cc26xx_Timer_setThreshold__I     
000005b8  ti_sysbios_rom_ROM_ti_sysbios_family_arm_cc26xx_Timer_start__E            
000005bc  ti_sysbios_rom_ROM_ti_sysbios_family_arm_cc26xx_TimestampProvider_get32__E
000005c0  ti_sysbios_rom_ROM_xdc_runtime_Startup_getState__I                        
000005c4  ti_sysbios_rom_ROM_xdc_runtime_System_SupportProxy_abort__E               
000005c8  ti_sysbios_rom_ROM_xdc_runtime_System_SupportProxy_exit__E                
00003227  ti_sysbios_rom_cortexm_cc26xx_CC26xx_badRomRevision__E                    
00005d8d  ti_sysbios_rom_cortexm_cc26xx_CC26xx_checkRevision__E                     
1001ca9b  ti_sysbios_rom_cortexm_cc26xx_CC26xx_getRevision__E                       
00002999  trimDevice                                                                
00006500  txPowerTable                                                              
00006590  txPwrTbl                                                                  
200025b0  user0Cfg                                                                  
000064d0  validRangeUUID                                                            
00000524  xdc_runtime_Assert_E_assertFailed__C                                      
1001c5a9  xdc_runtime_Assert_raise__I                                               
1001c6ed  xdc_runtime_Core_assignLabel__I                                           
1001c5f1  xdc_runtime_Core_assignParams__I                                          
1001c639  xdc_runtime_Core_constructObject__I                                       
1001c405  xdc_runtime_Core_createObject__I                                          
1001c4f9  xdc_runtime_Core_deleteObject__I                                          
1001c7a1  xdc_runtime_Core_destructObject__I                                        
00000528  xdc_runtime_Error_E_memory__C                                             
1001c7b9  xdc_runtime_Error_check__E                                                
1001c841  xdc_runtime_Error_init__E                                                 
0000052c  xdc_runtime_Error_policyFxn__C                                            
1001c487  xdc_runtime_Error_policySpin__E                                           
0000058c  xdc_runtime_Error_policy__C                                               
1001c769  xdc_runtime_Error_raiseX__E                                               
1001c885  xdc_runtime_Gate_enterSystem__E                                           
1001c879  xdc_runtime_Gate_leaveSystem__E                                           
00000530  xdc_runtime_IGateProvider_Interface__BASE__C                              
00000534  xdc_runtime_IHeap_Interface__BASE__C                                      
00000538  xdc_runtime_IModule_Interface__BASE__C                                    
UNDEFED   xdc_runtime_Main_Module_GateProxy_Handle__label__S                        
UNDEFED   xdc_runtime_Main_Module_GateProxy_Object__delete__S                       
UNDEFED   xdc_runtime_Main_Module_GateProxy_query__E                                
0000053c  xdc_runtime_Main_Module__diagsEnabled__C                                  
00000540  xdc_runtime_Main_Module__diagsIncluded__C                                 
00000544  xdc_runtime_Main_Module__diagsMask__C                                     
00000584  xdc_runtime_Main_Module__id__C                                            
1001bc89  xdc_runtime_Memory_HeapProxy_Handle__label__S                             
UNDEFED   xdc_runtime_Memory_HeapProxy_Handle__label__S__mangled__                  
1001bca9  xdc_runtime_Memory_HeapProxy_Object__delete__S                            
UNDEFED   xdc_runtime_Memory_HeapProxy_Object__delete__S__mangled__                 
1001c889  xdc_runtime_Memory_HeapProxy_alloc__E                                     
1001c88d  xdc_runtime_Memory_HeapProxy_free__E                                      
00000586  xdc_runtime_Memory_Module__id__C                                          
20000200  xdc_runtime_Memory_Module__state__V                                       
1001c489  xdc_runtime_Memory_alloc__E                                               
1001c84d  xdc_runtime_Memory_calloc__E                                              
00000548  xdc_runtime_Memory_defaultHeapInstance__C                                 
1001c801  xdc_runtime_Memory_free__E                                                
1001c859  xdc_runtime_Memory_getMaxDefaultTypeAlign__E                              
1001c785  xdc_runtime_Memory_valloc__E                                              
200001f0  xdc_runtime_Startup_Module__state__V                                      
00000001  xdc_runtime_Startup__EXECFXN__C                                           
00000001  xdc_runtime_Startup__RESETFXN__C                                          
0000054c  xdc_runtime_Startup_execImpl__C                                           
1001c559  xdc_runtime_Startup_exec__E                                               
00005edb  xdc_runtime_Startup_exec__I                                               
00006584  xdc_runtime_Startup_firstFxns__A                                          
00000514  xdc_runtime_Startup_firstFxns__C                                          
00003c69  xdc_runtime_Startup_getState__I                                           
0000051c  xdc_runtime_Startup_lastFxns__C                                           
00000550  xdc_runtime_Startup_maxPasses__C                                          
000060e1  xdc_runtime_Startup_reset__I                                              
00006564  xdc_runtime_Startup_sfxnRts__A                                            
00000554  xdc_runtime_Startup_sfxnRts__C                                            
000064d8  xdc_runtime_Startup_sfxnTab__A                                            
00000558  xdc_runtime_Startup_sfxnTab__C                                            
0000055c  xdc_runtime_Startup_startModsFxn__C                                       
1001c30d  xdc_runtime_Startup_startMods__I                                          
00000560  xdc_runtime_SysCallback_abortFxn__C                                       
1001c811  xdc_runtime_SysCallback_abort__E                                          
00003443  xdc_runtime_SysCallback_defaultAbort                                      
00003643  xdc_runtime_SysCallback_defaultExit                                       
00000564  xdc_runtime_SysCallback_exitFxn__C                                        
1001c821  xdc_runtime_SysCallback_exit__E                                           
1001bbe9  xdc_runtime_System_Module_GateProxy_Handle__label__S                      
UNDEFED   xdc_runtime_System_Module_GateProxy_Handle__label__S__mangled__           
1001bc09  xdc_runtime_System_Module_GateProxy_Object__delete__S                     
UNDEFED   xdc_runtime_System_Module_GateProxy_Object__delete__S__mangled__          
1001c891  xdc_runtime_System_Module_GateProxy_enter__E                              
1001c895  xdc_runtime_System_Module_GateProxy_leave__E                              
1001c269  xdc_runtime_System_Module_GateProxy_query__E                              
UNDEFED   xdc_runtime_System_Module_GateProxy_query__E__mangled__                   
200001f8  xdc_runtime_System_Module__state__V                                       
1001c87f  xdc_runtime_System_Module_startup__E                                      
UNDEFED   xdc_runtime_System_SupportProxy_abort__E                                  
UNDEFED   xdc_runtime_System_SupportProxy_exit__E                                   
00000568  xdc_runtime_System_abortFxn__C                                            
1001c899  xdc_runtime_System_abortSpin__E                                           
00004411  xdc_runtime_System_abortStd__E                                            
1001c749  xdc_runtime_System_abort__E                                               
1001c681  xdc_runtime_System_atexit__E                                              
0000056c  xdc_runtime_System_exitFxn__C                                             
1001c89b  xdc_runtime_System_exitSpin__E                                            
00004419  xdc_runtime_System_exitStd__E                                             
1001c7d1  xdc_runtime_System_exit__E                                                
00000570  xdc_runtime_System_maxAtexitHandlers__C                                   
1001c6b9  xdc_runtime_System_processAtExit__E                                       
00000588  xdc_runtime_Text_charCnt__C                                               
0000659b  xdc_runtime_Text_charTab__A                                               
00000574  xdc_runtime_Text_charTab__C                                               
1001c71d  xdc_runtime_Text_cordText__E                                              
0000058a  xdc_runtime_Text_isLoaded__C                                              
00000578  xdc_runtime_Text_nameEmpty__C                                             
0000057c  xdc_runtime_Text_nameStatic__C                                            
00000580  xdc_runtime_Text_nameUnknown__C                                           
1001c7e9  xdc_runtime_Text_ropeText__E                                              
1001c831  xdc_runtime_Timestamp_SupportProxy_get32__E                               
000058f5  xdc_runtime_Timestamp_SupportProxy_get32__E__mangled__                    
1001b9d1  xdc_runtime_Timestamp_SupportProxy_get64__E                               
UNDEFED   xdc_runtime_Timestamp_SupportProxy_get64__E__mangled__                    
1001c12f  xdc_runtime_Timestamp_SupportProxy_getFreq__E                             
UNDEFED   xdc_runtime_Timestamp_SupportProxy_getFreq__E__mangled__                  
1001c831  xdc_runtime_Timestamp_get32__E                                            
UNDEFED   xdc_runtime_Timestamp_get32__E__mangled__                                 
1001b9d1  xdc_runtime_Timestamp_get64__E                                            
UNDEFED   xdc_runtime_Timestamp_get64__E__mangled__                                 
1001c12f  xdc_runtime_Timestamp_getFreq__E                                          
UNDEFED   xdc_runtime_Timestamp_getFreq__E__mangled__                               


GLOBAL SYMBOLS: SORTED BY Symbol Address 

address   name                                                                      
-------   ----                                                                      
00000000  __ASM__                                                                   
00000000  ti_sysbios_family_arm_m3_Hwi_resetVectors                                 
00000001  xdc_runtime_Startup__EXECFXN__C                                           
00000001  xdc_runtime_Startup__RESETFXN__C                                          
00000068  __ISA__                                                                   
0000007a  __PLAT__                                                                  
000000a1  __TARG__                                                                  
000000c6  __TRDR__                                                                  
000000fd  GATTServApp_AddService                                                    
00000100  ti_sysbios_knl_Task_Object__PARAMS__C                                     
0000013c  ti_sysbios_knl_Mailbox_Object__PARAMS__C                                  
00000170  ti_sysbios_family_arm_m3_Hwi_Object__PARAMS__C                            
000001a0  ti_sysbios_hal_Hwi_Object__PARAMS__C                                      
000001cc  ti_sysbios_heaps_HeapMem_Module__FXNS__C                                  
000001f4  ti_sysbios_knl_Swi_Object__PARAMS__C                                      
0000021c  ti_sysbios_gates_GateHwi_Module__FXNS__C                                  
00000240  ti_sysbios_gates_GateMutex_Module__FXNS__C                                
00000264  ti_sysbios_heaps_HeapMem_Object__PARAMS__C                                
00000288  ti_sysbios_knl_Clock_Object__PARAMS__C                                    
000002ac  ti_sysbios_knl_Semaphore_Object__PARAMS__C                                
000002d0  ti_sysbios_family_arm_m3_Hwi_Object__DESC__C                              
000002f0  ti_sysbios_gates_GateHwi_Object__DESC__C                                  
00000310  ti_sysbios_gates_GateMutex_Object__DESC__C                                
00000330  ti_sysbios_hal_Hwi_Object__DESC__C                                        
00000350  ti_sysbios_heaps_HeapMem_Object__DESC__C                                  
00000370  ti_sysbios_knl_Clock_Object__DESC__C                                      
00000390  ti_sysbios_knl_Mailbox_Object__DESC__C                                    
000003b0  ti_sysbios_knl_Queue_Object__DESC__C                                      
000003d0  ti_sysbios_knl_Semaphore_Object__DESC__C                                  
000003f0  ti_sysbios_knl_Swi_Object__DESC__C                                        
00000400  __STACK_SIZE                                                              
00000410  ti_sysbios_knl_Task_Object__DESC__C                                       
00000430  ti_sysbios_gates_GateHwi_Object__PARAMS__C                                
00000448  ti_sysbios_gates_GateMutex_Object__PARAMS__C                              
00000460  ti_sysbios_knl_Queue_Object__PARAMS__C                                    
00000478  ti_sysbios_knl_Idle_funcList__C                                           
00000484  ti_sysbios_family_arm_cc26xx_Timer_startupNeeded__C                       
00000488  ti_sysbios_family_arm_m3_Hwi_E_alreadyDefined__C                          
0000048c  ti_sysbios_family_arm_m3_Hwi_E_hwiLimitExceeded__C                        
00000490  ti_sysbios_family_arm_m3_Hwi_NUM_INTERRUPTS__C                            
00000494  ti_sysbios_family_arm_m3_Hwi_Object__count__C                             
00000498  ti_sysbios_family_arm_m3_Hwi_Object__table__C                             
0000049c  ti_sysbios_family_arm_m3_Hwi_ccr__C                                       
000004a0  ti_sysbios_family_arm_m3_Hwi_excHandlerFunc__C                            
000004a4  ti_sysbios_family_arm_m3_Hwi_nullIsrFunc__C                               
000004a8  ti_sysbios_family_arm_m3_Hwi_numSparseInterrupts__C                       
000004ac  ti_sysbios_family_arm_m3_Hwi_priGroup__C                                  
000004b0  ti_sysbios_family_arm_m3_TaskSupport_stackAlignment__C                    
000004b4  ti_sysbios_heaps_HeapMem_E_memory__C                                      
000004b8  ti_sysbios_heaps_HeapMem_Module__gateObj__C                               
000004bc  ti_sysbios_heaps_HeapMem_Object__count__C                                 
000004c0  ti_sysbios_heaps_HeapMem_Object__table__C                                 
000004c4  ti_sysbios_heaps_HeapMem_reqAlign__C                                      
000004c8  ti_sysbios_knl_Clock_serviceMargin__C                                     
000004cc  ti_sysbios_knl_Mailbox_Object__count__C                                   
000004d0  ti_sysbios_knl_Mailbox_Object__table__C                                   
000004d4  ti_sysbios_knl_Queue_Object__count__C                                     
000004d8  ti_sysbios_knl_Queue_Object__table__C                                     
000004dc  ti_sysbios_knl_Swi_Object__count__C                                       
000004e0  ti_sysbios_knl_Swi_Object__table__C                                       
000004e4  ti_sysbios_knl_Swi_numPriorities__C                                       
000004e8  ti_sysbios_knl_Task_Object__count__C                                      
000004ec  ti_sysbios_knl_Task_Object__table__C                                      
000004f0  ti_sysbios_knl_Task_allBlockedFunc__C                                     
000004f4  ti_sysbios_knl_Task_defaultStackHeap__C                                   
000004f8  ti_sysbios_knl_Task_defaultStackSize__C                                   
000004fc  ti_sysbios_knl_Task_numConstructedTasks__C                                
00000501  ti_sysbios_BIOS_nullFunc__I                                               
00000502  ti_sysbios_family_arm_cc26xx_Timer_Module__id__C                          
00000504  ti_sysbios_family_arm_cc26xx_TimestampProvider_useClockTimer__C           
00000506  ti_sysbios_family_arm_m3_Hwi_Module__id__C                                
00000508  ti_sysbios_gates_GateHwi_Module__id__C                                    
0000050a  ti_sysbios_gates_GateMutex_Module__id__C                                  
0000050c  ti_sysbios_heaps_HeapMem_Module__id__C                                    
0000050e  ti_sysbios_knl_Task_initStackFlag__C                                      
00000510  ti_sysbios_knl_Clock_tickMode__C                                          
00000514  xdc_runtime_Startup_firstFxns__C                                          
0000051c  xdc_runtime_Startup_lastFxns__C                                           
00000524  xdc_runtime_Assert_E_assertFailed__C                                      
00000528  xdc_runtime_Error_E_memory__C                                             
0000052c  xdc_runtime_Error_policyFxn__C                                            
00000530  xdc_runtime_IGateProvider_Interface__BASE__C                              
00000534  xdc_runtime_IHeap_Interface__BASE__C                                      
00000538  xdc_runtime_IModule_Interface__BASE__C                                    
0000053c  xdc_runtime_Main_Module__diagsEnabled__C                                  
00000540  xdc_runtime_Main_Module__diagsIncluded__C                                 
00000544  xdc_runtime_Main_Module__diagsMask__C                                     
00000548  xdc_runtime_Memory_defaultHeapInstance__C                                 
0000054c  xdc_runtime_Startup_execImpl__C                                           
00000550  xdc_runtime_Startup_maxPasses__C                                          
00000554  xdc_runtime_Startup_sfxnRts__C                                            
00000558  xdc_runtime_Startup_sfxnTab__C                                            
0000055c  xdc_runtime_Startup_startModsFxn__C                                       
00000560  xdc_runtime_SysCallback_abortFxn__C                                       
00000564  xdc_runtime_SysCallback_exitFxn__C                                        
00000568  xdc_runtime_System_abortFxn__C                                            
0000056c  xdc_runtime_System_exitFxn__C                                             
00000570  xdc_runtime_System_maxAtexitHandlers__C                                   
00000574  xdc_runtime_Text_charTab__C                                               
00000578  xdc_runtime_Text_nameEmpty__C                                             
0000057c  xdc_runtime_Text_nameStatic__C                                            
00000580  xdc_runtime_Text_nameUnknown__C                                           
00000584  xdc_runtime_Main_Module__id__C                                            
00000586  xdc_runtime_Memory_Module__id__C                                          
00000588  xdc_runtime_Text_charCnt__C                                               
0000058a  xdc_runtime_Text_isLoaded__C                                              
0000058c  xdc_runtime_Error_policy__C                                               
00000590  ti_sysbios_rom_ROM_AONRTCChannelEnable                                    
00000594  ti_sysbios_rom_ROM_AONRTCCompareValueSet                                  
00000598  ti_sysbios_rom_ROM_AONRTCCurrentCompareValueGet                           
0000059c  ti_sysbios_rom_ROM_AONRTCEventClear                                       
000005a0  ti_sysbios_rom_ROM_ti_sysbios_family_arm_cc26xx_Timer_getCount64__E       
000005a4  ti_sysbios_rom_ROM_ti_sysbios_family_arm_cc26xx_Timer_getCurrentTick__E   
000005a8  ti_sysbios_rom_ROM_ti_sysbios_family_arm_cc26xx_Timer_getMaxTicks__E      
000005ac  ti_sysbios_rom_ROM_ti_sysbios_family_arm_cc26xx_Timer_initDevice__I       
000005b0  ti_sysbios_rom_ROM_ti_sysbios_family_arm_cc26xx_Timer_setNextTick__E      
000005b4  ti_sysbios_rom_ROM_ti_sysbios_family_arm_cc26xx_Timer_setThreshold__I     
000005b8  ti_sysbios_rom_ROM_ti_sysbios_family_arm_cc26xx_Timer_start__E            
000005bc  ti_sysbios_rom_ROM_ti_sysbios_family_arm_cc26xx_TimestampProvider_get32__E
000005c0  ti_sysbios_rom_ROM_xdc_runtime_Startup_getState__I                        
000005c4  ti_sysbios_rom_ROM_xdc_runtime_System_SupportProxy_abort__E               
000005c8  ti_sysbios_rom_ROM_xdc_runtime_System_SupportProxy_exit__E                
000005cc  ti_sysbios_gates_GateMutex_Instance_State_sem__O                          
000005d0  ti_sysbios_knl_Clock_Module_State_clockQ__O                               
000005d4  ti_sysbios_knl_Mailbox_Instance_State_dataQue__O                          
000005d8  ti_sysbios_knl_Mailbox_Instance_State_dataSem__O                          
000005dc  ti_sysbios_knl_Mailbox_Instance_State_freeQue__O                          
000005e0  ti_sysbios_knl_Mailbox_Instance_State_freeSem__O                          
000005e4  ti_sysbios_knl_Semaphore_Instance_State_pendQ__O                          
000005e8  ti_sysbios_knl_Task_Module_State_inactiveQ__O                             
00000963  ti_sysbios_family_arm_cc26xx_Power_defaultClockFunc__E                    
00000965  ti_sysbios_family_arm_cc26xx_Power_auxISR__E                              
00000cb1  ti_sysbios_family_arm_cc26xx_Power_sleep__E                               
0000145d  GAPRole_SetParameter                                                      
00001681  __aeabi_uldivmod                                                          
00001875  SysCtrlSetRechargeBeforePowerDown                                         
00001a3b  __aeabi_dsub                                                              
00001a45  __aeabi_dadd                                                              
00001bf1  PIN_init                                                                  
00001d79  GAPRole_GetParameter                                                      
000020a1  __aeabi_dmul                                                              
0000219d  ti_sysbios_family_arm_cc26xx_Power_startFirstMeasurement__E               
0000238b  ti_sysbios_family_arm_cc26xx_Power_defaultNotifyTrapFunc__E               
00002481  ti_sysbios_family_arm_cc26xx_Power_standbyPolicy__E                       
0000273d  ti_sysbios_family_arm_cc26xx_Power_setDependency__E                       
00002815  ti_sysbios_family_arm_cc26xx_Power_releaseDependency__E                   
00002999  ti_sysbios_family_arm_cc26xx_Boot_trimDevice                              
00002999  trimDevice                                                                
00002afd  ti_sysbios_knl_Clock_workFuncDynamic__E                                   
00002bad  ti_sysbios_family_arm_cc26xx_Power_initiateCalibration__E                 
00002c51  NOROM_AUXADCDisable                                                       
00002cf1  __TI_auto_init                                                            
00002e31  __aeabi_memcpy                                                            
00002e31  __aeabi_memcpy4                                                           
00002e31  __aeabi_memcpy8                                                           
00002e31  memcpy                                                                    
00002ecd  OSCHF_GetStartupTime                                                      
00002ecd  ti_sysbios_family_arm_cc26xx_Power_getXoscStartupTime__E                  
00002ff5  PIN_open                                                                  
00003085  ti_sysbios_family_arm_cc26xx_Power_LF_clockFunc__E                        
00003111  ti_sysbios_family_arm_cc26xx_Power_Module_startup__E                      
0000319d  NOROM_AUXADCEnableSync                                                    
00003227  ti_sysbios_rom_cortexm_cc26xx_CC26xx_badRomRevision__E                    
000032b1  ti_sysbios_family_arm_cc26xx_Timer_start__E                               
00003339  __aeabi_cdcmpeq                                                           
00003339  __aeabi_cdcmple                                                           
00003443  xdc_runtime_SysCallback_defaultAbort                                      
00003445  ICall_heapMalloc                                                          
0000354d  ICall_createRemoteTasks                                                   
000035c9  __aeabi_memclr                                                            
000035c9  __aeabi_memclr4                                                           
000035c9  __aeabi_memclr8                                                           
000035cb  __aeabi_memset                                                            
000035cb  __aeabi_memset4                                                           
000035cb  __aeabi_memset8                                                           
000035d1  memset                                                                    
00003643  xdc_runtime_SysCallback_defaultExit                                       
000036b9  adcIsr                                                                    
0000372d  ChipInfo_GetHwRevision                                                    
00003811  ICallPlatform_pwrUpdActivityCounter                                       
0000387d  SysCtrl_DCDC_VoltageConditionalControl                                    
00003a21  GATTServApp_ProcessCharCfg                                                
00003a85  OSCHF_AttemptToSwitchToXosc                                               
00003ae9  SysCtrlAdjustRechargeAfterPowerDown                                       
00003b4d  ti_sysbios_family_arm_cc26xx_Power_XOSC_HF_clockFunc__E                   
00003bad  ti_sysbios_family_arm_cc26xx_Timer_setNextTick__E                         
00003c0d  SimpleProfile_SetParameter                                                
00003c69  xdc_runtime_Startup_getState__I                                           
00003cc5  NOROM_DDI16BitfieldWrite                                                  
00003d79  ti_sysbios_family_arm_cc26xx_Power_notify__I                              
00003dd1  ICallPlatform_pwrRegisterNotify                                           
00003ecb  NOROM_OSCClockSourceSet                                                   
00003f1d  GAP_DeviceInit                                                            
00003f6d  GAP_UpdateAdvertisingData                                                 
0000405d  GAPRole_SendUpdateParam                                                   
00004141  copy_in                                                                   
0000418d  GATTServApp_ProcessCCCWriteReq                                            
00004221  Util_constructClock                                                       
000042f9  NOROM_DDI16BitfieldRead                                                   
00004341  GAP_TerminateLinkReq                                                      
00004385  SimpleProfile_GetParameter                                                
000043c9  ResetISR                                                                  
000043c9  _c_int00                                                                  
0000440d  C$$EXIT                                                                   
00004411  abort                                                                     
00004411  xdc_runtime_System_abortStd__E                                            
00004419  exit                                                                      
00004419  xdc_runtime_System_exitStd__E                                             
00004451  ti_sysbios_family_arm_cc26xx_Timer_initDevice__I                          
00004519  GAPRole_createTask                                                        
00004559  GATT_SendRsp                                                              
00004599  NOROM_OSCInterfaceEnable                                                  
000045d9  SimpleBLEPeripheral_createTask                                            
00004619  ti_sysbios_family_arm_cc26xx_Power_XOSC_HF                                
00004659  ti_sysbios_family_arm_cc26xx_Power_isStableXOSC_HF__E                     
00004699  ti_sysbios_family_arm_cc26xx_Timer_getCurrentTick__E                      
00004719  GAP_GetParamValue                                                         
00004755  GATTServApp_RegisterService                                               
00004791  ICallPlatform_pwrConfigACAction                                           
00004881  ti_sysbios_family_arm_cc26xx_Power_releaseConstraint__E                   
000048bd  GAPBondMgr_LinkEst                                                        
00004965  Util_restartClock                                                         
0000499d  linkDB_NumConns                                                           
000049d5  ti_sysbios_family_arm_cc26xx_Power_setConstraint__E                       
00004a0d  ti_sysbios_family_arm_cc26xx_Timer_setThreshold__I                        
00004ae7  SafeHapiAuxAdiSelect                                                      
00004b1d  ChipInfo_GetChipFamily                                                    
00004b51  GAPBondMgr_SetParameter                                                   
00004b85  GAP_SetParamValue                                                         
00004d25  osal_snv_read                                                             
00004d59  osal_snv_write                                                            
00004df5  OSCHF_SwitchToRcOscTurnOffXosc                                            
00004f51  ICall_heapInit                                                            
00004fb1  PIN_setOutputValue                                                        
00004fe1  ti_sysbios_BIOS_atExitFunc__I                                             
00005011  ti_sysbios_family_arm_cc26xx_Power_registerNotify__E                      
00005041  ti_sysbios_family_arm_cc26xx_Power_switchXOSC_HF__E                       
00005157  AONBatMonTemperatureGetDegC                                               
00005185  GAPBondMgr_Register                                                       
000051b1  HCI_EXT_ConnEventNoticeCmd                                                
000051dd  ICall_freeImpl                                                            
000051dd  ICall_heapFree                                                            
00005311  NOROM_AONRTCCurrentCompareValueGet                                        
0000533d  PIN_setConfig                                                             
00005393  Util_enqueueMsg                                                           
000053e7  GATTServApp_WriteCharCfg                                                  
00005439  ICall_init                                                                
00005501  SimpleProfile_AddService                                                  
00005551  ti_sysbios_family_arm_cc26xx_Power_isDependencyActive                     
00005579  ti_sysbios_family_arm_cc26xx_Timer_getMaxTicks__E                         
000055a1  NOROM_OSCClockSourceGet                                                   
000055c7  GAPBondMgr_LinkTerm                                                       
000055ed  GATTServApp_FindAttr                                                      
0000567d  ti_sysbios_BIOS_registerRTSLock__I                                        
000056a1  ti_sysbios_BIOS_removeRTSLock__I                                          
000056c5  ti_sysbios_BIOS_startFunc__I                                              
000056e9  ti_sysbios_family_arm_cc26xx_Timer_dynamicStub__E                         
00005775  GATTServApp_InitCharCfg                                                   
00005795  GATT_bm_alloc                                                             
00005895  Util_dequeueMsg                                                           
000058b5  __aeabi_ui2d                                                              
000058d5  ti_sysbios_BIOS_rtsLock__I                                                
000058f5  ti_sysbios_family_arm_cc26xx_TimestampProvider_get32__E                   
000058f5  xdc_runtime_Timestamp_SupportProxy_get32__E__mangled__                    
00005933  main                                                                      
0000598d  GAPRole_StartDevice                                                       
000059a9  GATT_bm_free                                                              
00005a51  ICall_enterCSImpl                                                         
00005a85  OSCHF_TurnOnXosc                                                          
00005ad3  ChipInfo_GetPackageType                                                   
00005aed  GAPRole_TerminateConnection                                               
00005b05  GATT_Notification                                                         
00005bad  ICallPlatform_pwrDispense                                                 
00005bc5  ICallPlatform_pwrRequire                                                  
00005ccd  Util_constructQueue                                                       
00005cfd  gapRole_clockHandler                                                      
00005d15  _args_main                                                                
00005d2d  __aeabi_lmul                                                              
00005d45  ti_sysbios_BIOS_rtsUnlock__I                                              
00005d5d  ti_sysbios_family_arm_cc26xx_Power_RFCORECLKS                             
00005d75  ti_sysbios_family_arm_cc26xx_Timer_getCount64__E                          
00005d8d  ti_sysbios_rom_cortexm_cc26xx_CC26xx_checkRevision__E                     
00005dd1  ICall_leaveCSImpl                                                         
00005e13  ti_sysbios_BIOS_exitFunc__I                                               
00005e29  DevInfo_AddService                                                        
00005e3d  ICallPlatform_pwrIsStableXOSCHF                                           
00005e51  SimpleProfile_RegisterAppCBs                                              
00005e65  ThisCodeIsBuiltForCC26xxHwRev22AndLater_HaltIfViolated                    
00005e79  _nop                                                                      
00005e7b  _register_unlock                                                          
00005e81  _register_lock                                                            
00005e8d  strlen                                                                    
00005eb5  ti_sysbios_knl_Clock_doTick__I                                            
00005ec9  NOROM_AUXADCReadFifo                                                      
00005edb  xdc_runtime_Startup_exec__I                                               
00005eed  DevInfo_SetParameter                                                      
00005efd  GAP_EndDiscoverable                                                       
00005f0d  GATTServApp_ReadCharCfg                                                   
00005f1d  ICallPlatform_pwrGetXOSCStartupTime                                       
00005f4d  Util_isActive                                                             
00005f5d  ICallPlatform_pwrGetTransitionState                                       
00005fa3  NOROM_VIMSModeGet                                                         
00005fcd  __TI_decompress_none                                                      
00006021  GAP_MakeDiscoverable                                                      
0000602d  GAP_TerminateAuth                                                         
00006039  GAP_UpdateLinkParamReq                                                    
00006045  GGS_SetParameter                                                          
0000608d  NOROM_CPUcpsid                                                            
00006099  NOROM_CPUcpsie                                                            
000060a5  __TI_zero_init                                                            
000060bd  ti_sysbios_BIOS_getThreadType__E                                          
000060c9  ti_sysbios_family_arm_cc26xx_Power_getTransitionState__E                  
000060d5  ti_sysbios_hal_Hwi_Params__init__S                                        
000060e1  xdc_runtime_Startup_reset__I                                              
000060ed  ICallPlatform_pwrSwitchXOSCHF                                             
00006101  GATT_Indication                                                           
00006121  GAP_RegisterForMsgs                                                       
00006127  GATT_RegisterForMsgs                                                      
0000612d  GGS_AddService                                                            
00006133  ICall_mallocImpl                                                          
00006139  PIN_registerIntCb                                                         
0000613f  __xdc__init                                                               
00006145  __TI_decompress_rle24                                                     
0000619f  Util_startClock                                                           
000061a3  Util_stopClock                                                            
000061ab  ti_sysbios_family_arm_cc26xx_Power_NOP                                    
000061af  ti_sysbios_knl_Clock_isActive__E                                          
00006418  ti_sysbios_family_arm_cc26xx_Power_db                                     
000064ac  primaryServiceUUID                                                        
000064ae  characterUUID                                                             
000064b0  gapServiceUUID                                                            
000064b2  gattServiceUUID                                                           
000064b4  secondaryServiceUUID                                                      
000064b6  includeUUID                                                               
000064b8  charExtPropsUUID                                                          
000064ba  charUserDescUUID                                                          
000064bc  clientCharCfgUUID                                                         
000064be  servCharCfgUUID                                                           
000064c0  charFormatUUID                                                            
000064c2  charAggFormatUUID                                                         
000064c4  deviceNameUUID                                                            
000064c6  appearanceUUID                                                            
000064c8  periPrivacyFlagUUID                                                       
000064ca  reconnectAddrUUID                                                         
000064cc  periConnParamUUID                                                         
000064ce  serviceChangedUUID                                                        
000064d0  validRangeUUID                                                            
000064d2  extReportRefUUID                                                          
000064d4  reportRefUUID                                                             
000064d8  xdc_runtime_Startup_sfxnTab__A                                            
00006500  txPowerTable                                                              
00006527  devInfoServUUID                                                           
00006529  devInfoSystemIdUUID                                                       
0000652b  devInfoModelNumberUUID                                                    
0000652d  devInfoSerialNumberUUID                                                   
0000652f  devInfoFirmwareRevUUID                                                    
00006531  devInfoHardwareRevUUID                                                    
00006533  devInfoSoftwareRevUUID                                                    
00006535  devInfoMfrNameUUID                                                        
00006537  devInfo11073CertUUID                                                      
00006539  devInfoPnpIdUUID                                                          
00006544  devInfoCBs                                                                
00006558  simpleProfileCBs                                                          
00006564  xdc_runtime_Startup_sfxnRts__A                                            
00006578  simpleProfileServUUID                                                     
0000657a  simpleProfilechar1UUID                                                    
0000657c  simpleProfilechar2UUID                                                    
0000657e  simpleProfilechar3UUID                                                    
00006580  simpleProfilechar4UUID                                                    
00006582  simpleProfilechar5UUID                                                    
00006584  xdc_runtime_Startup_firstFxns__A                                          
00006590  txPwrTbl                                                                  
0000659b  xdc_runtime_Text_charTab__A                                               
0000659c  ti_sysbios_family_arm_cc26xx_Power_Module_State_clockObj__O               
000065a0  ti_sysbios_family_arm_cc26xx_Power_Module_State_lfClockObj__O             
000065a4  ti_sysbios_family_arm_cc26xx_Power_Module_State_notifyQ__O                
000065a8  ti_sysbios_family_arm_cc26xx_Power_notifyTrapFunc__C                      
000065ac  ti_sysbios_family_arm_cc26xx_Power_totalTicksSTANDBY__C                   
000065b0  ti_sysbios_family_arm_cc26xx_Power_wakeDelaySTANDBY__C                    
000065b4  ti_sysbios_family_arm_m3_Hwi_disablePriority__C                           
000065b8  ti_sysbios_knl_Clock_tickPeriod__C                                        
000065bc  ti_sysbios_knl_Idle_funcList__A                                           
000065c0  __TI_static_base__                                                        
00006cd8  __TI_Handler_Table_Base                                                   
00006ce4  __TI_Handler_Table_Limit                                                  
00006d38  __TI_CINIT_Base                                                           
00006da0  __TI_CINIT_Limit                                                          
0001ffa8  __ccfg                                                                    
1001a001  ti_sysbios_knl_Mailbox_Instance_init__E                                   
1001a0cd  ti_sysbios_knl_Semaphore_pend__E                                          
1001a199  ti_sysbios_heaps_HeapMem_alloc__E                                         
1001a25d  ti_sysbios_knl_Task_Instance_init__E                                      
1001a319  ti_sysbios_family_arm_m3_Hwi_postInit__I                                  
1001a3c9  ti_sysbios_family_arm_m3_Hwi_Instance_init__E                             
1001a469  ti_sysbios_family_arm_cc26xx_Timer_periodicStub__E                        
1001a4fd  ti_sysbios_knl_Task_Instance_finalize__E                                  
1001a591  ti_sysbios_knl_Mailbox_post__E                                            
1001a615  ti_sysbios_knl_Task_postInit__I                                           
1001a699  ti_sysbios_family_arm_m3_Hwi_initNVIC__E                                  
1001a719  ti_sysbios_knl_Clock_startI__E                                            
1001a795  ti_sysbios_heaps_HeapMem_free__E                                          
1001a80d  ti_sysbios_knl_Clock_walkQueueDynamic__E                                  
1001a885  ti_sysbios_knl_Clock_workFunc__E                                          
1001a8fd  ti_sysbios_knl_Mailbox_pend__E                                            
1001a96d  ti_sysbios_knl_Task_sleep__E                                              
1001a9dd  ti_sysbios_knl_Mailbox_Instance_finalize__E                               
1001aa49  ti_sysbios_family_arm_m3_Hwi_dispatchC__I                                 
1001aab1  ti_sysbios_family_arm_m3_Hwi_Object__create__S                            
1001ab15  ti_sysbios_family_arm_m3_Hwi_create                                       
1001ab79  ti_sysbios_hal_Hwi_create                                                 
1001abdd  ti_sysbios_knl_Mailbox_create                                             
1001ac41  ti_sysbios_knl_Semaphore_post__E                                          
1001aca5  ti_sysbios_knl_Swi_Instance_init__E                                       
1001ad05  ti_sysbios_knl_Swi_create                                                 
1001ad61  ti_sysbios_knl_Swi_restoreHwi__E                                          
1001adbd  ti_sysbios_knl_Task_Module_startup__E                                     
1001ae19  ti_sysbios_knl_Task_create                                                
1001ae75  ti_sysbios_knl_Task_startCore__E                                          
1001aed1  ti_sysbios_family_arm_m3_Hwi_Instance_finalize__E                         
1001af29  ti_sysbios_family_arm_m3_Hwi_construct                                    
1001af81  ti_sysbios_knl_Mailbox_construct                                          
1001afd9  ti_sysbios_knl_Swi_run__I                                                 
1001b031  ti_sysbios_knl_Swi_schedule__I                                            
1001b085  ti_sysbios_knl_Swi_construct                                              
1001b0d5  ti_sysbios_knl_Swi_runLoop__I                                             
1001b125  ti_sysbios_knl_Task_construct                                             
1001b175  ti_sysbios_knl_Task_schedule__I                                           
1001b1c1  ti_sysbios_family_arm_m3_Hwi_Module_startup__E                            
1001b209  ti_sysbios_heaps_HeapMem_getStats__E                                      
1001b251  ti_sysbios_knl_Mailbox_Module_startup__E                                  
1001b299  ti_sysbios_family_arm_m3_Hwi_disableInterrupt__E                          
1001b2dd  ti_sysbios_family_arm_m3_Hwi_enableInterrupt__E                           
1001b321  ti_sysbios_knl_Swi_post__E                                                
1001b365  ti_sysbios_knl_Task_allBlockedFunction__I                                 
1001b3a9  ti_sysbios_knl_Task_yield__E                                              
1001b3ed  ti_sysbios_knl_Clock_create                                               
1001b429  ti_sysbios_knl_Task_exit__E                                               
1001b463  ti_sysbios_gates_GateHwi_Instance_init__E                                 
1001b465  ti_sysbios_family_arm_m3_Hwi_getStackInfo__E                              
1001b49d  ti_sysbios_family_arm_m3_TaskSupport_start__E                             
1001b4d5  ti_sysbios_heaps_HeapMem_Instance_init__E                                 
1001b50d  ti_sysbios_knl_Clock_Instance_init__E                                     
1001b545  ti_sysbios_heaps_HeapMem_init__I                                          
1001b579  ti_sysbios_knl_Clock_construct                                            
1001b5ad  ti_sysbios_knl_Semaphore_create                                           
1001b5e1  ti_sysbios_knl_Swi_restore__E                                             
1001b615  ti_sysbios_knl_Task_blockI__E                                             
1001b649  ti_sysbios_gates_GateMutex_Object__create__S                              
1001b679  ti_sysbios_gates_GateMutex_create                                         
1001b6a9  ti_sysbios_gates_GateMutex_enter__E                                       
1001b6d9  ti_sysbios_knl_Clock_getTicks__E                                          
1001b709  ti_sysbios_knl_Semaphore_construct                                        
1001b739  ti_sysbios_knl_Task_processVitalTaskFlag__I                               
1001b769  ti_sysbios_family_arm_cc26xx_Timer_postInit__I                            
1001b795  ti_sysbios_family_arm_cc26xx_Timer_startup__E                             
1001b795  ti_sysbios_knl_Clock_TimerProxy_startup__E                                
1001b7c1  ti_sysbios_family_arm_m3_Hwi_Object__get__S                               
1001b7ed  ti_sysbios_gates_GateMutex_construct                                      
1001b819  ti_sysbios_hal_Hwi_initStack                                              
1001b845  ti_sysbios_heaps_HeapMem_Object__create__S                                
1001b871  ti_sysbios_heaps_HeapMem_Object__get__S                                   
1001b89d  ti_sysbios_knl_Mailbox_Object__get__S                                     
1001b8c9  ti_sysbios_knl_Mailbox_postInit__I                                        
1001b8f5  ti_sysbios_knl_Queue_construct                                            
1001b921  ti_sysbios_knl_Queue_create                                               
1001b94d  ti_sysbios_knl_Semaphore_pendTimeout__I                                   
1001b979  ti_sysbios_knl_Swi_Object__get__S                                         
1001b9a5  ti_sysbios_knl_Task_unblockI__E                                           
1001b9d1  ti_sysbios_family_arm_cc26xx_TimestampProvider_get64__E                   
1001b9d1  xdc_runtime_Timestamp_SupportProxy_get64__E                               
1001b9d1  xdc_runtime_Timestamp_get64__E                                            
1001b9f9  ti_sysbios_hal_Hwi_Instance_init__E                                       
1001ba21  ti_sysbios_knl_Clock_addI__E                                              
1001ba49  ti_sysbios_knl_Task_restore__E                                            
1001ba71  ti_sysbios_family_arm_cc26xx_Timer_Module_startup__E                      
1001ba95  ti_sysbios_gates_GateHwi_Object__create__S                                
1001bab9  ti_sysbios_BIOS_RtsGateProxy_Object__delete__S                            
1001bab9  ti_sysbios_gates_GateMutex_Object__delete__S                              
1001bab9  ti_sysbios_heaps_HeapMem_Module_GateProxy_Object__delete__S               
1001badd  ti_sysbios_knl_Clock_Object__delete__S                                    
1001bb01  ti_sysbios_knl_Semaphore_Instance_init__E                                 
1001bb25  ti_sysbios_knl_Semaphore_Object__delete__S                                
1001bb49  ti_sysbios_family_arm_cc26xx_Timer_Module__startupDone__S                 
1001bb69  ti_sysbios_family_arm_cc26xx_TimestampProvider_Module_startup__E          
1001bb89  ti_sysbios_family_arm_m3_Hwi_Module__startupDone__S                       
1001bba9  ti_sysbios_family_arm_m3_Hwi_Object__delete__S                            
1001bba9  ti_sysbios_hal_Hwi_HwiProxy_Object__delete__S                             
1001bbc9  ti_sysbios_family_arm_m3_Hwi_excHandler__I                                
1001bbe9  ti_sysbios_gates_GateHwi_Handle__label__S                                 
1001bbe9  xdc_runtime_System_Module_GateProxy_Handle__label__S                      
1001bc09  ti_sysbios_gates_GateHwi_Object__delete__S                                
1001bc09  xdc_runtime_System_Module_GateProxy_Object__delete__S                     
1001bc29  ti_sysbios_BIOS_RtsGateProxy_Handle__label__S                             
1001bc29  ti_sysbios_gates_GateMutex_Handle__label__S                               
1001bc29  ti_sysbios_heaps_HeapMem_Module_GateProxy_Handle__label__S                
1001bc49  ti_sysbios_gates_GateMutex_Object__destruct__S                            
1001bc69  ti_sysbios_hal_Hwi_Object__delete__S                                      
1001bc89  ti_sysbios_heaps_HeapMem_Handle__label__S                                 
1001bc89  xdc_runtime_Memory_HeapProxy_Handle__label__S                             
1001bca9  ti_sysbios_heaps_HeapMem_Object__delete__S                                
1001bca9  xdc_runtime_Memory_HeapProxy_Object__delete__S                            
1001bcc9  ti_sysbios_knl_Clock_Module_startup__E                                    
1001bce9  ti_sysbios_knl_Clock_Object__destruct__S                                  
1001bd09  ti_sysbios_knl_Idle_run__E                                                
1001bd29  ti_sysbios_knl_Mailbox_Object__delete__S                                  
1001bd49  ti_sysbios_knl_Queue_Object__delete__S                                    
1001bd69  ti_sysbios_knl_Queue_Object__get__S                                       
1001bd89  ti_sysbios_knl_Semaphore_Object__destruct__S                              
1001bda9  ti_sysbios_knl_Swi_Object__delete__S                                      
1001bdc9  ti_sysbios_knl_Task_Object__delete__S                                     
1001bde9  ti_sysbios_knl_Task_Object__get__S                                        
1001be09  ti_sysbios_knl_Task_enter__I                                              
1001be29  ti_sysbios_knl_Task_restoreHwi__E                                         
1001be49  ti_sysbios_hal_Hwi_HwiProxy_create                                        
1001be67  ti_sysbios_knl_Clock_logTick__E                                           
1001be69  ti_sysbios_family_arm_m3_Hwi_Object__destruct__S                          
1001be85  ti_sysbios_family_arm_m3_Hwi_setPriority__E                               
1001bea1  ti_sysbios_gates_GateMutex_Instance_init__E                               
1001bebd  ti_sysbios_knl_Clock_scheduleNextTick__E                                  
1001bed9  ti_sysbios_knl_Mailbox_Object__destruct__S                                
1001bef5  ti_sysbios_knl_Queue_Object__destruct__S                                  
1001bf11  ti_sysbios_knl_Queue_get__E                                               
1001bf2d  ti_sysbios_knl_Queue_put__E                                               
1001bf49  ti_sysbios_knl_Swi_Object__destruct__S                                    
1001bf65  ti_sysbios_knl_Task_Object__destruct__S                                   
1001bf81  ti_sysbios_knl_Task_sleepTimeout__I                                       
1001bf9b  ti_sysbios_knl_Swi_Instance_finalize__E                                   
1001bf9d  ti_sysbios_gates_GateMutex_leave__E                                       
1001bfb5  ti_sysbios_knl_Task_unblock__E                                            
1001bfcd  ti_sysbios_knl_Clock_Instance_finalize__E                                 
1001bfe3  ti_sysbios_knl_Clock_start__E                                             
1001bff9  ti_sysbios_BIOS_getCpuFreq__E                                             
1001c00d  ti_sysbios_family_arm_m3_Hwi_switchFromBootStack__E                       
1001c021  ti_sysbios_hal_Hwi_Module_startup__E                                      
1001c035  ti_sysbios_BIOS_exit__E                                                   
1001c045  ti_sysbios_BIOS_setThreadType__E                                          
1001c055  ti_sysbios_BIOS_start__E                                                  
1001c065  ti_sysbios_family_arm_m3_Hwi_plug__E                                      
1001c075  ti_sysbios_gates_GateMutex_Instance_finalize__E                           
1001c085  ti_sysbios_hal_Hwi_HwiProxy_Object__create__S                             
1001c095  ti_sysbios_knl_Clock_TimerProxy_getCurrentTick__E                         
1001c0a5  ti_sysbios_knl_Clock_TimerProxy_getMaxTicks__E                            
1001c0b5  ti_sysbios_knl_Clock_TimerProxy_setNextTick__E                            
1001c0c5  ti_sysbios_knl_Semaphore_Instance_finalize__E                             
1001c0d5  ti_sysbios_knl_Swi_disable__E                                             
1001c0e5  ti_sysbios_knl_Swi_enabled__E                                             
1001c0f5  ti_sysbios_knl_Task_disable__E                                            
1001c105  ti_sysbios_heaps_HeapMem_restore__E                                       
1001c113  ti_sysbios_knl_Queue_empty__E                                             
1001c121  ti_sysbios_knl_Queue_remove__E                                            
1001c12f  ti_sysbios_family_arm_cc26xx_TimestampProvider_getFreq__E                 
1001c12f  xdc_runtime_Timestamp_SupportProxy_getFreq__E                             
1001c12f  xdc_runtime_Timestamp_getFreq__E                                          
1001c13d  ti_sysbios_family_arm_m3_Hwi_Params__init__S                              
1001c13d  ti_sysbios_hal_Hwi_HwiProxy_Params__init__S                               
1001c149  ti_sysbios_family_arm_m3_Hwi_disableFxn__E                                
1001c155  ti_sysbios_family_arm_m3_Hwi_enableFxn__E                                 
1001c161  ti_sysbios_family_arm_m3_TaskSupport_getStackAlignment__E                 
1001c16d  ti_sysbios_gates_GateHwi_enter__E                                         
1001c179  ti_sysbios_BIOS_RtsGateProxy_Params__init__S                              
1001c179  ti_sysbios_gates_GateMutex_Params__init__S                                
1001c179  ti_sysbios_heaps_HeapMem_Module_GateProxy_Params__init__S                 
1001c185  ti_sysbios_knl_Clock_Params__init__S                                      
1001c191  ti_sysbios_knl_Clock_getTimerHandle__E                                    
1001c19d  ti_sysbios_knl_Mailbox_Params__init__S                                    
1001c1a9  ti_sysbios_knl_Queue_dequeue__E                                           
1001c1b5  ti_sysbios_knl_Queue_enqueue__E                                           
1001c1c1  ti_sysbios_knl_Semaphore_Params__init__S                                  
1001c1cd  ti_sysbios_knl_Swi_Params__init__S                                        
1001c1d9  ti_sysbios_knl_Task_Params__init__S                                       
1001c1e5  ti_sysbios_knl_Task_self__E                                               
1001c1f1  ti_sysbios_hal_Hwi_Instance_finalize__E                                   
1001c1fb  ti_sysbios_family_arm_m3_Hwi_doSwiRestore__I                              
1001c203  ti_sysbios_family_arm_m3_Hwi_startup__E                                   
1001c20b  ti_sysbios_knl_Idle_loop__E                                               
1001c213  ti_sysbios_family_arm_m3_Hwi_doTaskRestore__I                             
1001c219  ti_sysbios_family_arm_m3_Hwi_restoreFxn__E                                
1001c21f  ti_sysbios_gates_GateHwi_leave__E                                         
1001c225  ti_sysbios_knl_Clock_stop__E                                              
1001c22b  ti_sysbios_knl_Queue_Instance_init__E                                     
1001c231  ti_sysbios_knl_Queue_elemClear__E                                         
1001c237  ti_sysbios_knl_Swi_Module_startup__E                                      
1001c23d  ti_sysbios_knl_Swi_startup__E                                             
1001c243  ti_sysbios_knl_Task_enable__E                                             
1001c249  ti_sysbios_BIOS_RtsGateProxy_enter__E                                     
1001c24d  ti_sysbios_BIOS_RtsGateProxy_leave__E                                     
1001c251  ti_sysbios_family_arm_cc26xx_Timer_getExpiredTicks__E                     
1001c255  ti_sysbios_family_arm_cc26xx_Timer_getPeriod__E                           
1001c259  ti_sysbios_family_arm_cc26xx_Timer_setPeriod__E                           
1001c25d  ti_sysbios_family_arm_m3_Hwi_delete                                       
1001c261  ti_sysbios_family_arm_m3_Hwi_destruct                                     
1001c265  ti_sysbios_family_arm_m3_TaskSupport_Module__startupDone__S               
1001c269  ti_sysbios_gates_GateHwi_query__E                                         
1001c269  xdc_runtime_System_Module_GateProxy_query__E                              
1001c26d  ti_sysbios_gates_GateMutex_delete                                         
1001c271  ti_sysbios_gates_GateMutex_destruct                                       
1001c275  ti_sysbios_BIOS_RtsGateProxy_query__E                                     
1001c275  ti_sysbios_gates_GateMutex_query__E                                       
1001c275  ti_sysbios_heaps_HeapMem_Module_GateProxy_query__E                        
1001c279  ti_sysbios_hal_Hwi_HwiProxy_Module__startupDone__S                        
1001c27d  ti_sysbios_hal_Hwi_HwiProxy_delete                                        
1001c281  ti_sysbios_hal_Hwi_HwiProxy_disableInterrupt__E                           
1001c281  ti_sysbios_hal_Hwi_disableInterrupt__E                                    
1001c285  ti_sysbios_hal_Hwi_HwiProxy_enableInterrupt__E                            
1001c285  ti_sysbios_hal_Hwi_enableInterrupt__E                                     
1001c289  ti_sysbios_hal_Hwi_HwiProxy_getStackInfo__E                               
1001c289  ti_sysbios_hal_Hwi_getStackInfo__E                                        
1001c28d  ti_sysbios_hal_Hwi_HwiProxy_startup__E                                    
1001c28d  ti_sysbios_hal_Hwi_startup__E                                             
1001c291  ti_sysbios_hal_Hwi_HwiProxy_switchFromBootStack__E                        
1001c295  ti_sysbios_hal_Hwi_delete                                                 
1001c299  ti_sysbios_hal_Hwi_switchFromBootStack__E                                 
1001c29d  ti_sysbios_heaps_HeapMem_Module_GateProxy_enter__E                        
1001c2a1  ti_sysbios_heaps_HeapMem_Module_GateProxy_leave__E                        
1001c2a5  ti_sysbios_heaps_HeapMem_isBlocking__E                                    
1001c2a9  ti_sysbios_knl_Clock_TimerProxy_Module__startupDone__S                    
1001c2ad  ti_sysbios_knl_Clock_TimerProxy_getExpiredTicks__E                        
1001c2b1  ti_sysbios_knl_Clock_TimerProxy_getPeriod__E                              
1001c2b5  ti_sysbios_knl_Clock_delete                                               
1001c2b9  ti_sysbios_knl_Clock_destruct                                             
1001c2bd  ti_sysbios_knl_Clock_removeI__E                                           
1001c2c1  ti_sysbios_knl_Clock_setTimeout__E                                        
1001c2c5  ti_sysbios_knl_Mailbox_delete                                             
1001c2c9  ti_sysbios_knl_Mailbox_destruct                                           
1001c2cd  ti_sysbios_knl_Queue_delete                                               
1001c2d1  ti_sysbios_knl_Queue_destruct                                             
1001c2d5  ti_sysbios_knl_Queue_head__E                                              
1001c2d9  ti_sysbios_knl_Queue_next__E                                              
1001c2dd  ti_sysbios_knl_Semaphore_delete                                           
1001c2e1  ti_sysbios_knl_Semaphore_destruct                                         
1001c2e5  ti_sysbios_knl_Swi_delete                                                 
1001c2e9  ti_sysbios_knl_Swi_destruct                                               
1001c2ed  ti_sysbios_knl_Swi_postInit__I                                            
1001c2f1  ti_sysbios_knl_Task_SupportProxy_Module__startupDone__S                   
1001c2f5  ti_sysbios_knl_Task_SupportProxy_getStackAlignment__E                     
1001c2f9  ti_sysbios_knl_Task_SupportProxy_start__E                                 
1001c2fd  ti_sysbios_knl_Task_SupportProxy_swap__E                                  
1001c301  ti_sysbios_knl_Task_delete                                                
1001c305  ti_sysbios_knl_Task_destruct                                              
1001c309  ti_sysbios_knl_Task_startup__E                                            
1001c30d  xdc_runtime_Startup_startMods__I                                          
1001c405  xdc_runtime_Core_createObject__I                                          
1001c487  xdc_runtime_Error_policySpin__E                                           
1001c489  xdc_runtime_Memory_alloc__E                                               
1001c4f9  xdc_runtime_Core_deleteObject__I                                          
1001c559  xdc_runtime_Startup_exec__E                                               
1001c5a9  xdc_runtime_Assert_raise__I                                               
1001c5f1  xdc_runtime_Core_assignParams__I                                          
1001c639  xdc_runtime_Core_constructObject__I                                       
1001c681  xdc_runtime_System_atexit__E                                              
1001c6b9  xdc_runtime_System_processAtExit__E                                       
1001c6ed  xdc_runtime_Core_assignLabel__I                                           
1001c71d  xdc_runtime_Text_cordText__E                                              
1001c749  xdc_runtime_System_abort__E                                               
1001c769  xdc_runtime_Error_raiseX__E                                               
1001c785  xdc_runtime_Memory_valloc__E                                              
1001c7a1  xdc_runtime_Core_destructObject__I                                        
1001c7b9  xdc_runtime_Error_check__E                                                
1001c7d1  xdc_runtime_System_exit__E                                                
1001c7e9  xdc_runtime_Text_ropeText__E                                              
1001c801  xdc_runtime_Memory_free__E                                                
1001c811  xdc_runtime_SysCallback_abort__E                                          
1001c821  xdc_runtime_SysCallback_exit__E                                           
1001c831  xdc_runtime_Timestamp_SupportProxy_get32__E                               
1001c831  xdc_runtime_Timestamp_get32__E                                            
1001c841  xdc_runtime_Error_init__E                                                 
1001c84d  xdc_runtime_Memory_calloc__E                                              
1001c859  xdc_runtime_Memory_getMaxDefaultTypeAlign__E                              
1001c879  xdc_runtime_Gate_leaveSystem__E                                           
1001c87f  xdc_runtime_System_Module_startup__E                                      
1001c885  xdc_runtime_Gate_enterSystem__E                                           
1001c889  xdc_runtime_Memory_HeapProxy_alloc__E                                     
1001c88d  xdc_runtime_Memory_HeapProxy_free__E                                      
1001c891  xdc_runtime_System_Module_GateProxy_enter__E                              
1001c895  xdc_runtime_System_Module_GateProxy_leave__E                              
1001c899  xdc_runtime_System_abortSpin__E                                           
1001c89b  xdc_runtime_System_exitSpin__E                                            
1001c89d  ti_sysbios_family_arm_m3_Hwi_dispatch__I                                  
1001c96d  ti_sysbios_family_arm_m3_TaskSupport_buildTaskStack                       
1001c9b9  ti_sysbios_family_arm_m3_Hwi_initStacks__E                                
1001ca01  ti_sysbios_family_arm_m3_Hwi_excHandlerAsm__I                             
1001ca21  ti_sysbios_family_xxx_Hwi_switchAndRunFunc                                
1001ca3f  ti_sysbios_family_arm_m3_Hwi_pendSV__I                                    
1001ca57  ti_sysbios_family_arm_m3_Hwi_return                                       
1001ca59  ti_sysbios_family_arm_m3_TaskSupport_glue                                 
1001ca69  ti_sysbios_family_arm_m3_TaskSupport_swap__E                              
1001ca71  ti_sysbios_knl_Task_swapReturn                                            
1001ca9b  ti_sysbios_rom_cortexm_cc26xx_CC26xx_getRevision__E                       
20000000  ti_sysbios_family_arm_m3_Hwi_ramVectors                                   
20000100  ti_sysbios_knl_Task_Module__state__V                                      
20000144  ti_sysbios_family_arm_m3_Hwi_Module__state__V                             
20000178  ti_sysbios_knl_Clock_Module__state__V                                     
200001a4  ti_sysbios_BIOS_Module__state__V                                          
200001c8  ti_sysbios_knl_Swi_Module__state__V                                       
200001e4  ti_sysbios_family_arm_cc26xx_Timer_Module__state__V                       
200001ec  ti_sysbios_family_arm_cc26xx_TimestampProvider_Module__state__V           
200001f0  xdc_runtime_Startup_Module__state__V                                      
200001f8  xdc_runtime_System_Module__state__V                                       
20000200  xdc_runtime_Memory_Module__state__V                                       
20000c78  ti_sysbios_heaps_HeapMem_Instance_State_0_buf__A                          
200012f8  ti_sysbios_knl_Task_Instance_State_0_stack__A                             
200014f8  PIN_NumPins                                                               
20001558  PIN_HandleTable                                                           
200015d4  ti_sysbios_family_arm_m3_Hwi_dispatchTable                                
200016b8  driverlib_release_0_43243                                                 
200016c0  temp_volt                                                                 
200016c8  i                                                                         
200016d0  led_blink_time                                                            
200016da  singleTempSample                                                          
200016dc  singleMtrSample                                                           
200016e8  LED_value                                                                 
200016ec  htempsem                                                                  
200016f0  hmtrsem                                                                   
200016f4  j                                                                         
20001718  sample_avg                                                                
20001720  sample_sum                                                                
20001728  adcFlag                                                                   
20001750  adcSamples                                                                
20001778  tempsem                                                                   
20001794  mtrsem                                                                    
200017b0  adc_hwi                                                                   
20001834  sbpTask                                                                   
20001884  sbpTaskStack                                                              
20001b40  linkDBNumConns                                                            
20001c54  gapRoleTask                                                               
20001ca4  gapRoleTaskStack                                                          
2000220c  ti_sysbios_family_arm_cc26xx_Power_refCount                               
2000221f  ti_sysbios_family_arm_cc26xx_Power_constraintCounts                       
20002224  ti_sysbios_family_arm_cc26xx_Power_resourceHandlers                       
20002230  ti_sysbios_family_arm_cc26xx_Timer_Module__root__V                        
20002238  ti_sysbios_family_arm_m3_Hwi_Module__root__V                              
20002240  ti_sysbios_family_arm_m3_Hwi_Module_State_0_excActive__A                  
20002244  ti_sysbios_family_arm_m3_Hwi_Module_State_0_excContext__A                 
20002248  ti_sysbios_family_arm_m3_Hwi_Module_State_0_excStack__A                   
2000224c  ti_sysbios_gates_GateHwi_Module__root__V                                  
20002254  ti_sysbios_gates_GateHwi_Object__table__V                                 
20002258  ti_sysbios_gates_GateMutex_Module__root__V                                
20002260  ti_sysbios_hal_Hwi_Module__root__V                                        
20002268  ti_sysbios_heaps_HeapMem_Module__root__V                                  
20002270  ti_sysbios_heaps_HeapMem_Object__table__V                                 
20002288  ti_sysbios_knl_Clock_Module__root__V                                      
20002290  ti_sysbios_knl_Event_Module__root__V                                      
20002298  ti_sysbios_knl_Mailbox_Module__root__V                                    
200022a0  ti_sysbios_knl_Queue_Module__root__V                                      
200022a8  ti_sysbios_knl_Semaphore_Module__root__V                                  
200022b0  ti_sysbios_knl_Swi_Module__root__V                                        
200022b8  ti_sysbios_knl_Task_Module__root__V                                       
200022c0  ti_sysbios_knl_Task_Module_State_0_idleTask__A                            
200022c4  __xdc__init__addr                                                         
200022c8  ICall_dispatcher                                                          
200022d0  ICall_enterCriticalSection                                                
200022d4  ICall_leaveCriticalSection                                                
20002354  ti_sysbios_family_arm_cc26xx_Power_Module__state__V                       
200023c4  TSK_idle                                                                  
200023c4  ti_sysbios_knl_Task_Object__table__V                                      
20002410  ti_sysbios_family_arm_cc26xx_Timer_Object__table__V                       
20002458  ti_sysbios_gates_GateMutex_Object__table__V                               
20002490  rfRegTbl                                                                  
200024c4  ti_sysbios_family_arm_m3_Hwi_Object__table__V                             
200024f4  ti_sysbios_knl_Swi_Module_State_0_readyQ__A                               
20002524  ti_sysbios_knl_Swi_Object__table__V                                       
20002554  ti_sysbios_knl_Task_Module_State_0_readyQ__A                              
20002584  BoardGpioInitTable                                                        
200025b0  user0Cfg                                                                  
200025e8  lastAppOpcodeSent                                                         
200025ec  pfnBMAlloc                                                                
200025f0  pfnBMFree                                                                 
200025fc  _lock                                                                     
20002600  _unlock                                                                   
20002604  __TI_cleanup_ptr                                                          
20002608  __TI_dtors_ptr                                                            
2000260c  main_func_sp                                                              
20003fe4  __stack                                                                   
200043e4  __STACK_END                                                               
200043e4  __STACK_TOP                                                               
e000e000  ti_sysbios_family_arm_m3_Hwi_nvic                                         
ffffffff  __binit__                                                                 
ffffffff  __c_args__                                                                
ffffffff  binit                                                                     
UNDEFED   SHT$$INIT_ARRAY$$Base                                                     
UNDEFED   SHT$$INIT_ARRAY$$Limit                                                    
UNDEFED   ti_sysbios_BIOS_RtsGateProxy_Handle__label__S__mangled__                  
UNDEFED   ti_sysbios_BIOS_RtsGateProxy_Object__delete__S__mangled__                 
UNDEFED   ti_sysbios_BIOS_RtsGateProxy_Params__init__S__mangled__                   
UNDEFED   ti_sysbios_BIOS_RtsGateProxy_query__E__mangled__                          
UNDEFED   ti_sysbios_hal_Hwi_HwiProxy_Module__startupDone__S__mangled__             
UNDEFED   ti_sysbios_hal_Hwi_HwiProxy_Object__delete__S__mangled__                  
UNDEFED   ti_sysbios_hal_Hwi_HwiProxy_Params__init__S__mangled__                    
UNDEFED   ti_sysbios_hal_Hwi_HwiProxy_disableInterrupt__E__mangled__                
UNDEFED   ti_sysbios_hal_Hwi_HwiProxy_enableInterrupt__E__mangled__                 
UNDEFED   ti_sysbios_hal_Hwi_HwiProxy_getStackInfo__E__mangled__                    
UNDEFED   ti_sysbios_hal_Hwi_HwiProxy_startup__E__mangled__                         
UNDEFED   ti_sysbios_hal_Hwi_HwiProxy_switchFromBootStack__E__mangled__             
UNDEFED   ti_sysbios_hal_Hwi_disableInterrupt__E__mangled__                         
UNDEFED   ti_sysbios_hal_Hwi_enableInterrupt__E__mangled__                          
UNDEFED   ti_sysbios_hal_Hwi_getStackInfo__E__mangled__                             
UNDEFED   ti_sysbios_hal_Hwi_startup__E__mangled__                                  
UNDEFED   ti_sysbios_hal_Hwi_switchFromBootStack__E__mangled__                      
UNDEFED   ti_sysbios_heaps_HeapMem_Module_GateProxy_Handle__label__S__mangled__     
UNDEFED   ti_sysbios_heaps_HeapMem_Module_GateProxy_Object__delete__S__mangled__    
UNDEFED   ti_sysbios_heaps_HeapMem_Module_GateProxy_Params__init__S__mangled__      
UNDEFED   ti_sysbios_heaps_HeapMem_Module_GateProxy_query__E__mangled__             
UNDEFED   ti_sysbios_knl_Clock_TimerProxy_Module__startupDone__S__mangled__         
UNDEFED   ti_sysbios_knl_Clock_TimerProxy_startup__E__mangled__                     
UNDEFED   ti_sysbios_knl_Task_SupportProxy_Module__startupDone__S__mangled__        
UNDEFED   ti_sysbios_knl_Task_SupportProxy_getStackAlignment__E__mangled__          
UNDEFED   ti_sysbios_knl_Task_SupportProxy_start__E__mangled__                      
UNDEFED   ti_sysbios_knl_Task_SupportProxy_swap__E__mangled__                       
UNDEFED   xdc_runtime_Main_Module_GateProxy_Handle__label__S                        
UNDEFED   xdc_runtime_Main_Module_GateProxy_Object__delete__S                       
UNDEFED   xdc_runtime_Main_Module_GateProxy_query__E                                
UNDEFED   xdc_runtime_Memory_HeapProxy_Handle__label__S__mangled__                  
UNDEFED   xdc_runtime_Memory_HeapProxy_Object__delete__S__mangled__                 
UNDEFED   xdc_runtime_System_Module_GateProxy_Handle__label__S__mangled__           
UNDEFED   xdc_runtime_System_Module_GateProxy_Object__delete__S__mangled__          
UNDEFED   xdc_runtime_System_Module_GateProxy_query__E__mangled__                   
UNDEFED   xdc_runtime_System_SupportProxy_abort__E                                  
UNDEFED   xdc_runtime_System_SupportProxy_exit__E                                   
UNDEFED   xdc_runtime_Timestamp_SupportProxy_get64__E__mangled__                    
UNDEFED   xdc_runtime_Timestamp_SupportProxy_getFreq__E__mangled__                  
UNDEFED   xdc_runtime_Timestamp_get32__E__mangled__                                 
UNDEFED   xdc_runtime_Timestamp_get64__E__mangled__                                 
UNDEFED   xdc_runtime_Timestamp_getFreq__E__mangled__                               

[823 symbols]
